:020000040800F2
:1000000000000110FD7C03084D500308F9D70008DB
:10001000017E0308017E0308017E03080000000042
:100020000000000000000000000000005550030820
:10003000515003080000000049500308FDD000089B
:10004000017E0308017E0308017E0308017E030888
:10005000017E0308017E030869D8000895D90008CD
:1000600059D900081DD90008E1D8000859B6000880
:1000700049B6000839B6000829B6000819B60008C4
:1000800005B60008F1B50008017E0308017E0308EB
:10009000017E0308017E0308017E0308A5D800083D
:1000A000017E0308017E0308017E0308017E030828
:1000B000C1C80008017E0308B1C80008017E03081A
:1000C000017E0308017E0308017E0308017E030808
:1000D000017E0308017E0308D1D1000831D1000858
:1000E0002DD80008017E030861510308017E030832
:1000F00081C80008017E030891C80008DDB500082A
:10010000017E0308017E0308A1C80008017E0308E0
:10011000017E0308017E030871CD010855CD010859
:10012000C9B50008B5B50008A1B500088DB500082F
:1001300079B50008017E0308017E0308017E0308EB
:10014000017E0308017E0308017E03080D4A0308AF
:1001500065B5000851B500083DB50008017E0308EB
:10016000017E0308017E0308017E0308017E030867
:10017000017E0308017E0308017E0308017E030857
:08018000017E0308017E030863
:0801880094780300010000005F
:1001900002020300A81D0020A41D00200000000092
:1001A00000000000F7010600B41D0020AC1D002077
:1001B00000000000A005000827000400C82300205C
:1001C0003424002000000000A605000816000800E6
:1001D0004C2400206424002000000000AA05000830
:1001E000010104005C250020882F00200000000091
:1001F0000000000008020900482F00208C2F00207A
:10020000000000003DB9000802000C00542F00203F
:10021000982F002000000000000000000A020A00E1
:10022000EC250020A42F002000000000B2050008EB
:1002300003123300F7330020C43300200000000015
:10024000BC05000825005A00F03200204A33002087
:100250000000000000000000150070007031002058
:10026000E031002000000000000000002A006000D3
:10027000B03000201031002000000000D921020819
:100280002C001000A4330020B43300200000000034
:10029000CDDE01082B0024004E3400202A3400203B
:1002A000000000009DDE01082900500050320020AF
:1002B000A0320020000000000000000003010A003E
:1002C000CC360020D836002000000000F0050008E1
:1002D0001A000800E03C0020F83C0020000000006C
:1002E000FA0500080300010078370020003D0020D7
:1002F0000000000000000000140002000041002087
:100300007C410020000000000206000826000E00CC
:10031000544400204444002000000000915302088F
:100320000B20100028420020644400200000000040
:10033000040600081F000E00B0450020844700207E
:100340000000000014060008050201009845002086
:100350009447002000000000220600080510060057
:100360000E4900207049002000000000240600080B
:100370000C002400D648002078490020000000002E
:10038000EBC701080E20EA00CA4700209C49002064
:10039000000000000122020812200C00B0470020DB
:1003A000884A0020000000002A060008020103001D
:1003B000AB470020944A002000000000ADC70108B0
:1003C0000002050098470020984A00200000000025
:1003D00000000000F90104004C4F0020504F0020A5
:1003E0000000000025B90008FD012400244F002072
:1003F000544F002000000000B5B8000806001600A9
:10040000AC4B0020784F002000000000952102082E
:10041000FB010100E84A0020904F0020000000008E
:1004200059B70008FC0109007458002060590020E9
:100430000000000025B700080A10120048580020EC
:100440006C5900200000000036060008340010003F
:10045000984F002080590020000000005121020820
:100460001E00040090590020045D002000000000E0
:100470004806000822000C00305C0020085D0020C7
:10048000000000004C0600080E020200D8620020A6
:100490002C63002000000000580600081300040030
:1004A0002463002030630020000000005C06000888
:1004B00010000300206300203463002000000000CF
:1004C0006006000828001000106300203863002038
:1004D00000000000153F0208230010000063002008
:1004E00048630020000000002D3F020819000500AD
:1004F000F862002058630020000000006406000835
:10050000F8110100F4620020606300200000000088
:100510006A06000800010400F06200206463002005
:10052000000000006C0600082F001100DC620020B3
:100530006863002000000000700600080120080029
:10054000FC680020286900200000000082060008E6
:1005500018102C00C4690020386A00200000000038
:1005600051E101080D002C00F0690020646A0020B0
:1005700000000000B5080308FE010900886C002097
:10058000C07200200000000061B700080400800075
:1005900094850020948600200000000000000000E8
:1005A00000000100000020030000C4090000190140
:1005B000282800004A01B400D60100000000000015
:1005C000000000000000000000000000000000002B
:1005D000000000000000000000000000000000001B
:1005E000000000000000000000000000000001000A
:1005F000040101006C16000000007E05EA05B40548
:10060000320003002B21231E6400020000000100C1
:100610000A012900000000000000010000000005A0
:1006200000000000200003010000000000010005A0
:10063000454C4C30000000300100005A0000000022
:1006400090012C01C800640000000100C800141EC5
:10065000010064002C0128000000000008000000D8
:1006600000010500000028010000040090010000C6
:10067000000000000000000000000000000000007A
:0A0680000000E8036400040A000112
:10068A005001000007000000020000000000000006
:10069A00000000000102030406070809FF00000029
:1006AA000101000000BC03083CE40308000000004C
:1006BA000000000010BC030818BC0308000000007A
:1006CA00012000001CBC030824BC03080000000031
:1006DA000140000028BC030888DA03080000000073
:1006EA000120000034BC030840BC030800000000DD
:1006FA000400000044BC030850BC030800000000CA
:10070A000400000054BC0308F0C8030800000000FD
:10071A0001000000020100000000803F0000803F4D
:10072A000000803F00000000000000000000000000
:10073A00F89603080508040000000000CCAE030880
:10074A0074AA0308B8AE030800000000249703083F
:10075A0005080A0000000000CCAE030874AA0308CA
:10076A0078B3030800000000FFFFFFFF2D202D2DA6
:10077A00202D2D2D2D202D2D2D2D000000000000C7
:10078A00000000000000000000000000000000005F
:10079A00010203040102030406070809000101011A
:1007AA000100000098C103080000000000000000DA
:1007BA00BDC70108A0860100040000000000000077
:1007CA00000000000000000000000000000000001F
:1007DA00000000000000000030E7030854E00308AE
:1007EA0000000000F53601087D0000000600000048
:1007FA0000000000000000000000000000000000EF
:10080A0000000000000000000000000098E003085B
:10081A00000000000000000081050108E803000054
:10082A0003000000000000000000000000000000BB
:10083A0000000000000000000000000000000000AE
:10084A00A0E003080000000000000000DD14030817
:10085A001027000003000000000000000000000054
:10086A00000000000000000000000000000000007E
:10087A0000000000ACE003080000000035D00208C8
:10088A0095DF0008204E000005000000000000006F
:10089A00000000000000000000000000000000004E
:1008AA00000000000000000030C303080000000040
:1008BA000000000045DA00081027000001000000CF
:1008CA00000000000000000000000000000000001E
:1008DA00000000000000000000000000B0E0030873
:1008EA000000000000000000F1B60008E803000064
:1008FA0005000000000000000000000000000000E9
:10090A0000000000000000000000000000000000DD
:10091A00BCE00308000000000000000009CA01084A
:10092A00204E00000300000000000000000000004C
:10093A0000000000000000000000000000000000AD
:10094A0000000000CCE003080000000000000000E6
:10095A0011C80108204E000003000000000000003A
:10096A00000000000000000000000000000000007D
:10097A000000000000000000DCE0030800000000A6
:10098A00000000005D090108400D0300030000009B
:10099A00000000000000000000000000000000004D
:1009AA0000000000000000000000000038C3030837
:1009BA00000000000000000005C002081027000027
:1009CA00030000000000000000000000000000001A
:1009DA00000000000000000000000000000000000D
:1009EA00ECE003080000000000000000ED6D0308C1
:1009FA00A0860100010000000000000000000000C5
:100A0A0000000000000000000000000000000000DC
:100A1A000000000044C303080000000000000000BA
:100A2A00C10B0108A00F0000010000000000000037
:100A3A0000000000000000000000000000000000AC
:100A4A000000000000000000A8C303080000000026
:100A5A00000000005D660208102700000100000087
:100A6A00000000000000000000000000000000007C
:100A7A0000000000000000000000000040E0030841
:100A8A000000000000000000512C03081A41000079
:100A9A00010000000000000000000000000000004B
:100AAA00000000000000000000000000000000003C
:100ABA00F4E003080000000000000000A569030834
:100ACA00400D0300000000000000000000000000CC
:100ADA00000000000000000000000000000000000C
:100AEA0000000000FCE00308000000000000000015
:100AFA0061690308400D03000000000000000000C7
:100B0A0000000000000000000000000000000000DB
:100B1A00000000000000000004E1030800000000DB
:100B2A000000000025820208A086010003000000E0
:100B3A0000000000000000000000000000000000AB
:100B4A0000000000000000000000000000FFFF009D
:100B5A0000000000AA550501000001AA550B01007A
:100B6A0000AA5507010000AA55090200000000006A
:100B7A0001000000C012AA5503009F0001010100F4
:100B8A000D7902080000000074060020CCE2030878
:100B9A00000000000000000000000000000000004B
:100BAA003CE403080000000000000000E00600200A
:100BBA000400000070E203080C00000091800208A3
:100BCA00C40A00200000000090E103080C000000A5
:100BDA00B9800208B80A002000000000ECE203080D
:100BEA000800000000000000AC0A00200400000019
:100BFA00DCE203080C000000B5790208A00A002014
:100C0A00000000007CE1030803000000E92A030851
:100C1A00940A002000000000E4E203080300000038
:100C2A00E92A0308880A00200000000080E103087E
:100C3A0001000000000000000000000000000000A9
:100C4A00000000000D00000000000000000000008D
:100C5A0000000000CCE203080000000000000000D1
:100C6A0000000000000000003CE40308000000004F
:100C7A0000000000E00600200400000008E203086B
:100C8A0003000000517E02087C0A002008000000D0
:100C9A00DCE203080C000000B5790208A00A002073
:100CAA00000000007CE1030803000000E92A0308B1
:100CBA00940A002000000000E4E203080300000098
:100CCA00E92A0308880A00200000000080E10308DE
:100CDA000100000000000000000000000000000009
:100CEA00000000000D0000000000000000000000ED
:100CFA0000000000F4E20308000000000000000009
:100D0A0000000000000000003CE4030800000000AE
:100D1A0000000000E00600200400000010E20308C2
:100D2A0003000000E92A0308D00A0020000000009E
:100D3A0080E103080100000000000000000000003C
:100D4A0000000000000000000D000000000000008C
:100D5A00000000000000000020700020702D7200CA
:100D6A002D202D2D202D2D2D2D202D2D2D00000057
:100D7A000000000000000000000000000000000069
:100D8A00A447002088136F1701000000A64700201F
:100D9A0088136F170000000054E1030800000000E8
:100DAA0000000000000000000000000064E10308E9
:100DBA0008000000000000000C07002004000000EA
:100DCA0070E103080800000000000000000700208E
:100DDA00000000007CE1030804000000E57E020830
:100DEA00000000000000000080E10308010000008C
:100DFA0000000000000000000000000000000000E9
:100E0A000D000000000000000000000000000000CB
:100E1A00A247002088136F170100000090450020A8
:100E2A0088136F17000000006D79020800000000A7
:100E3A001807002039490020010000008CAE030881
:100E4A00924500200100000098AE03088845002062
:100E5A0002000000A0AE03085A860020000000002D
:100E6A00000000005886002000000000000000007A
:100E7A005686002000000000000000005486002072
:100E8A000000000000000000528600200000000060
:100E9A000000000050860020000000000000000052
:100EAA00F40400200000000000000000A147002018
:100EBA0002000000ACAE0308C0E103080000000015
:100ECA0000000000000000000000000064E10308C8
:100EDA0008000000000000009C0700200400000039
:100EEA0070E10308080000000000000090070020DD
:100EFA00000000007CE103080400000041790208B8
:100F0A00000000000000000080E10308010000006A
:100F1A0000000000000000000000000000000000C7
:100F2A000D000000000000000000000000000000AA
:100F3A00D0E10308000000000000000000000000EB
:100F4A0000000000E0E103080C0000003580020800
:100F5A00CC07002004000000ECE103080C000000AC
:100F6A0091790208C007002004000000F8E1030894
:100F7A000C000000F97F0208B407002000000000FE
:100F8A0004E2030803000000717E0208A80700209B
:100F9A000800000010E2030803000000E92A030821
:100FAA00D00A00200000000080E1030801000000D0
:100FBA000000000000000000000000000000000027
:100FCA000D0000000000000000000000000000000A
:100FDA0018E2030800000000000000000000000002
:100FEA000000000020E2030804000000017F02085C
:100FFA00000000000000000080E10308010000007A
:10100A0000000000000000000000000000000000D6
:10101A000D000000000000000000000000000000B9
:10102A0078E2030800000000000000000000000051
:10103A000000000088E203080C0000000000000025
:10104A002C0800200400000090E2030808000000B9
:10105A000000000020080020040000009CE20308B1
:10106A00080000000000000014080020040000002E
:10107A00A4E203080800000000000000080800209D
:10108A0004000000ACE203080800000000000000B1
:10109A00FC07002004000000B4E203080800000076
:1010AA0000000000F007002004000000BCE2030872
:1010BA000800000000000000E4070020040000000F
:1010CA00C4E203080800000000000000D80700205E
:1010DA000400000080E10308010000000000000095
:1010EA000000000000000000000000000D000000E9
:1010FA00000000000000000000000000597902080A
:10110A000000000038080020000000000000000075
:10111A00B008002000000000000000005009002074
:10112A008E45002004000000B8AE03088C4500205C
:10113A00E0150C17000000008B4500200800000095
:10114A0074AA03088A45002005000000CCAE0308F3
:10115A000000000000000000A009002001000000BB
:10116A000101D60185CB0208000000000000000042
:10117A000000803F000000000000000000000000A6
:10118A000000803F00000000000000000000000096
:10119A000000000000000000000000000000000045
:1011AA0000000000000000000000803F0000000076
:1011BA000000000000000000010000000000000024
:1011CA000000000058180020FFFFFFFFFA0000008F
:1011DA00010000000100000018E2030800000000FE
:1011EA0000000000000000000000000058EA0308A8
:1011FA0004000000CB7D020800000000000000008F
:10120A0080E1030801000000000000000000000067
:10121A0000000000000000000D00000000000000B7
:10122A0000000000000000004A4900200100C40933
:10123A0000000000484900200100C4090000000025
:10124A00464900200100C40900000000444900206A
:10125A000100C40900000000404900200100C4093F
:10126A0000000000424900200100C40900000000FB
:10127A003E4900200100C409000000003C4900204A
:10128A000100C40900000000000000000000000086
:10129A00580B0020A83600209CFF2C0100000000FB
:1012AA00FC0400200A00000078B303089E470020CF
:1012BA00E0150C1700000000FE04002008000000E2
:1012CA0074AA0308FD04002005000000CCAE030840
:1012DA00A04700200200000090B303081449002030
:1012EA000100FF7F010000000D49002002000000FC
:1012FA009CB30308BE47002003000000ACB30308F8
:10130A00BD47002003000000ACB30308BC4800201E
:10131A000000F40101000000BA4800200000F401B6
:10132A0001000000B84800200000F401010000009C
:10133A00B64800200000F40101000000B448002073
:10134A0000FF0100D4480020E803D0070A0000008B
:10135A00D2480020006401000A000000CE480020A4
:10136A0000640100CD48002000640100D348002039
:10137A00006401000A000000CC480020006401005B
:10138A000A000000D1480020006401000A000000A1
:10139A00D0480020006401000A000000CF48002065
:1013AA00006401000A000000CB48002000FF010091
:1013BA000A000000CA48002000FF01000A000000DD
:1013CA00C64700200000F40101000000C4470020C5
:1013DA000000F40101000000C24700200000F401EF
:1013EA0001000000C04700200000F40101000000D5
:1013FA00C64800201400E80301000000C448002089
:10140A00E803307501000000C348002000C801004D
:10141A00C248002000C80100C148002000C80100DD
:10142A00C0480020006401000A000000BF480020F4
:10143A0000FF01000A0000000349002000C8010063
:10144A000249002000C801000149002000C801002B
:10145A000049002000C80100FF48002000C8010020
:10146A00FE48002000C80100FD48002000C8010015
:10147A00FC48002000C80100FB48002000C8010009
:10148A007CEA0308000000000000000000000000E1
:10149A00000000008CEA03080900000000000000B8
:1014AA00FC0B00200400000094EA03080900000075
:1014BA0000000000F00B0020040000003CEE0308CE
:1014CA000900000000000000E40B002004000000F6
:1014DA009CEA03080900000000000000D80B002065
:1014EA0004000000A0EA0308090000000000000050
:1014FA00CC0B002004000000A8EA03080900000041
:10150A0000000000C00B002004000000B0EA03083D
:10151A000900000000000000B40B002004000000D5
:10152A00B8EA03080900000000000000A80B002028
:10153A000400000080E10308010000000000000030
:10154A000000000000000000000000000D00000084
:10155A00000000000000000000000000CCEB0308BF
:10156A000000000000000000000000000000000071
:10157A003CE403080000000000000000EC0000202A
:10158A0004000000D8EB03080C0000002D7E0208BE
:10159A00500C00200000000070E203080C0000005C
:1015AA00C5780208440C00200000000090E10308FE
:1015BA000C000000A9780208380C00200000000086
:1015CA00ECE2030808000000000000002C0C0020D8
:1015DA0004000000DCE203080C000000F5770208B2
:1015EA00200C002000000000DCEB030809000000CA
:1015FA0000000000140C0020040000007CE1030835
:10160A0003000000E92A0308080C0020000000007B
:10161A0080E1030801000000000000000000000053
:10162A0000000000000000000D00000000000000A3
:10163A000000000000000000E4EB030800000000C6
:10164A00000000000000000000000000F4EB0308A6
:10165A000C00000000000000680C002000000000E0
:10166A00FCEB03080A0000000000000021490020EA
:10167A000000000008EC03080A0000000000000057
:10168A00294900200000000010EC03080A000000AD
:10169A0000000000314900200000000018EC030897
:1016AA0008000000000000005C0C002000000000A0
:1016BA0080E10308010000000000000000000000B3
:1016CA0000000000000000000D0000000000000003
:1016DA00000000000000000020EC030800000000E9
:1016EA0000000000000000000000000034EC0308C5
:1016FA000C00000000000000800C00200000000028
:10170A0044EC030804000000FD8002080000000009
:10171A00000000004CEC03080C0000000000000070
:10172A00740C00200000000060EC030804000000B4
:10173A00E1800208000000000000000080E10308C8
:10174A00010000000000000000000000000000008E
:10175A00000000000D000000000000000000000072
:10176A000000000068EC0308000000000000000010
:10177A0000000000000000007CEC030807000000E5
:10178A0000000000BC0C00200000000088EC0308E8
:10179A000800000000000000B00C0020000000005B
:1017AA0094EC03080800000000000000A40C0020CC
:1017BA0000000000A0EC0308080000000000000080
:1017CA00980C002000000000ACEC030808000000A0
:1017DA00000000008C0C00200000000080E10308DB
:1017EA0001000000000000000000000000000000EE
:1017FA00000000000D0000000000000000000000D2
:10180A0000000000B8EC030800000000000000001F
:10181A00DB06002000000000C4EC03080B000000F7
:10182A0000000000340D002000000000CCEC03088A
:10183A000B00000000000000280D0020000000003E
:10184A00D8EC03080B000000000000001C0D00206B
:10185A0000000000E4EC03080B0000000000000098
:10186A00100D002000000000F0EC03080B0000003F
:10187A0000000000040D002000000000FCEC03083A
:10188A000B00000000000000F80C0020000000001F
:10189A0004ED03080B00000000000000EC0C00201F
:1018AA000000000010ED030807000000000000001F
:1018BA00E40C00200000000018ED030807000000F7
:1018CA0000000000DC0C00200000000024ED0308EA
:1018DA000B00000000000000D00C002000000000F7
:1018EA0030ED03080800000000000000C40C0020CE
:1018FA000000000080E10308010000000000000071
:10190A000000000000000000000000000D000000C0
:10191A000000000000000000000000003CED030889
:10192A0000000000000000000000000000000000AD
:10193A0050ED03080800000000000000640D0020BC
:10194A00000000005CED0308080000000000000031
:10195A00580D00200000000068ED03080800000090
:10196A00000000004C0D00200000000074ED030888
:10197A000800000000000000400D002000000000E8
:10198A0080E10308010000000000000000000000E0
:10199A0000000000000000000D0000000000000030
:1019AA0000000000000000007CED030800000000B9
:1019BA0000000000D8060020000000008CED03089B
:1019CA000B00000000000000AC0D00200000000029
:1019DA0098ED03080B00000000000000A00D002095
:1019EA0000000000A4ED030807000000000000004A
:1019FA00980D002000000000B0ED03080700000069
:101A0A0000000000900D002000000000BCED03085B
:101A1A000700000000000000880D00200000000000
:101A2A00C8ED030808000000000000007C0D00203B
:101A3A0000000000D0ED03080800000000000000CC
:101A4A00700D00200000000080E103080100000082
:101A5A00000000000000000000000000000000007C
:101A6A000D0000000000000000000000000000005F
:101A7A00D8ED03080000000000000000D80600208E
:101A8A0000000000E4ED0308070000000000000069
:101A9A00F80D002000000000ECED0308070000002C
:101AAA0000000000F00D002000000000F4ED030823
:101ABA000700000000000000E80D00200000000000
:101ACA00FCED03080700000000000000E00D002004
:101ADA000000000004EE03080700000000000000F8
:101AEA00D80D0020000000000CEE030807000000DB
:101AFA0000000000D00D00200000000014EE0308D2
:101B0A000700000000000000C80D002000000000CF
:101B1A001CEE03080700000000000000C00D0020B2
:101B2A000000000024EE0308070000000000000087
:101B3A00B80D00200000000080E103080100000049
:101B4A00000000000000000000000000000000008B
:101B5A000D0000000000000000000000000000006E
:101B6A0000000000417A0208000E0020BC47002055
:101B7A001B000000BCB30308AF4700200A32010073
:101B8A00AE47002001FA0100AA47002000C8010060
:101B9A00A8470020E803D00701000000454C4C4547
:101BAA00300000003178020800000000DC0E00203E
:101BBA00917E0208897C0208B80F0020577A020831
:101BCA000000000058100020E97A0208B97A0208D9
:101BDA00E4100020757B0208BD7B020884110020F6
:101BEA00C8480020010301008D7A0208697A0208B8
:101BFA009C120020197B0208198102082813002070
:101C0A00E97B020875810208F0130020BE48002013
:101C1A00010301002CEE0308000000000000000090
:101C2A00000000000000000038EE03080800000071
:101C3A0000000000101500200000000040EE03081C
:101C4A000700000000000000081500200000000046
:101C5A0050EE0308070000000000000000150020F5
:101C6A00000000005CEE030807000000000000000E
:101C7A00F81400200000000068EE03080C000000C1
:101C8A0000000000EC1400200000000074EE0308BD
:101C9A0003000000E92A0308E01400200000000005
:101CAA0080E10308010000000000000000000000BD
:101CBA0000000000000000000D000000000000000D
:101CCA0000000000000000007CEE03080000000095
:101CDA000000000000000000000000008CEE030875
:101CEA000A0000000000000088BD03080000000090
:101CFA0094EE03080A00000000000000E0BB03089D
:101D0A00000000009CEE03080A000000000000002A
:101D1A000449002000000000A4EE03080A000000A5
:101D2A00000000001C1500200000000080E10308EC
:101D3A000100000000000000000000000000000098
:101D4A00000000000D00000000000000000000007C
:101D5A0000000000ACEE03080000000000000000D4
:101D6A00000000000000000068E90308030000000A
:101D7A00E92A03083015002000000000C0EE03081D
:101D8A0003000000E92A0308000500200000000003
:101D9A00C8EE030803000000E92A030824150020FE
:101DAA000000000080E103080100000000000000BC
:101DBA000000000000000000000000000D0000000C
:101DCA00000000000000000000000000D0EE030840
:101DDA0000000000000000000000000000000000F9
:101DEA00DCEE030807000000C18102088C15002000
:101DFA000000000030E7030803000000E92A030896
:101E0A008015002000000000E8EE0308030000002F
:101E1A00E92A03087415002000000000F0EE030808
:101E2A0003000000E92A03086815002000000000EA
:101E3A00F8EE030807000000A581020860150020DB
:101E4A000000000094E2030803000000E92A0308E6
:101E5A00541500200000000004EF030803000000EE
:101E6A00E92A0308481500200000000010EF0308C3
:101E7A0003000000E92A03083C15002000000000C6
:101E8A0080E10308010000000000000000000000DB
:101E9A0000000000000000000D000000000000002B
:101EAA0000000000000000000D7A0208D97902083B
:101EBA0094150020557C02080000000048160020F6
:101ECA000000000000000000D4160020317C020847
:101EDA00DD8102084C1700201CEF030800000000F7
:101EEA0000000000000000000000000028EF0308C6
:101EFA0003000000E92A03084C1800200000000033
:101F0A0030EF030803000000E92A03084018002004
:101F1A00000000003CEF030803000000E92A030860
:101F2A00341800200000000048EF030803000000F6
:101F3A00E92A0308281800200000000050EF0308CF
:101F4A0002000000F529030800000000000000005C
:101F5A0058EF030802000000F529030801000000F9
:101F6A000000000064EF030802000000F5290308DE
:101F7A000200000000000000000000000D00000048
:101F8A0000000000000000000000000025490308CE
:101F9A00DD48030899500308000000001D460308A5
:101FAA0051470308D1470308B94603080000000057
:101FBA000000000011460308A55F03085D690308D5
:101FCA00A15F0308955F0308915F03089D5F0308FB
:101FDA00995F030805460308F945030825690308BC
:101FEA00A546030811690308FD680308E9680308A0
:101FFA00040309041201000202020040830440574C
:10200A00000201020301000009024300020100C0AC
:10201A003209040000010202010005240010010532
:10202A002401000104240202052406000107058296
:10203A00030800FF09040100020A00000007050165
:10204A00024000000705810240000000FF00000076
:10205A00791B0208FD4703082D160208614603088A
:10206A00B9490308714603088D4603085146030817
:10207A004146030800000000000000000060024022
:10208A001060024000000000000B00000000200069
:10209A0000000000000000000060024028600240CA
:1020AA0000000000060C00000000200000000000F4
:1020BA000000000000600240406002400000000092
:1020CA00100D0000000020000000000000000000C9
:1020DA00006002405860024000000000160E000036
:1020EA000000200000000000000000000060024024
:1020FA007060024000000000200F00000000200075
:10210A0000000000000000000060024088600240F9
:10211A00000000002610000000002000000000005F
:10212A000000000000600240A060024000000000C1
:10213A003011000000002000000000000000000034
:10214A0000600240B860024000000000362F000024
:10215A0000002000000000000000000000640240AF
:10216A001064024000000000003800000000400037
:10217A0000000000000000000064024028640240E1
:10218A0000000000063900000000400000000000C6
:10219A0000000000006402404064024000000000A9
:1021AA00103A00000000400000000000000000009B
:1021BA00006402405864024000000000163B000020
:1021CA00000040000000000000000000006402401F
:1021DA007064024000000000203C00000000400043
:1021EA000000000000000000006402408864024011
:1021FA00000000002644000000004000000000002B
:10220A000000000000640240A064024000000000D8
:10221A0030450000000040000000000000000000FF
:10222A0000640240B8640240000000003646000024
:10223A000000400000000000000000000000803F95
:10224A00C41B002000000000000000000000000085
:10225A000000000000000000000000000000000074
:10226A000000000000000000000000000000000064
:10227A000000000000000000000000000000000054
:10228A000000000000000000000000000000000044
:10229A000000000000000000000000000000000034
:1022AA0000000000430000000000000000000000E1
:1022BA000000000000000000000000000000000014
:1022CA0000000000430000000000000000000000C1
:1022DA0000000000000000000000000000000000F4
:1022EA0000000000430000000000000000000000A1
:1022FA0000000000000000000000000000000000D4
:10230A000000000043000000000000000000000080
:10231A0000000000000000000000000000000000B3
:10232A000000000043000000000000000000000060
:10233A000000000000000000000000000000000093
:10234A000000000043000000000000000000000040
:10235A000000000000000000000000000000000073
:10236A000000000043000000000000000000000020
:10237A000000000000000000000000000000000053
:10238A00000000002B8003080780030800000000FB
:10239A00F6EF030854EA0308C4EF0308C4EF03087E
:1023AA00C4EF0308C4EF0308C4EF0308C4EF03082B
:1023BA00C4EF0308C4EF0308C4EF0308FFFFFFFFDD
:1023CA00FFFFFFFFFFFFFFFFFFFF00000100415378
:1023DA00434949000000000000000000000000001E
:1023EA00000000000000000000000000000041534F
:1023FA0043494900000000000000000000000000FE
:10240A0000000000000000000000000000000000C2
:04241A0001000000BD
:10800000002870B51EDB0928044620DD012303EBA0
:1080100083035B00B0FBF3F2092AF8D87BB10E4E64
:10802000B4FBF3F00928CCBF57223022A6FB03E5AE
:10803000024403FB1044EB0801F8012BF0D10023AC
:108040000B7070BD2D230B7040420131DBE73030E7
:1080500001F8010BF3E700BFCDCCCCCC884230B4A3
:108060004FF001042ED301FB04F4B0FBF4F58D4274
:10807000F9D284B1AAB901E0B0FBF4F5092DCCBF67
:10808000572230222A4404FB150003F8012BB4FBCD
:10809000F1F4002CF0D100221A7030BC7047B0FB14
:1080A000F4F5092DCCBF372230222A4404FB1500F9
:1080B00003F8012BB4FBF1F4002CF0D100221A706C
:1080C00030BC70470546002AEBD1D7E703685A1C3D
:1080D00002601970704700BF2DE9F047089C2578B1
:1080E000002B804689460CBF4FF0200A4FF0300A23
:1080F000661C35B3002A29DD334601E0024698B1FB
:1081000013F8011B501E0029F8D1971E60B13D469F
:10811000013D51464046C8476B1C002BF8DC2578D2
:1081200027EAE770013055B1041B29464046C8478D
:10813000301916F8015B002DF7D1BDE8F087BDE8D6
:10814000F087002A04DC2846BDE8F0870020EBE732
:10815000571EDCE783684268D0ED037A00EB8301A9
:108160000133934281ED040A836004BF00238360DE
:1081700000EB830393ED047A036870EE277A9A424A
:10818000C0ED037A77EEC77AC0ED037A0CDA0133DB
:1081900007EE103AF8EEC76AB7EE007A87EEA60A45
:1081A000036030EE070A704707EE102AB8EEC77A70
:1081B00087EE870A704700BF90ED057A90ED004A80
:1081C000D0ED066AD0ED014AD0ED047A90ED035A65
:1081D000D0ED025AA4EE007AB0EE406AB0EE470A43
:1081E000B0EE667AA6EE247A67EEC07AA0EE457A03
:1081F000E6EE257A80ED057AC0ED067A704700BF7D
:10820000D0ED057A90ED013AD0ED003AD0ED064A76
:1082100090ED024A90ED077A90ED035A90ED086ACE
:10822000D0ED045AC0ED067AF0EE406A27EE830ADC
:10823000C0ED056AA3EEA60A80ED087AA4EE240A32
:10824000A5EE470AA5EEC60A80ED070A704700BFF3
:10825000D0ED007A90ED017A30EE670AE7EE007A11
:10826000B0EE670AC0ED007A704700BF704700BFEC
:108270000A44914214D030B40139551E41F2210212
:1082800011F8014F082380EA042004044CBF82EA5D
:1082900040004000013B80B2F7D18D42F0D130BCAC
:1082A00070474378007840EA032010FB01F04FF458
:1082B000807190FBF1F000F30F0000B2704710B531
:1082C000064C23780BB9002010BD04F0D3FD636881
:1082D000C01AD0F5FA50F6D410BD00BF981D00208A
:1082E0004FF40063838270474FF4006383827047CA
:1082F000012380F845307047BFF34F8F0549064B87
:10830000CA6802F4E0621343CB60BFF34F8F00BF33
:10831000FDE700BF00ED00E00400FA0570B4037B48
:1083200004681F2B08D9203B2021626801FA03F35F
:108330001A421CD170BC70472021226801FA03F355
:108340001A42F7D0426914495C2000FB02125168BE
:108350005689CD680868296821F001012960828961
:1083600092B222EA06028281A36070BC7047426921
:1083700009495C2000FB021251685689CD680868E3
:10838000296821F001012960828992B222EA06025D
:108390008281E36070BC7047D44B00202B4B19786E
:1083A000002951D02A4B30B41C68988800226262A0
:1083B000A5899A80284380B20129A08143D09C6876
:1083C00098896262A589284380B20229A0819A8196
:1083D00039D01C69988A6262A589284380B2032932
:1083E000A0819A822FD09C69988B6262A5892843CC
:1083F00080B20429A0819A8325D01C6A988C62627D
:10840000A589284380B20529A0819A841BD09C6A43
:10841000988D6262A589284380B20629A0819A8539
:1084200011D01C6B988E6262A589284380B20729FF
:10843000A0819A8607D0986B998F426284892143E4
:1084400089B281819A8730BC704700BFB44E00204A
:10845000B84E0020014B186804F06EBF041E0020C7
:10846000F8B5057B466903681F2D29D9A5F12004BD
:108470005F682021A1400F422A4613D01022A2405B
:10848000D960DA605A68E240D10703D5012202FAC6
:1084900004F4DC600446304604F0EAFE227B2368E4
:1084A0001F2A20D9A2F1200008215A6881401142D8
:1084B00000D0D9600422596882400A4221D1F8BD17
:1084C00020211C68A9400C422A460CD01022AA4048
:1084D00099609A601A68EA40D207DBD5012202FA55
:1084E00005F59D60D6E7082118689140014200D04B
:1084F00099600421186801FA02F2024203D09A60DE
:10850000F8BDDA60F8BDF8BD064B984202D04FF0D6
:10851000FF307047044A538B01339BB25383508B17
:1085200080B27047003800409C6C0020F8B50546CA
:10853000806816461F4610B1036882885A8341F04E
:108540008001686840F2E93401E0002C44D00389DE
:10855000013C13F0020FA4B2F7D089B2818140F23E
:10856000E93101E0002937D00389013913F0010F07
:1085700089B2F7D0838983894FF0000C4FF47A7168
:108580004FF6FF734FF0FF0E674502D11DE0994291
:1085900019D004890139A40789B2F8D5A0F80CE0F4
:1085A0004FF47A7102E0A1B299420CD00289D2074D
:1085B00001F1FF34F7D5828992B20EB132700136E3
:1085C0000CF1010CE0E7FFF79FFFAB6813B11A68ED
:1085D0009B8813830120F8BDFFF796FF6868CAE700
:1085E00038B504460D46FFF76AFE246808B104F06A
:1085F0008DFC054B00221A7049215B782A462046E3
:10860000FFF794FF012038BD981D002070B58368E6
:108610000446164613B11A689B885383606840F27B
:10862000E93301E0002B30D00589013B15F0020F42
:108630009BB2F7D089B2818140F2E93300E023B3E5
:108640000289013B12F0010F9BB2F8D0838940F2FE
:10865000E93300E0EBB10189013B11F0020F9BB25D
:10866000F8D0B6B2868140F2E93300E08BB10289DE
:10867000013B12F0010F9BB2F8D08389A36813B1BC
:108680001A689B881383012070BDFFF73DFF606867
:10869000DDE7FFF739FFF1E70378022B01D0002077
:1086A000704770B5836801F07F0113B11C689B8827
:1086B000638304461646406840F2E93301E0002B2C
:1086C00030D00589013B15F0020F9BB2F7D089B27B
:1086D000818140F2E93300E023B30289013B12F0CB
:1086E000010F9BB2F8D0838940F2E93300E0EBB18F
:1086F0000189013B11F0020F9BB2F8D0B6B286811E
:1087000040F2E93300E08BB10289013B12F0010F26
:108710009BB2F8D08389A3685BB11A689B881383E6
:10872000012070BDFFF7F0FE6068DDE7FFF7ECFEAB
:10873000F1E7012070BD00BF2DE9F04F87B090F840
:1087400055300390002B40F07985039BBF4CC04D02
:10875000DFF804931033184680226B210293FFF751
:108760009BFFBC48DFF8F4E24FF0640A4FF0100CB6
:108770004FF47A76D9F80430C3F30803002B40F0A5
:108780005B84EFF31183002B40F0568421688268EC
:1087900000BF23689942F9D12F6806FB07F39B1AA3
:1087A000B3FBF7F306FB013101270191D9F804303F
:1087B000C3F30803002B40F00584EFF31183002B73
:1087C00040F000842368816800BF22689342F9D199
:1087D000D5F800B006FB0BF2521AB2FBFBF206FB17
:1087E0000323019A9B1AB3F57A7FDFD3BAF1010A0A
:1087F000C0D1072268210298DFF85C92954EFFF7FE
:108800004BFFDFF858C24FF0640A4FF010084FF4E6
:108810007A77D9F80430C3F30803002B40F0F083D3
:10882000EFF31183002B40F0EB832168B26800BFA7
:1088300023689942F9D1286807FB00F39B1AB3FB20
:10884000F0F307FB013101200191D9F80430C3F3A3
:108850000803002B40F09983EFF31183002B40F0C5
:1088600094832368B16800BF22689342F9D1D5F898
:1088700000B007FB0BF2521AB2FBFBF207FB03231B
:10888000019A9B1AB3F57A7FDFD3BAF1010AC0D1FE
:1088900052466B210298DFF8C091FFF7FDFE6D484C
:1088A000DFF8B8E14FF0640A4FF0100C4FF47A761D
:1088B000D9F80430C3F30803002B40F06984EFF3C8
:1088C0001183002B40F064842168826800BF236814
:1088D0009942F9D12F6806FB07F39B1AB3FBF7F314
:1088E00006FB013101270191D9F80430C3F30803D5
:1088F000002B40F02D83EFF31183002B40F02883F1
:108900002368816800BF22689342F9D1D5F800B08E
:1089100006FB0BF2521AB2FBFBF206FB0323019A91
:108920009B1AB3F57A7FDFD3BAF1010AC0D10122D5
:108930006B210298DFF82091FFF7AEFE4548DFF883
:108940001CE14FF00F0A4FF0100C4FF47A76D9F873
:108950000430C3F30803002B40F0FD83EFF31183D1
:10896000002B40F0F8832168826800BF2368994299
:10897000F9D12F6806FB07F39B1AB3FBF7F306FB4D
:10898000013101270191D9F80430C3F30803002B0A
:1089900040F0C182EFF31183002B40F0BC822368CA
:1089A000816800BF22689342F9D1D5F800B006FB78
:1089B0000BF2521AB2FBFBF206FB0323019A9B1A3D
:1089C000B3F57A7FDFD3BAF1010AC0D1039B0298D5
:1089D00093F84F30DFF88090042B34BF18221A220E
:1089E0001B21FFF759FE1B48DFF870E04FF00F0A1C
:1089F0004FF0100C4FF47A76D9F80430C3F3080323
:108A0000002B40F0FE83EFF31183002B40F0F9833D
:108A10002168826800BF23689942F9D12F6806FB5C
:108A200007F39B1AB3FBF7F306FB01310127019112
:108A3000D9F80430C3F30803002B40F04F82EFF362
:108A40001183002B40F04A820AE000BF306A002008
:108A5000346A002010E000E000ED00E02C6A002005
:108A60002368816800BF22689342F9D1D5F800B02D
:108A700006FB0BF2521AB2FBFBF206FB0323019A30
:108A80009B1AB3F57A7FD3D3BAF1010AB4D1182275
:108A90001C210298DFF8E892FFF7FEFDB648DFF8E8
:108AA000DCE24FF00F0A4FF0100C4FF47A76D9F851
:108AB0000430C3F30803002B40F08783EFF31183E6
:108AC000002B40F082832168826800BF23689942AE
:108AD000F9D12F6806FB07F39B1AB3FBF7F306FBEC
:108AE000013101270191D9F80430C3F30803002BA9
:108AF00040F0D781EFF31183002B40F0D28123683F
:108B0000816800BF22689342F9D1D5F800B006FB16
:108B10000BF2521AB2FBFBF206FB0323019A9B1ADB
:108B2000B3F57A7FDFD3BAF1010AC0D1039B029873
:108B300093F84E20DFF848921A21FFF7ADFD8E48DA
:108B4000DFF838E24FF00F0A4FF0100C4FF47A764E
:108B5000D9F80430C3F30803002B40F0A682EFF3EA
:108B60001183002B40F0A1822168826800BF236836
:108B70009942F9D12F6806FB07F39B1AB3FBF7F371
:108B800006FB013101270191D9F80430C3F3080332
:108B9000002B40F06981EFF31183002B40F06481DA
:108BA0002368816800BF22689342F9D1D5F800B0EC
:108BB00006FB0BF2521AB2FBFBF206FB0323019AEF
:108BC0009B1AB3F57A7FDFD3BAF1010AC0D1039BB8
:108BD000029893F85020DFF8A8911921FFF75CFD67
:108BE0006548DFF898E14FF0640A4FF0100C4FF43D
:108BF0007A76D9F80430C3F30803002B40F03982A9
:108C0000EFF31183002B40F034822168826800BFAB
:108C100023689942F9D12F6806FB07F39B1AB3FB2F
:108C2000F7F306FB013101270191D9F80430C3F3B2
:108C30000803002B40F0FB80EFF31183002B40F082
:108C4000F6802368816800BF22689342F9D1D5F885
:108C500000B006FB0BF2521AB2FBFBF206FB032339
:108C6000019A9B1AB3F57A7FDFD3BAF1010AC0D11A
:108C7000102237210298DFF80891FFF70DFD3E48DA
:108C8000DFF8F8E04FF00F0A4FF0100C4FF47A764F
:108C9000D9F80430C3F30803002B40F04082EFF30F
:108CA0001183002B40F03B822168826800BF23685B
:108CB0009942F9D12F6806FB07F39B1AB3FBF7F330
:108CC00006FB013101270191D9F80430C3F30803F1
:108CD000002B40F08F80EFF31183002B40F08A804F
:108CE0002368816800BF22689342F9D1D5F800B0AB
:108CF00006FB0BF2521AB2FBFBF206FB0323019AAE
:108D00009B1AB3F57A7FDFD3BAF1010AC0D13821BB
:108D10000298DFF86C80194F0122FFF7BDFC16495D
:108D20004FF00F094FF0100E4FF47A70D8F804305E
:108D3000C3F30803002B40F0D481EFF31183002B21
:108D400040F0CF8122688E6800BF23689A42F9D133
:108D5000D5F800C000FB0CF39B1BB3FBFCF300FB3E
:108D6000023301930126D8F80430C3F308032BBB68
:108D7000EFF3118313BB05E010E000E02C6A002044
:108D800000ED00E02368D1F808A000BF22689342FC
:108D9000F8D1D5F800B000FB0BFCACEB0A0CBCFB27
:108DA000FBFC00FB03C3019A9B1AB3F57A7FDAD36D
:108DB000B9F10109BAD107B0BDE8F08FEFF3118A1C
:108DC0008EF312888A680B68DB0344BF3E608A68B2
:108DD0002368D7F800C05FFA8AFA8AF31188D5F8B9
:108DE00000A09C4400FB0AF39B1AB3FBFAF300FBC0
:108DF0000C33D8E7EFF311888CF31288816803688D
:108E0000DB0344BFCEF8007081682368DEF80020E1
:108E10005FFA88F888F31188D5F800801A4406FBB9
:108E200008F35B1AB3FBF8F306FB023367E7EFF3D3
:108E300011888CF3128881680368DB0344BFCEF885
:108E4000007081682368DEF800205FFA88F888F3F4
:108E50001188D5F800801A4406FB08F35B1AB3FBAF
:108E6000F8F306FB0233FBE6EFF311888CF312886C
:108E700081680368DB0344BFCEF800708168236813
:108E8000DEF800205FFA88F888F31188D5F80080B2
:108E90001A4406FB08F35B1AB3FBF8F306FB023334
:108EA0008DE6EFF311888CF3128881680368DB0389
:108EB00044BFCEF8007081682368DEF800205FFAB6
:108EC00088F888F31188D5F800801A4406FB08F367
:108ED0005B1AB3FBF8F306FB02331FE6EFF31188CE
:108EE0008CF3128881680368DB0344BFCEF80070FE
:108EF00081682368DEF800205FFA88F888F311881B
:108F0000D5F800801A4406FB08F35B1AB3FBF8F3AC
:108F100006FB0233B3E5EFF311888CF31288816806
:108F20000368DB0344BFCEF8007081682368DEF875
:108F300000205FFA88F888F31188D5F800801A4479
:108F400006FB08F35B1AB3FBF8F306FB023335E5C7
:108F5000EFF311888CF3128881680368DB0344BF48
:108F6000CEF8007081682368DEF800205FFA88F888
:108F700088F31188D5F800801A4406FB08F35B1AC1
:108F8000B3FBF8F306FB0233C9E4EFF3118E88F369
:108F90001288B1683368DB0344BFCCF80000B168C5
:108FA0002368DCF800205FFA8EFE8EF31188D5F876
:108FB00000E01A4407FB0EF35B1AB3FBFEF307FB5A
:108FC00002335DE4EFF311888CF312888168036843
:108FD000DB0344BFCEF8007081682368DEF8002010
:108FE0005FFA88F888F31188D5F800801A4406FBE8
:108FF00008F35B1AB3FBF8F306FB0233FFF7F1BB90
:10900000EFF3118288F31288B0683368D90303D56F
:109010000123CCF80030B0682368DCF80010D2B22D
:1090200082F311882A68194407FB02F31B1AB3FB69
:10903000F2F307FB013106E4EFF311828CF312889F
:1090400087680368D90303D50123CEF80030876809
:109050002368DEF80010D2B282F311882A6819441E
:1090600006FB02F3DB1BB3FBF2F306FB0131FFF758
:109070009BBBEFF311828CF3128887680368D903D6
:1090800003D50123CEF8003087682368DEF800108E
:10909000D2B282F311882A68194406FB02F3DB1B63
:1090A000B3FBF2F306FB0131BDE5EFF311828CF364
:1090B000128887680368D90303D50123CEF80030EE
:1090C00087682368DEF80010D2B282F311882A681C
:1090D000194406FB02F3DB1BB3FBF2F306FB013181
:1090E00050E5EFF311868EF31288D1F808C00B68B3
:1090F000DA0303D501233B60D1F808C023683A683E
:10910000F6B286F311882E681A4400FB06F3A3EB2F
:109110000C03B3FBF6F300FB0233019322E6EFF3FB
:1091200011828CF3128887680368D90303D5012361
:10913000CEF8003087682368DEF80010D2B282F3E0
:1091400011882A68194406FB02F3DB1BB3FBF2F318
:1091500006FB0131B6E5EFF311828CF312888768C4
:109160000368D90303D50123CEF80030876823684C
:10917000DEF80010D2B282F311882A68194406FB87
:1091800002F3DB1BB3FBF2F306FB0131FFF7F9BB84
:10919000EFF311828CF3128887680368D90303D533
:1091A0000123CEF8003087682368DEF80010D2B2C1
:1091B00082F311882A68194406FB02F3DB1BB3FB18
:1091C000F2F306FB0131FFF78DBBEFF311828CF355
:1091D000128887680368D90303D50123CEF80030CD
:1091E00087682368DEF80010D2B282F311882A68FB
:1091F000194406FB02F3DB1BB3FBF2F306FB013160
:109200006FE4EFF311828CF3128887680368D90347
:1092100003D50123CEF8003087682368DEF80010FC
:10922000D2B282F311882A68194406FB02F3DB1BD1
:10923000B3FBF2F306FB0131FFF7F8BB1C09013C5D
:10924000032C03F00F0300F29A80654A32F81400F1
:1092500040FA03F2D20740F19280012505FA03F3A8
:10926000013B18402EF0C6FB5E4B5F4F1E5D06446F
:1092700017EBC60400F0838057F83600B4F804E01A
:10928000026912EA0E027FF460AA00F13F4303F57F
:109290007E035649E2719B0ACB5C03F01F025B0917
:1092A0002021032B05FA02F2A17170D0042B00F0EB
:1092B0009180022B00F0898004A90025CDF810E0F0
:1092C000059518F0DFFEA088039A494BD360B0FAE9
:1092D00080F0C0F11F00431C56D0C3B203F0FC0E57
:1092E0000EF1804E0EF59C3E03F00302910057F8FC
:1092F0003630DEF808603F4FDFF808C10F228A40A1
:1093000026EA0202039E03F13F430C3647F8206031
:1093100003F57E03CEF80820C3F38722DEF8083079
:10932000354F8A4001261A4306FA00F3CEF808208A
:109330007B613968DFF8D0E0DA4311403960796841
:1093400011407960396819433960B9681140B960D2
:10935000F9680A40FA60DCF80070284A1F43115C83
:10936000CCF800701EF80100F02815DC002B3FF44B
:10937000ECA921490A6813430B60FFF7E6B9039A89
:109380001B4BD360FFF7E1B901238340EEE71C4993
:109390000B6C1A430A648FE70A4404A8137C8DF807
:1093A0001030F02203238DF811308DF812508DF813
:1093B00013600EF8012018F0A5FCA388B3FA83F31C
:1093C000C3F11F0306FA03F3D0E70D494B6C1A43B0
:1093D0004A6471E70A490B6B1A430A636CE700BFE2
:1093E0003CB5030838B50308EC6A00208CAF0308CD
:1093F000F1820008BC1D0020003C01405091030890
:1094000000380240083C0140FC1D00202DE9F04FCF
:10941000AC4A436983B09342019000F0A281AA490B
:109420008B420CBF282130211A88A84CDFF8A88273
:10943000A74E22F040021204120C1A801A8892B22F
:1094400022F03802114319801A8892B242F0400289
:109450001A8003F00FFDDFF884E29E49844610274E
:109460004FF47A750120DEF80430C3F30803002BB3
:1094700040F03681EFF31183002B40F031812368F7
:10948000D1F8089000BF22689342F8D1D8F800A024
:1094900005FB0AF2A2EB0902B2FBFAF205FB032379
:1094A0009C45E0D0019D2846FFF746F9AB6913B112
:1094B0001A689B885383019B586940F2E93302E0A4
:1094C000002B00F046810289013B12F0020F9BB293
:1094D000F6D06A23838140F2E93302E0002B00F0EA
:1094E00038810289013B12F0010F9BB2F6D08389CB
:1094F00040F2E93302E0002B00F030810289013BA9
:1095000012F0020F9BB2F6D01023838140F2E933B0
:1095100002E0002B00F022810289013B12F0010FD2
:109520009BB2F6D08389019B9B6913B11A689B8813
:109530001383DFF8A8916748654F4FF0640A4FF036
:10954000100E4FF47A75D9F80430C3F30803002BDA
:1095500040F0E480EFF31183002B40F0DF802168BE
:10956000826800BF23689942F9D1D8F8006005FBF2
:1095700006F39B1AB3FBF6F305FB013101260091BC
:10958000D9F80430C3F30803002B63D1EFF3118340
:10959000002B5FD12368816800BF22689342F9D114
:1095A000D8F800B005FB0BF2521AB2FBFBF205FB38
:1095B0000323009A9B1AB3F57A7FE1D3BAF1010A2B
:1095C000C1D1019B3F4A5B69934207D0DFF8F8A005
:1095D000534514BF4FF0080A4FF0000A1A883D4D5A
:1095E0003B4F22F040021204120C1A801A8892B2E9
:1095F00022F038024AEA020AA3F800A01A8892B2BE
:1096000042F040021A8003F035FCDFF8D0C08146FA
:109610004FF0100E4FF47A760120DCF80430C3F3DB
:109620000803002B31D1EFF3118373BB2368A968C2
:1096300000BF22689342F9D1D8F800A006FB0AF2D5
:10964000521AB2FBFAF206FB03239945E5D003B0A8
:10965000BDE8F08FEFF3118C8EF3128881680368F8
:10966000DA0344BF3E60816823683A685FFA8CFC85
:109670008CF31188D8F800C01A4405FB0CF35B1A70
:10968000B3FBFCF305FB023393E7EFF311818EF399
:109690001288D5F808A02B68DB0344BF3860D5F8E2
:1096A00008A023683A68C9B281F31188D8F800107D
:1096B0001A4406FB01F3A3EB0A03B3FBF1F306FB29
:1096C0000233C2E700380040003C0040306A00200E
:1096D0002C6A002010E000E0346A002000ED00E079
:1096E000EFF3118987F31288D1F808A00B68DB0328
:1096F00044BF3060D1F808A0236832685FFA89F966
:1097000089F31188D8F800901A4405FB09F3A3EBFC
:109710000A03B3FBF9F305FB0233C1E6EFF3118251
:109720008EF3128886680368D90302D501233B6053
:10973000866823683968D2B282F31188D8F800208D
:10974000194405FB02F39B1BB3FBF2F305FB01314C
:1097500014E7FEF7D9FE019B5869C9E6FEF7D4FE6F
:10976000E1E6282160E600BFF0B5876983B00646D0
:1097700017B13B68BA885A837069DFF8A4E083891F
:10978000C3244FF47A734FF0060C6D464FF6FF7109
:109790000EF1010E03E0013B9BB28B4220D0028907
:1097A0009207F8D5A3B283814FF47A7302E0A3B293
:1097B0008B4215D00289D20703F1FF34F7D5828995
:1097C00092B20DB12A700135BCF1000F0BD00CF133
:1097D000FF3CFF24BEF1000FE1D09EF80040D7E728
:1097E000FEF792FEB76917B13B68BA881A839DF8F5
:1097F00005009DF801509DF802109DF803409DF86A
:1098000004209DF8063041EA052143EA002342EA9C
:109810000422012031877287B38703B0F0BD00BFF7
:1098200068910308037C022B01D000207047F0B53B
:10983000836983B013B11A689B885383044640F24E
:10984000E933406901E0002B58D00289013B12F056
:10985000020F9BB2F7D0C323838140F2E93301E0CA
:10986000002B4BD00289013B12F0010F9BB2F7D0C5
:10987000838983894FF0060E4FF47A736E464FF654
:10988000FF71FF2703E0013B9BB28B4233D002897B
:109890009507F8D587814FF47A7302E0ABB28B421B
:1098A00029D00289D20703F1FF35F7D5828992B218
:1098B0000EB132700136BEF1010EE8D1A36913B1C9
:1098C0001A689B8813839DF804009DF800609DF83A
:1098D00001109DF802509DF803209DF8053041EAE3
:1098E000062143EA002342EA0522012021876287FC
:1098F000A38703B0F0BDFEF707FEDFE7FEF704FE27
:109900006069B6E7037A022B01D000207047F0B5FA
:10991000036983B013B11A689B885383044640F2ED
:10992000E933C06801E0002B58D00289013B12F0F6
:10993000020F9BB2F7D0BB23838140F2E93301E0F1
:10994000002B4BD00289013B12F0010F9BB2F7D0E4
:10995000838983894FF0060E4FF47A736E464FF673
:10996000FF71FF2703E0013B9BB28B4233D002899A
:109970009507F8D587814FF47A7302E0ABB28B423A
:1099800029D00289D20703F1FF35F7D5828992B237
:109990000EB132700136BEF1010EE8D1236913B168
:1099A0001A689B8813839DF804009DF800609DF859
:1099B00001109DF802509DF803209DF8053041EA02
:1099C000062143EA002342EA05220120E1822283A4
:1099D000638303B0F0BDFEF797FDDFE7FEF794FD6C
:1099E000E068B6E7427A02B9704710B504460368EA
:1099F000406804F10A0198470023637210BD00BF5C
:109A0000437A5A1C0344D2B242729972037A934247
:109A100000D802B9704710B504460368406804F1E5
:109A20000A0198470023637210BD00BF50B30123A1
:109A3000302803FA01F122D0312820D032281ED05C
:109A400033281CD034281ED035281CD020281AD00A
:109A5000212818D0102812D0112810D012280ED08A
:109A600013280CD014280ED015280CD0162801D09D
:109A7000172806D111F0030018BF012070474A07CC
:109A800003D1002070478B07FBD00120704700BF37
:109A9000302829D0312829D0322829D0332829D07C
:109AA000342829D0352829D0202829D0212829D088
:109AB000102829D0112829D0122829D0132829D0DC
:109AC000142829D0152829D0162805D0172808BF12
:109AD0000F2302D0002070470E23114A03EB4303EB
:109AE000134493F8220070470023F6E70123F4E7BC
:109AF0000223F2E70323F0E70423EEE70523ECE774
:109B00000623EAE70723E8E70823E6E70923E4E773
:109B10000A23E2E70B23E0E70C23DEE70D23DCE773
:109B20005091030870B5448806460D46C4F30B04F3
:109B30002246002128462FF09BFA3369094A9342B6
:109B400009D3094A934206D2224628461946BDE85F
:109B500070402FF068BA23B121462846BDE8704016
:109B6000184770BDA00500088A06000838B5054CE6
:109B7000054DAC4200D338BD61682046FFF7D2FFE7
:109B80001434F6E790010008A0050008064B0749C9
:109B90008B4202D30023184670471A88C2F30B0287
:109BA0009042F8D01433F3E790010008A0050008B4
:109BB000024A136823EA0000106070472463002003
:109BC000F8B5174D2B78A52B28D16B78BE2B25D156
:109BD000022229464FF6FF70FEF74AFB114FAC1CDC
:109BE00022884AB1A618BE4218D2052A16D92146A3
:109BF000FEF73EFB3446F3E721460222FEF738FB30
:109C00000222A118FEF734FB0634074B641B1C80AC
:109C100041F60F53C31A58425841F8BD0020F8BD11
:109C20000040000800800008463500200378202B03
:109C3000024600F10100F9D0092BF7D02D2B2CD0D2
:109C40002B2B03BF5378B7EE000A0246B7EE000A8B
:109C5000A3F13001C8B209289FED467A10D8F2EE80
:109C6000046A07EE901AF8EEE77A12F8013FE7EE81
:109C7000267AA3F13001C8B20928B0EE677AF0D98C
:109C80002E2B4CD003F0DF03452B0BD0F7EE007AE0
:109C900067EE276A20EE260A70475378BFEE000A67
:109CA0000246D5E710B451782D2959D02B290ABF87
:109CB0009178501C901C0024A1F13003092B53D83B
:109CC000002303EB830301EB430310F8011FA1F111
:109CD0003002092AA3F13003F3D9B3F59A7F28BFE4
:109CE0004FF49A73072B42D9DFED236A1A46F7EE39
:109CF000007A083A072A67EEA67AFAD803F0070333
:109D00002BB1F2EE046A013B67EEA67AFBD124B3D5
:109D1000C7EE276A5DF8044B20EE260A7047537899
:109D2000A3F13001C8B2092802F10102AAD8F2EE6B
:109D3000046AF0EE665A07EE901AF8EEE77A12F827
:109D4000013F87EEA66AA3F13001C8B2092866EE8A
:109D5000A56A37EE067AEED994E767EE276AD9E767
:109D6000901C91780124A7E7F7EE007ACFE7F7EE91
:109D7000007AC5E70000000020BCBE4CB5EEC00A6A
:109D8000DFED317AF1EE10FACCBF30EE270A30EE7B
:109D9000670ADFED2E7A20EE270A30B5FDEEC07A95
:109DA00087B017EE904A054684EAE470002303A9C1
:109DB000A0EBE4700193009302932CF081F9002C46
:109DC000ACBF20232D2303A88DF800302DF018F907
:109DD000012803A924D002282DD0032805BF302351
:109DE000684668468DF801302FF04AF968462DF034
:109DF00007F90338C4B22246694628462FF077F99E
:109E000000232B5528462DF0FBF82E22431C2A5404
:109E10000DEB0401E8182FF050F9284607B030BDCB
:109E2000302368468DF801308DF802308DF803300C
:109E30002FF026F9DAE7302368468DF801308DF8E7
:109E400002302FF01DF9D1E76F12033A00007A4477
:109E50002DE9F041064615460846B6FBF2F43CB93A
:109E600005FB1464124B1B5D00F8013BBDE8F0815B
:109E7000B4FBF2F767B90E4B05FB174705FB1464FB
:109E8000DA5D00F8012B1B5D00F8013BBDE8F081B5
:109E9000B7FBF2F8B8F1000F02D04046FFF7D8FF49
:109EA00005FB1878024B13F8082000F8012BE3E7B4
:109EB0001CBB03082DE9F04714461D460646002347
:109EC0004FF47A72204629462DF044FDDFF8488190
:109ED0004B4A4C4F88FB00310144C31782FB002ED4
:109EE000C3EB611188FB012887FB00278644464AA3
:109EF000C3EBEE2EC1EB011C82FB0E29A0EB8C0CF8
:109F00000744424A86F806C0C3EB27474FEAEE7C77
:109F100008EB010ACCEBA90C82FB07824FEAE1783F
:109F20000CEB4C0CC8EB6A18AEEBCC0EC8EB081867
:109F3000DFF8E8C086F804E0A1EB880171718CFBC2
:109F40000010F917C1EBE21240F2B55101FB127299
:109F5000C3EBE050B2F5896F4FEA800740DA40F278
:109F6000DA239A4244DCB2F5B77FB4BF4FF0000C5D
:109F70004FF0010C4FEA4C08254B08EB0C0103EBAA
:109F8000C1031FFA8CFEB3F86600224908EB0C03EC
:109F900001EBC30116310B2301E031F8020D8242BF
:109FA0001BDA013BF9D11A4BC44403EBCC0C01235F
:109FB000BCF85000B37007F2B2770132121ABE44F7
:109FC000F270A6F800E0204629464FF47A7200238A
:109FD0002DF0C0FC3281BDE8F0870133DBB2E9E748
:109FE0004FF0030EF44640F296504FF00608CCE7CF
:109FF0004FF0020EF44640F229404FF00408C4E747
:10A00000C5B3A29107452EC2ABAAAA2A73B06D169A
:10A0100050910308A091030889888888792D03113D
:10A02000104B2DE93048D3E9004554EA05020BD125
:10A030000346012200201871587198719A70DA70E5
:10A0400018801881BDE83088074B1A6814EB020BA2
:10A0500045F1000C5A466346FFF72CFF0120BDE88E
:10A06000308800BF58240020306A0020F0B40288F5
:10A070008578164FC37804794179A2F2B27202F062
:10A08000030606EB4606013D05EB860507EB450595
:10A09000013BB5F850608579008940F2B5579208C8
:10A0A00007FB0232931903EB430304EBC303C3EB37
:10A0B000031301EB8303C3EB031305EB83030021BD
:10A0C0004FF47A72C2FB0301F0BC70475091030851
:10A0D000FAB170B48E18044603E0101A14D1B142DC
:10A0E00014D014F8012BA2F14103192B11F8013BF4
:10A0F000A3F1410598BF2032192D03F12000ECD9BE
:10A10000D01A01D1002BEAD170BC7047002070BC7E
:10A1100070471046704700BF4FF0FF32FFF7D8BFBF
:10A12000A0F16103192B98BF20387047A0F14103BB
:10A13000192B98BF20307047202805D009380428F3
:10A140008CBF00200120704701207047613819281A
:10A150008CBF002001207047413819288CBF002097
:10A1600001207047303809288CBF0020012070473B
:10A17000A0F13003092B07D920F02000413819281D
:10A180008CBF0020012070470120704730B4026866
:10A190001146531C036011F8024B0160D31C517827
:10A1A00003609378151D05601B0443EA0123D078F2
:10A1B000234343EA006030BC704700BF0368591C6A
:10A1C0001A46016012F8021B0260587841EA00202A
:10A1D000704700BF03685A1C02601878704700BFC0
:10A1E00038B50446006815462EF01DFF22682A4443
:10A1F000226038BD036810B40A0E5C1C04601A703B
:10A2000003680A0C5C1C04601A7003680A0A5C1C70
:10A2100004601A7003685A1C026019705DF8044BE0
:10A22000704700BF036810B40A0A5C1C04601A700F
:10A2300003685A1C026019705DF8044B704700BF38
:10A2400003685A1C026010B4197003680A0A5C1C87
:10A2500004601A7003680A0C5C1C04601A700368BE
:10A26000090E5A1C026019705DF8044B704700BF5C
:10A2700003685A1C026019700368090A5A1C0260BC
:10A28000197070472DE9F047002488B080460F46CA
:10A290001E46A14605AD531C0393117839B32529F9
:10A2A00033D1931CCDF810900393507830284ED0C2
:10A2B0004FF0000AA0F13003DBB2092B42D96C2821
:10A2C00019D0642800F0938024D825281CD063D9A5
:10A2D000582876D063281BD131784046B847039A76
:10A2E000531C03931178043601340029D7D120463A
:10A2F00008B0BDE8F087039B5A1C03921B78642BBF
:10A300007CD02AD8252B54D1252140460134B8478A
:10A31000039AC0E7732833D044D975284FD106F18A
:10A32000040E30682B4600220A217646FDF796FE81
:10A33000049A0095534639464046FDF7CDFE039AF0
:10A340000444A8E704AA03A91FF00AFBB7E7D31C3B
:10A35000039390784FF0010AACE7732B10D05BD9D0
:10A36000752B3AD0782B96D1A3F15802B2FA82F22B
:10A37000306852092B4610210436FDF76FFED7E7EF
:10A380003368049A0093394600234046FDF7A4FE43
:10A3900004360444039A7EE70028B9D1204608B069
:10A3A000BDE8F0876E28B3D1039A336804361C6089
:10A3B00071E72AD9582BD7D0632B8DD06BE778283B
:10A3C000A6D1A0F15802B2FA82F2306852092B46A7
:10A3D0001021FDF743FE0436AAE706F1040E3068AB
:10A3E0002B4600220A217646FDF738FEA0E7331DF2
:10A3F000306829461E46FDF703FE99E7331D306895
:10A4000029461E46FDF7FCFD92E7002B7FF443AF83
:10A41000204608B0BDE8F0876E2BC6D03BE700BFF2
:10A420000EB400B584B005AB019053F8042B064977
:10A43000039301A8FFF726FF019B00221A7004B0C6
:10A440005DF804EB03B07047CD8000080FB430B561
:10A4500083B006AB0A490B4853F8042B096800681F
:10A460000193FFF70FFF084C0546206802F054FFE8
:10A470000028FAD0284603B0BDE8304004B0704749
:10A48000242F0020282F0020041E0020DFED2B7A2F
:10A49000B4EEE70AF1EE10FA4ADDDFED296A9FED2E
:10A4A000297A01E0B0EE670AB4EEC70AF1EE10FABD
:10A4B00070EE667AF6DC9FED247AF4EEC77AF1EE60
:10A4C00010FA38D5DFED1E6A9FED207A01E0F0EE3C
:10A4D000407AF4EEC77AF1EE10FA37EEA60AF6D417
:10A4E000DFED1B7AB4EEE70AF1EE10FA14DDDFEDD2
:10A4F000137A37EEC00A60EE006A9FED166A9FED90
:10A50000167ADFED167AA6EE867A20EE266AE6EE59
:10A51000877AA6EE270A7047DFED117AB4EEE70AD4
:10A52000F1EE10FA44BFDFED087A37EEC00AE2E739
:10A53000F0EE407ABFE7B0EE670AD1E7DB0F4940A3
:10A54000DB0FC940E4CB1641DB0F49C0E4CB16C199
:10A55000DB0FC93F92E741B99730083C15A82ABEE6
:10A56000DB0FC9BF09B909E0194690FBF1F301FB04
:10A5700013030846002BF7D1084670470146FBE756
:10A58000F0EEC07AB0EEE07AB4EEE77AF1EE10FACF
:10A59000B4BFB0EE676AB0EE476AB5EE406AF1EE5E
:10A5A00010FA46D0B4EEE77AF1EE10FA8CBFF0EE76
:10A5B000675AF0EE475AC5EE866A9FED1F3A9FED47
:10A5C0001F6A9FED1F4A9FED1F5ADFED1F3ADFED17
:10A5D0001F4ADFED1F5AA6EEC36AE6EEA34AA6EEB7
:10A5E000864AB7EE006AA6EE845AA6EEA46AE6EEA4
:10A5F000855AC5EE866AB4EEE77AF1EE10FA48BFE6
:10A60000DFED147AF5EEC00A48BF77EEE66AF1EEA8
:10A6100010FA48BFDFED107AB5EEC00A48BF77EEFA
:10A62000E66AF1EE10FA48BFF1EE666AB0EE660A2D
:10A630007047DFED076ADEE739094E3DE3B59E3E20
:10A6400088FA163E45FE7F3F99FB243F69A2163EDD
:10A65000A7DFA834DB0FC93FDB0F4940DFED317ABC
:10A6600030EE277AFDEEC76A16EE903A2033402B83
:10A6700002D99FED2D0A7047B4EEE70AF1EE10FA09
:10A680004DDD9FED2A6ADFED2A6A01E0B0EE677AC0
:10A69000B4EEE67AF1EE10FA77EE467AF6DC9FED4C
:10A6A000257AF4EEC77AF1EE10FA35D5DFED1F6AA0
:10A6B0009FED217A01E0F0EE407AF4EEC77AF1EEF8
:10A6C00010FA37EEA60AF6D4DFED167AB4EEE70AF2
:10A6D000F1EE10FA1BDCDFED197AB4EEE70AF1EEC9
:10A6E00010FA44BFDFED137A37EEC00A60EE006A5D
:10A6F0009FED136A9FED137ADFED137AA6EE867A4B
:10A7000020EE266AE6EE877AA6EE270A7047DFED8E
:10A710000F7A37EEC00AE9E7B0EE670AD4E7F0EE49
:10A72000477ABCE7DB0FC93F00000000DB0FC940E0
:10A73000E4CB1641DB0F49C0E4CB16C1DB0FC9BF28
:10A7400092E741B99730083C15A82ABEDB0F494073
:10A75000FDEEC07A17EE903A2033402B51D8DFED52
:10A760002D7AB4EEE70AF1EE10FA50DDDFED2A6A39
:10A770009FED2A7A01E0B0EE670AB4EEC70AF1EE67
:10A7800010FA70EE667AF6DC9FED257AF4EEC77A61
:10A79000F1EE10FA38D5DFED206A9FED227A01E064
:10A7A000F0EE407AF4EEC77AF1EE10FA37EEA60A30
:10A7B000F6D4DFED1D7AB4EEE70AF1EE10FA1BDCF9
:10A7C000DFED1A7AB4EEE70AF1EE10FA44BFDFEDDE
:10A7D000147A37EEC00A60EE006A9FED156A9FEDAD
:10A7E000157ADFED157AA6EE867A20EE266AE6EE79
:10A7F000877AA6EE270A7047DFED067A37EEC00AA1
:10A80000E9E79FED0E0A7047B0EE670AD1E7F0EE78
:10A81000407AB9E7DB0F4940DB0FC940E4CB164172
:10A82000DB0F49C0E4CB16C1DB0FC93FDB0FC9BF4B
:10A8300092E741B99730083C15A82ABE00000000F5
:10A8400007EE901AF8EE677A9FED837A27EE800A7A
:10A8500020EE070AFDEEC07A17EE903A2033402B27
:10A8600000F28C80DFED7D7AB4EEE70AF1EE10FAAB
:10A8700040F3E880B0EE407A9FED796ADFED796AC7
:10A8800001E0B0EE677AB4EEE67AF1EE10FA77EE18
:10A89000467AF6DC9FED747AF4EEC77AF1EE10FAA0
:10A8A00040F1CD809FED6E6ADFED706A01E0F0EE61
:10A8B000477AF4EEE67AF1EE10FA37EE867AF6D4BD
:10A8C000DFED6B7AB4EEE77AF1EE10FA51DCDFEDF2
:10A8D000697AB4EEE77AF1EE10FA44BFDFED627AFE
:10A8E00037EEC77A27EE076ADFED635ADFED637A4A
:10A8F000DFED636A9FED635AE6EE257A67EE065A4E
:10A90000E6EE276AF7EE007AA5EEA67AF0EE675A31
:10A91000E7EE055AE7EE457A87EEA55ADFED547A61
:10A9200030EE277AFDEEC76A16EE903A2033402BC0
:10A9300029D99FED557AF6EE006AB7EE006AF7EE78
:10A94000004AC4EEA57A0023836143610362C361B8
:10A9500080ED045A67EEA66A27EE866A27EE877AAC
:10A96000C0ED006AC0ED026A80ED016A80ED037AF5
:10A970007047DFED3A7A37EEC77AB3E7B7EE005AA1
:10A98000F0EE455ACAE7B4EEE70AF1EE10FA5FDDE1
:10A990009FED336ADFED336A01E0B0EE677AB4EE23
:10A9A000E67AF1EE10FA77EE467AF6DC9FED2E7A33
:10A9B000F4EEC77AF1EE10FA47D59FED296ADFED84
:10A9C0002B6A01E0F0EE477AF4EEE67AF1EE10FA47
:10A9D00037EE867AF6D4DFED267AB4EEE77AF1EE3A
:10A9E00010FA27DCDFED237AB4EEE77AF1EE10FA05
:10A9F00044BFDFED1D7A37EEC77A27EE076ADFED39
:10AA00001E4ADFED1E6ADFED1E7AE6EE246A67EE6F
:10AA1000064AE6EE267AB7EE006AA4EEA77AF6EECC
:10AA2000006A36EE476AF8EE007A27EE277A66EE7D
:10AA3000266A84E7DFED097A37EEC77ADDE7B0EE04
:10AA4000677A3DE7F0EE407A24E7B0EE677AC2E736
:10AA5000F0EE477AAAE700BF27D4D236DB0F494091
:10AA6000DB0FC940E4CB1641DB0F49C0E4CB16C174
:10AA7000DB0FC93FDB0FC9BF92E741B99730083CF4
:10AA800015A82ABEF304353F0000008070B40668A4
:10AA90008E4217D90139751E002311F8014F082283
:10AAA000634013F0800F4FEA430318BF83F0D503D0
:10AAB000013ADBB2F5D18D42EFD1721C02603370E6
:10AAC00070BC70470023F8E710B44C09012250F81D
:10AAD000243001F01F0102FA01F10B4340F8243049
:10AAE0005DF8044B704700BF4B0901F01F0150F89F
:10AAF0002320012303FA01F1114214BF184600205C
:10AB0000704708B5FDF782FD0A2002F0FFF9012029
:10AB100008BDF8B50F4D46686A701446027A0F46B4
:10AB200042F0800225213046FFF7EBFF3A4626210E
:10AB30003046FFF7E6FF04F00F0242F080022721C3
:10AB40003046FFF7DEFF02F095F9686001202870BB
:10AB5000F8BD00BF981D002070B50478032C0E4688
:10AB6000154603D0BDE87040FDF796BD4468027AF3
:10AB700025212046FFF7C5FF324626212046FFF754
:10AB8000C0FF2A4663212046FFF7BBFF8122272111
:10AB90002046FFF7B6FF012070BD2DE9F0410E46BB
:10ABA0000178032990461F4621D14468027A252165
:10ABB00042F080022046FFF7A4FF324626212046BD
:10ABC000FFF79FFF07F00F0242F080022721204687
:10ABD000FFF797FF042002F0F3F972B649213B46D4
:10ABE00042462046FDF7A2FC62B6BDE8F08102298C
:10ABF00005D146F08001BDE8F041FDF797BC00208B
:10AC0000BDE8F08137B500F10C04054600220A21A9
:10AC10002046FFF7A1FF0F220A212046FFF79CFFE5
:10AC200001AA032310212046FFF7B7FF9DF8043047
:10AC300080336B839DF805308033AB839DF80630FD
:10AC40008033EB8300220A212046FFF785FF0DF1B8
:10AC50000302012302212046FFF79FFF01230DF18C
:10AC6000030209212046FFF798FF11220A212046FE
:10AC7000FFF772FF012003B030BD2DE9FF47037BD2
:10AC80000546884600F10C061BB1022B06D9032BA2
:10AC90003DD00024204604B0BDE8F08701230DF12B
:10ACA000070202213046FFF778FF0028F1D09DF817
:10ACB0000730D907EDD5072302AA03213046FFF755
:10ACC0006CFF0446002CE4D09DF80E7011220A217E
:10ACD0003046FFF741FF3B07DBD4B5F91A1002A855
:10ACE000FDF7DFFA4042A8F80000B5F91C100DF19D
:10ACF0000A00FDF7D6FA4042A8F80200B5F91E1086
:10AD000003A8FDF7CEFA4042A8F80400C2E7234F9B
:10AD10004FF0010A0024B9463B7A012B1BD00FD318
:10AD2000022BCFD1FDF7CBFA81460028B1D102A981
:10AD300005F11000FDF754FC87F808900446C1E7C0
:10AD40003B7823B9012202213046FFF7E2FE0123BE
:10AD500089F808309DE7FDF7B2FA002899D102A9D9
:10AD600005F11000FDF73CFC9DF80830044608B1E1
:10AD7000DA0707D4002389F80830BAF1000F88D029
:10AD80009A46C9E73B7823B9072203213046FFF7EB
:10AD9000C0FE022389F808307BE700BF981D002021
:10ADA0000C4B984213D0A3F5806398420FD003F563
:10ADB000804398420BD003F58063984207D003F597
:10ADC0008063984203D0044B186840087047024BD8
:10ADD000186870470004014068500020F0B5774BB8
:10ADE000774A87B01968914200AF00F0DB800023FA
:10ADF000744A3B607B60136843F48033136003E064
:10AE00003B68B3F5A04F09D0136803F400337B60AF
:10AE10003B6801333B607B68002BF1D0694B1B68BA
:10AE200013F4003318BF01237B607B68012B7BD0B8
:10AE3000654D644B654AEA606549586F654A08602C
:10AE4000AA605E6B644C654A654826F080065E63C6
:10AE50005E6F46F080765E67196B0C431C63596B1E
:10AE60005963996B9963196C41F05B5141F47B1103
:10AE700041F41F6141F00F011964596C07F1180486
:10AE80000A4348F2FF715A6444F8101D0026214617
:10AE90000123FB733E737E73BE7317F0F3F82146F4
:10AEA0004FF6FF734F48BB6017F0ECF84FF6FF7397
:10AEB00021464D48BB6017F0E5F821464B4817F096
:10AEC000E1F821464A4817F0DDF82146494817F0D5
:10AED000D9F82146484817F0D5F82146474817F0D9
:10AEE000D1F82146464817F0CDF8204616F042FF2B
:10AEF000444B454C1B68BA6844484549A4FB03438E
:10AF00009B09A0FB0202013B920CB3F1807F0A6017
:10AF100007D2404AF0200721536085F8230096604D
:10AF200011601C37BD46F0BD264B3B4D1A6C3B48AB
:10AF300042F080521A642C684268816844F44044AC
:10AF40002C609C689C609C6844F400449C609C68F5
:10AF500044F4A0549C600068120642EA801242F455
:10AF60008002490842F01902013942EA01425A605E
:10AF70001A6842F080721A601A689201FCD528495A
:10AF8000104A40F205700860996821F00301996049
:10AF9000996841F002019960936803F00C03082B53
:10AFA000FAD145E700221A6062B61E4B1B6883F394
:10AFB00008881D4B1B689847FEE700BFFCFF012077
:10AFC000EFBEADDE0038024000ED00E00005FA05FE
:10AFD000484F002000000008FF916700335F070022
:10AFE000000002400004024000080240000C024041
:10AFF000001002400014024000180240001C0240F1
:10B000000020024068500020D34D621083DE1B43B5
:10B01000346A002010E000E00070004000000020D2
:10B02000003C02400000FF1F0400FF1F08B5054B55
:10B030001B6803B19847044B044A1A6072B6FDF7C7
:10B040005BF900BF783D0020FCFF0120EFBEADDEC4
:10B05000F8B50468C4F30D0405460E4604B32F6822
:10B0600016F0FCFF092840F08980464C236923F440
:10B0700040732361236943F400732361236943F020
:10B08000010323613E6016F0E9FF2369092823F0DC
:10B090000103236172D12B6804332B600020F8BDBB
:10B0A000394B3A4A93422CD902F58042934227D930
:10B0B00002F5804293422BD902F58042934229D96E
:10B0C00002F58032934227D902F50032934225D906
:10B0D00002F50032934223D902F50032934221D97E
:10B0E00002F5003293421FD902F5802293421DD906
:10B0F000B3F1016F1CD305201EF0ECFCFFF796FFA7
:10B10000082416F0ABFF092814D04FF0FF30F8BD2B
:10B110001024F6E71824F4E72024F2E72824F0E7C7
:10B120003024EEE73824ECE74024EAE74824E8E757
:10B130005824E6E7134F3B6923F440733B613B69B6
:10B1400043F400733B613B6923F0F8033B613B69C7
:10B1500043F002031C433C613B6943F480333B6191
:10B1600016F07CFF3B6923F002033B613B69092831
:10B1700023F0F8033B613FF472AFC6E76FF00100C4
:10B18000F8BD00BF003C024000400008FF3F00083F
:10B19000F8B504460D468E180027B54201D1206946
:10B1A000F8BDE368591CE160234415F8012B1A72BD
:10B1B0000429F2D1206918B9A1682046FFF748FF99
:10B1C0002061E760E9E72DE9F04FDFF850914E4F3D
:10B1D0008BB00326A7EB09071822002104A82DF045
:10B1E00047FF4A4BCDF8109005971A69002A04DAF8
:10B1F000474A5A6002F188325A6001228DF82420B1
:10B20000F322DA60434B444C1B88ADF80030022235
:10B21000694604A8FFF7BCFF022269464FF6FF709B
:10B22000FDF726F8DFF8F8A080464FF0000B5445F4
:10B230003BD30AAC002524F8245D0222214604A851
:10B24000FFF7A6FF022221464046FDF711F840BA5B
:10B25000C043ADF80800022202A904A8FFF798FF36
:10B26000079878B106ABC0F10402294618442DF0C6
:10B27000FFFE089818B9069904A8FFF7E9FE002315
:10B28000089007939DF82430089A23B11F490B6951
:10B2900043F000430B61013E2FD0002A9CD1FEF702
:10B2A0008FFC60B30BB0BDE8F08F65888DF80DB0F2
:10B2B000C5F30B05AB1DADF808302388C3F30B02B3
:10B2C000ADF80A201B0B062202A904A88DF80C3049
:10B2D000FFF75EFF062202A94046FCF7C9FF61683E
:10B2E00080462A4604A8FFF753FF616840462A4675
:10B2F000FCF7BEFF1434804699E7002ACFD0052022
:10B300001EF0E8FBFFF792FE00800008003C0240C0
:10B3100023016745009203089001000800400008DF
:10B32000A005000808B5034B1B6803B1984772B627
:10B33000FCF7E2FF783D00202DE9F04F7A4C54F8FD
:10B34000204083B0002C00F0EA80D4F86090B9F17E
:10B35000000F00F0E680D9F81050D9F80470734E51
:10B36000A16004F166012660616104F266264FF473
:10B370000071A661E1602161A765A0464DB3DFF8C9
:10B38000B4C14FF0000E61464E68B54201F11C0198
:10B3900006D00EF1010EBEF1100FF5D14FF0000EE8
:10B3A000CEEBCE0E0CEB8E01DFF884C10E69DCF81B
:10B3B00030E04FF00C0A4EEA060E461CCCF830E0A6
:10B3C00081F818A04E76D9F80810E1630437676554
:10B3D00065630546D9F80C001F46164600283CD088
:10B3E000DFF850C1002163465A68904203F11C0304
:10B3F00003D001311029F7D10021C1EBC1010CEBC1
:10B4000081014B4B0A69186BDFF82CE1104318637C
:10B410000B200876681C4876186B024399F81F00C9
:10B420001A63830991F80DC08DF8053000220123BD
:10B430004C61C1F808E001A88DF806208DF80730AE
:10B440008DF804C016F05EFCA36DD9F80810D9F889
:10B450000C20A26304332164236594F8650001F095
:10B46000E9F9824694F8640001F0E4F9834699F81A
:10B470001C00002850D1380739D4B2070ED5BAF1D4
:10B48000000F0BD00B226B1C8AF806208AF80730BD
:10B49000504699F81D20222101F034F8F30716D404
:10B4A000E36B83B999F81E208DF8042099F82020C9
:10B4B0008DF8063001A8930901228DF805308DF82A
:10B4C000072016F01FFC404603B0BDE8F08FBBF12B
:10B4D000000FE5D001350C238BF807508BF80630B0
:10B4E000584699F81D20222101F00CF8D8E70135C3
:10B4F000EDB2BAF1000F04D00B238AF807508AF896
:10B50000063017F0100F50460CBF1221022199F897
:10B510001D2000F0F7FFC3E729F04CFEABE7A04683
:10B52000D1E7C846CFE700BF302F002004920308C0
:10B5300000380240FC190020618400080348D0F85C
:10B54000AC3113B100F5D27018477047FC190020D8
:10B550000348D0F8903113B100F5C4701847704714
:10B56000FC1900200348D0F8743113B100F5B6700F
:10B5700018477047FC1900200348D0F8583113B120
:10B5800000F5A87018477047FC1900200348D0F850
:10B590003C3113B100F59A7018477047FC19002030
:10B5A0000348D0F8203113B100F58C70184770476C
:10B5B000FC1900200348D0F804310BB1FC301847C7
:10B5C000704700BFFC1900200348D0F8E8300BB1E9
:10B5D000E0301847704700BFFC1900200348D0F83E
:10B5E000CC300BB1C4301847704700BFFC190020A5
:10B5F0000348D0F8B0300BB1A8301847704700BFEF
:10B60000FC1900200348D0F894300BB18C30184757
:10B61000704700BFFC1900200248836F0BB17030E7
:10B6200018477047FC1900200248C36D0BB1543015
:10B6300018477047FC1900200248036C0BB13830E2
:10B6400018477047FC1900200248436A0BB11C30B0
:10B6500018477047FC1900200248836803B1184757
:10B66000704700BFFC1900201549164B16480A68A0
:10B6700010B48C681549B2FBF4F203FB02F30360CB
:10B68000D1F88820124B134C42F47002C1F8882084
:10B690001A68002042F001021A6098601A6822F0CD
:10B6A000847222F480321A605C601A684FF0006481
:10B6B00022F480221A60D8608C605DF8044B7047D9
:10B6C0000000002040420F006850002000ED00E024
:10B6D0000038024010300024044B4FF4F0700A216F
:10B6E000022283E80700FFF7BFBF00BF0000002071
:10B6F00038B50B4C23688BB15A68821A002A05466C
:10B7000004DA0CE05A68AA1A002A07DB9A68226059
:10B7100018461A6890472368002BF3D138BD38BD0E
:10B72000E45F00200B4B002210B4027203F1C0044E
:10B73000032102E0072A09DC9979890702D51979E2
:10B74000815401329C4203F11803F3D15DF8044B9C
:10B75000704700BF60B4030812230370704700BF36
:10B760000123342135224170427103720370037149
:10B77000704700BF436A8269D154436A0169826B92
:10B7800001338B4228BF00234362002A2FD0EFF3FE
:10B790001182502383F31288836B1968C9072CD454
:10B7A00070B45E686EB9456A816A8D4217D084694B
:10B7B0000C44DC600ED9691A59608562002180F85A
:10B7C0005C10196841F00101D2B2196082F311884E
:10B7D00070BC70470469611A59608662EEE7012304
:10B7E00080F85C30D2B282F3118870BC7047826DF1
:10B7F000D36843F08003D3607047D2B282F31188DC
:10B80000704700BF426B10B462B1C36CC268446938
:10B81000D11A013B615C5DF8044B08BF1346C36459
:10B82000C8B27047016A4369C4685B5C0131A142D8
:10B8300028BF114601625DF8044BD8B2704700BFC3
:10B84000836B13B190F85C007047836A406A181AE2
:10B85000B0FA80F040097047416A836A99420AD37E
:10B86000CB1A816B026961B14968501E0B44834257
:10B870000AD2C01A704702691144CB1A816B0029A1
:10B88000F2D1501EC01A704700207047436B43B17D
:10B89000C26C5B6893422FBF981AC0689B1AC0188D
:10B8A0007047C269036A9A422FBFD01AC0688018D5
:10B8B000C01A70470A4B30B503F1100493F9002009
:10B8C0005D78072AC8BF143A811804330D7313F842
:10B8D000025C855413F8012C0A76A342EED130BDE8
:10B8E0002C92030803682DE9F041DF691FB13B4644
:10B8F000BDE8F0411847002A164611DD04460D4602
:10B900000E4400E023689B68204698470028F9D041
:10B91000236815F8011B1B6820469847AE42F1D1F9
:10B92000BDE8F08110B424211824322200230470D1
:10B9300041708270C3705DF8044B70472D234370D3
:10B940002E2303712F23C371704700BF038A2DE993
:10B95000F0478589ADB21D4029D00F4606464FF00D
:10B9600000484FF00009B5FA85F328FA03F2D243F4
:10B9700091B21B3B15403182042B16D8DFE803F04F
:10B980003129211903007B6A002B32D003F1FF3AE1
:10B990001FFA8AFAC7F824903C6A34B1236820461B
:10B9A000514698476468002CF8D1002DDBD1BDE8E2
:10B9B000F0873868716B036889B29847002DD2D13F
:10B9C000F5E77868B16B036889B29847002DCAD152
:10B9D000EDE7B868F16B036889B29847002DC2D1D2
:10B9E000E5E7F868316C036889B29847002DBAD151
:10B9F000DDE7F36A1FFA83FACEE700BF30B50446ED
:10BA0000806D61718389A26823F400531B041B0CB1
:10BA1000838185B0A379009213F004022ED04FF4F5
:10BA2000805213F00203ADF804203CD1ADF806308B
:10BA30004FF480630022ADF8083011F00103ADF837
:10BA40000C2026D1ADF80A3008238A07694648BF82
:10BA5000ADF80A3016F0DCF9A379A26D13F0080FE7
:10BA6000938A1BD123F008031B041B0C9382938938
:10BA70009BB243F40053938105B030BD13F0020331
:10BA8000ADF8042012D04FF400551346ADF806501F
:10BA9000D0E70423ADF80A300C23D6E79BB243F07D
:10BAA00008039382E3E74FF40053BFE7ADF8063095
:10BAB000C0E700BF10B50446806DA160838923F400
:10BAC00000531B041B0C8381A37984B013F0040280
:10BAD000009133D04FF4805213F00203ADF80420EC
:10BAE0003CD1ADF806304FF480636279ADF8083090
:10BAF000D1074FF00003ADF80A30ADF80C3045BF68
:10BB00000423ADF80A3008230C236946920748BF86
:10BB1000ADF80A3016F07CF9A379A26D13F0080F86
:10BB2000938A16D123F008031B041B0C938293897C
:10BB30009BB243F40053938104B010BD13F0020391
:10BB4000ADF804200DD04FF400511346ADF80610A7
:10BB5000CBE79BB243F008039382E8E74FF400532E
:10BB6000BFE7ADF80630C0E7022810B428BF0220B6
:10BB7000064C074B207000EB8001064A5DF8044B31
:10BB8000C0EBC10003EB400010607047B0470020DD
:10BB9000CA4700209042002010B5FDF7E7FF094A90
:10BBA000094B0A490A4C0B48146000221A705A705B
:10BBB000086022F0F7F8FFF706FBBDE8104022F01E
:10BBC000D9B800BF90420020B04700209442002026
:10BBD000CA470020D648002008B522F0E3F8FFF756
:10BBE000F2FABDE8084022F0C5B800BF38B5484BAE
:10BBF0005A899989914224BF00225A81198ADA8987
:10BC0000914224BF0022DA81DA78CAB1072A414979
:10BC10006AD091F85300404D012400210A282C706D
:10BC20009C70D9715DD00C2807D0002A6CD0DFED54
:10BC30003B7A072A0ED00A2862D0DFED397A09E074
:10BC4000344A92F853000A2856D00C285BD1D9798F
:10BC5000DFED347A344C9FED350AA278002918BF05
:10BC6000F0EE407A062A04D8314901EB820191EDC9
:10BC7000040A217979B1013A032A0BD8F7EE007A48
:10BC800087EE800A2CF02EFA2388984228BF1846A7
:10BC9000208038BD38BD9B781F4A07EE103A1178D6
:10BCA000B8EEC77A67EE277A07EE101AB8EEC77AB1
:10BCB00027EE277AB4EEC70AF1EE10FAEADD80EE3D
:10BCC000277AFDEEC77A17EE903A102BA8BF102303
:10BCD000012BB8BF0123DBB28B4238BF0B46137078
:10BCE00038BDDFED147AA4E791F853000A2803D099
:10BCF0000C28ACD0D9799AE7D979DFED0E7AA9E78B
:10BD0000DFED0D7AA6E7D979DFED047AA2E700BF6F
:10BD1000485800206C500020F46200206F12033954
:10BD20006F12833A0AD7A339AC4B00206F12033845
:10BD30002C9203085304E9380F506E3A2DE9F0476E
:10BD4000AE4FAF4E22F02EF8BE421ED2DFF82C834B
:10BD5000DFF82C934446258862197DB14A450DD2FF
:10BD6000052D0BD933886188C3F30B03994200F08A
:10BD7000E880144625886219002DEFD1716830469D
:10BD80001436FDF7CFFEBE42E4D39E4A1378A3F1EA
:10BD9000170102290FD99C4911F83300002840F0FF
:10BDA000FF80D8000144497829B1984911F833300F
:10BDB0000BB918231370964B5A78022A00F2E180CF
:10BDC0009449954802EB420201EB82011A78016026
:10BDD000022A00F2DF8002EB8201904BC2EBC1022B
:10BDE00003EB4203998C5A8C8D4C9142236001D312
:10BDF00000225A848B4B9A78042A00F0F28032B9E0
:10BE00001A88B2F5F07F84BF4FF4F0721A80864D25
:10BE1000FFF7ECFE2B68854A1A40002A00F0EA8002
:10BE2000D80700F1D980590400F1D1801A0700F138
:10BE3000C0809B0400F1C48027F00AFF10B97C4841
:10BE400024F038FD4FF40070FDF7B2FE4FF480305F
:10BE5000FDF7AEFE4FF40030FDF7AAFE4FF4802050
:10BE6000FDF7A6FE4FF40010FDF7A2FE4FF00070A4
:10BE7000FDF79EFE4FF08060FDF79AFE26F0D8F9A0
:10BE8000002130226B482DF0F3F8206817F090F86D
:10BE9000694B256803F1500102E0043399427DD0DB
:10BEA0001A78002AF9D19C78D8788442F5D263496F
:10BEB000634B0A7028461D601CF05AFB614A6249B8
:10BEC0001079624A624B1160C822642111FB002183
:10BED000002259609A60DA601A615A619A61DA61E7
:10BEE00083F8202083F8212019F0DCF8594B9FEDCE
:10BEF0005A5A1B88594A9FED5A6A5079594906EE99
:10BF0000903AF8EEE66A1388C5EE265A07EE103A24
:10BF100053881279C1ED005A07EE903AB8EEC77A0D
:10BF2000514BF8EEE77A18725A7227EE067A67EEEE
:10BF3000867ABDE8F04783ED017AC3ED007A21F0FF
:10BF400019BF63799B077FF414AF716894F804A05C
:10BF50003046FDF7E7FD3388BAEB133F04D01436C3
:10BF6000BE42FFF4F7AE10E773887068AA1FC3F3F0
:10BF70000B039A4204F10601A8BF1A462DF053F8AC
:10BF8000EDE700225A701A78234822490160022AFC
:10BF90007FF621AF00221A70204B23E7012286E7AB
:10BFA000D8000C186468002C7FF4FCAE17241470C1
:10BFB000F8E62E48FDF7FCFD2B689B047FF53CAFAF
:10BFC0002B48FDF7F5FD4020FDF7F2FD34E7294849
:10BFD000FDF7EEFD2B6829E72748FDF7E9FD2B6803
:10BFE00021E79A8AB2F57A7FBFF411AF4FF47A72E3
:10BFF0009A820CE743F008032B6011E7A0050008C4
:10C00000900100080041002044B50308F4AA030889
:10C01000B0470020D648002094420020CA470020A4
:10C0200090420020AC4B00202463002009600002F5
:10C03000F0690020F01E002050320020380B002054
:10C04000241F0020FC68002006630020381F002009
:10C050000C410020C8230020C0C9FB484C2400200C
:10C0600017B7D138CC230020E0680020016000021F
:10C070000940000209200002086000020240000896
:10C080000080000808B521F08DFEFFF79CF821F034
:10C0900071FEBDE8084051E6F0B50C2934D8DFE860
:10C0A00001F0893333335E333333343333330700B2
:10C0B000048C9689B2F802E01788734D24F48054FA
:10C0C0002404240C0484038C8488818B23F400537F
:10C0D00021F4E6411B0409041B0C46EA0E06090C78
:10C0E00043EA063341EA0721A8429BB2A4B289B2CF
:10C0F00000F09E8005F58065A84200F09980926866
:10C100008480818302640384F0BD048C9589B2F835
:10C1100002C0B2F800E05C4F24F480742404240CC4
:10C120000484038C8688818B23F400731B0421F024
:10C1300073011B0C45EA0C04090443EA0423090CAF
:10C14000B8429BB2B6B241EA0E015CD04F4CA0425D
:10C1500059D0926886808183C2630384F0BD048CC9
:10C160009589B2F802C0B2F800E0474E24F01004FE
:10C170002404240C0484038C8788018B23F020037F
:10C1800021F4E6411B0409041B0C45EA0C04090CCC
:10C1900043EA041341EA0E21B0429BB2BFB289B216
:10C1A0005DD03A4CA0425AD0926887800183826366
:10C1B0000384F0BD048C9789B2F802E01688324DF2
:10C1C00024F001042404240C0484038C8488018B4F
:10C1D00023F002031B0421F073011B0C47EA0E0736
:10C1E00009043B43090CA8429BB2A4B241EA0601F0
:10C1F00025D005F58065A84221D09268848001830E
:10C2000042630384F0BDD589148A578A23F40063FE
:10C2100043EA05254FF6FF332B40958826F4405618
:10C220003C4343EA052346EA04169BB2B6B290E7C4
:10C23000158A24F4804444EA8514A4B25FE7D689C1
:10C24000158A578A23F00803334324F440749688F0
:10C250003D4323F004032C433343A4B2CDE7D489F8
:10C26000158A568A23F0800343EA04134FF6BF74FD
:10C270001C40938827F44067354344EA031347EA98
:10C2800085079BB2BFB28FE7000001400004014068
:10C290002DE9F04FA022002183B08A488A4CDFF8B4
:10C2A0004C928A4D8A4E8B4FDFF844822CF0E0FE90
:10C2B00089488A49DFF83CE2DFF83CC20022135982
:10C2C000834200F0D480B3F1804F00F0E480AB42B1
:10C2D00000F0E380B34200F0E280BB4200F0E18076
:10C2E000734500F0E080634500F0DF80434500F0D7
:10C2F000DE80DFF808A2534500F0DB800AF5806A93
:10C30000534500F0D8800AF5806A534500F0D58087
:10C31000AAF5983A534500F0D2800AF5806A534551
:10C3200000F084800AF5806A534508BF0D237ED053
:10C330001832D82AC3D1644C694E6A4F6A4D04F151
:10C34000D80802E01834A0456DD0A379002BF9D0AD
:10C3500023794FEA131909F1FF39B9F1030F03F0FB
:10C360000F03EFD836F8190040FA03F2D207E9D5E7
:10C370004FF0010A0AFA03F3013B18402BF03AFB95
:10C3800017F80930184415EBC002DBD055F830001F
:10C39000DFF86CE1217A00F13F4303F57E039B0A4D
:10C3A0001EF8033003F01F0E5B09032B0AFA0EFA86
:10C3B0005FD0042B66D0022B07D1DFF820E1DEF836
:10C3C00044304AEA0303CEF8443093880093B3FA2A
:10C3D00083F3C3F11F039BB2DA0800EB820203F080
:10C3E0000703D2F820E09B004FF00F0C0CFA03FC7F
:10C3F0002EEA0C0EC2F820E0D2F820E001FA03F396
:10C4000043EA0E03136269460023022218348DF8B2
:10C4100004208DF805308DF806308DF8073015F0C2
:10C4200031FEA04591D103B0BDE8F08F0C2309EB9C
:10C43000C3034FF0010A1B7903F01F0B5B09032BA9
:10C440000AFA0BFA09D0042B0CD0022B7FF470AF40
:10C450004B6C4AEA03034B646AE70B6C4AEA03033A
:10C460000B6465E70B6B4AEA03030B6360E7002389
:10C47000DDE7DFF868E0DEF840304AEA0303CEF893
:10C480004030A2E7DFF854E0DEF830304AEA030338
:10C49000CEF8303099E70123C9E70223C7E7032329
:10C4A000C5E70423C3E70523C1E70623BFE7072346
:10C4B000BDE70823BBE70923B9E70A23B7E70B2346
:10C4C000B5E700BF7424002060B4030800040040F6
:10C4D00000080040000C004000000140003802400D
:10C4E0003CB5030838B50308EC6A002014AF030814
:10C4F00000040140001000400014004000400140D2
:10C500008CAF030800286AD003682DE9F04F03F1CF
:10C510003F4404F57E045F4EA40A0125345D04F017
:10C520001F066409032C05FA06F559D0042C00F007
:10C53000AC80022C59D08588B5FA85F0C0F11F0077
:10C5400080B2C40803EB840400F00700266A800070
:10C550000F27874026EA07062662276A01F00306AE
:10C560008240701E3A430128C1F3810CC1F30018C8
:10C570002262C1F341113DD90024224601274FF028
:10C58000030E03E0102A04F1020426D007FA02F099
:10C59000A84302F10102F5D1D3F800C00EFA04F06D
:10C5A000C04300EA0C0CC3F800C0D3F8008006FAC0
:10C5B00004FC4CEA080CC3F800C0D3F80CC000EA35
:10C5C0000C00D860D3F80CC001FA04F040EA0C006B
:10C5D000102AD86004F10204D8D1BDE8F08F70476A
:10C5E0002D4C266C35432564A5E72B4C666C3543F2
:10C5F0006564A0E7002002464FF0010E4FF00309EA
:10C6000004E00132102A00F102003CD00EFA02F7D9
:10C6100037EA0504F5D1D3F800A009FA00F4E443A1
:10C620000AEA040AC3F800A0D3F800B006FA00FA38
:10C630004AEA0B0AC3F800A0D3F808A004EA0A0AE1
:10C64000C3F808A0D3F808B00CFA00FA4AEA0B0ABB
:10C65000C3F808A0D3F804A02AEA07075F60D3F85C
:10C6600004A008FA02F747EA0A075F60DF683C4067
:10C67000DC60DF6801FA00F401323C43102ADC6020
:10C6800000F10200C2D1BDE8F08F034C266B3543A8
:10C69000256350E78CAF03080038024003682DE99A
:10C6A000F04F03F13F4404F57E04604EA40A0125D7
:10C6B000345D04F01F066409032C05FA06F500F04A
:10C6C000AF80042C00F0A780022C54D08588B5FAE6
:10C6D00085F0C0F11F0080B2C40803EB840400F0B1
:10C6E0000700266A80000F27874026EA0706266291
:10C6F000276A01F0030602FA00F0721E3843012A8D
:10C70000C1F3810CC1F300182062C1F3411137D984
:10C710000024224601274FF0030E03E0102A04F103
:10C72000020426D007FA02F0A84302F10102F5D173
:10C73000D3F800C00EFA04F0C04300EA0C0CC3F8B2
:10C7400000C0D3F8008006FA04FC4CEA080CC3F8D9
:10C7500000C0D3F80CC000EA0C00D860D3F80CC0BD
:10C7600001FA04F040EA0C00102AD86004F1020437
:10C77000D8D1BDE8F08F2E4C666C35436564A5E7D3
:10C78000002002464FF0010E4FF0030904E0013291
:10C79000102A00F102003CD00EFA02F737EA050435
:10C7A000F5D1D3F800A009FA00F4E4430AEA040A38
:10C7B000C3F800A0D3F800B006FA00FA4AEA0B0A60
:10C7C000C3F800A0D3F808A004EA0A0AC3F808A036
:10C7D000D3F808B00CFA00FA4AEA0B0AC3F808A02A
:10C7E000D3F804A02AEA07075F60D3F804A008FA88
:10C7F00002F747EA0A075F60DF683C40DC60DF68F9
:10C8000001FA00F401323C43102ADC6000F102001E
:10C81000C2D1BDE8F08F064C266B3543256355E742
:10C82000034C266C3543256450E700BF8CAF0308EA
:10C830000038024010B50409013C032C17D80D4BF9
:10C8400033F8142000F00F0042FA00F313F0010354
:10C850000DD0012303FA00F0013810402BF0CAF884
:10C86000054A064B125D104403EBC00010BD0020CA
:10C8700010BD00BF3CB5030838B50308EC6A0020C2
:10C8800001490248FFF762B8EC240020000401408F
:10C8900001490248FFF75AB8EC2400200004014087
:10C8A00001490248FFF752B8C4240020000C0040A0
:10C8B00001490248FFF74AB89C24002000080040C4
:10C8C00002494FF08040FFF741B800BF74240020B8
:10C8D000F0B50468434DA30AAB4269D05BD9424D21
:10C8E000AB4251D03E35AB4266D14FF0980E032695
:10C8F0004779B0004FEA970C00295FD063460227C2
:10C90000A5899F4083190CEB43032F4303F1040CCB
:10C91000364DBFB245F8231045F82C20A781EFF320
:10C920001181502282F31288821905EBC202136929
:10C9300073B313620433821905EBC202576917B14E
:10C940001F6053690433821905EBC202976917B15E
:10C950001F6093690433821905EBC202D76917B1CE
:10C960001F60D36904330027CAB21F6082F31188A5
:10C97000304405EBC000036AA3B9A38923F0010387
:10C980001B041B0CA381F0BD4FF0700E0226AFE715
:10C9900005EB0E03CFE7B3F5801F0ED14FF0200E4D
:10C9A0000026A5E7A3899BB243F00103A381F0BD54
:10C9B0004FF0480E01269BE7F0BDF0BD0223BF08F3
:10C9C00003FA07F7A389094D9BB223EA07038719E6
:10C9D0000CEB470CA3810CF1040345F82C1045F82F
:10C9E00023209CE7020010000300100074240020A4
:10C9F00010B5036882480139834282B089B200F0E1
:10CA0000CA80A0F58060834200F0C58000F58040B8
:10CA1000834200F0B78000F58060834200F0B2806E
:10CA200000F58060834200F0AD80764C1888246861
:10CA30006408B4FBF2F4013CA4B282B2B3F1804FBB
:10CA40000AD07148834207D000F58060834203D04A
:10CA500000F58060834202D122F0700292B26B48EE
:10CA6000834200F0A18000F58060834200F0A68040
:10CA700022F4407200F56C4092B283421A80D9626F
:10CA80001C854FD05E4A93424CD001229A821A886C
:10CA900092B242F001021A80B3F1804F00F0988008
:10CAA000594A934200F0968002F58062934200F06A
:10CAB000938002F58062934200F0908002F58062DC
:10CAC000934200F08D8002F58062934200F08A80EC
:10CAD00002F57042934200F0878002F57052934253
:10CAE00000F0848002F58062934200F0818002F5BC
:10CAF000806293427ED0A2F5983293427CD002F5B8
:10CB0000806293427AD002F58062934208BF0D2280
:10CB100015D002A84FF0012340F8043D15F0F2F8BB
:10CB200002B010BD0122002119869A821A88384865
:10CB300092B242F0010283421A80ADD10A46354BCF
:10CB400003EBC20301A85C798DF8044001230022A5
:10CB50008DF805308DF807308DF8062015F0D2F8E5
:10CB60001B2C08D02E2CDBD12B4B019301A815F0E8
:10CB7000C9F802B010BD294B019301A815F0C2F805
:10CB800002B010BD1F4C18882468B4FBF2F4013CBD
:10CB9000A4B282B252E71B4C18882468B4FBF2F4AA
:10CBA000013CA4B282B257E701201A80D9621C85E9
:10CBB00098821A8892B202431A8071E701201A8083
:10CBC000D9621C8598821A8892B202431A8063E760
:10CBD0000122B4E70222B2E70322B0E70422AEE763
:10CBE0000522ACE70622AAE70722A8E70822A6E763
:10CBF0000922A4E70A22A2E70B22A0E70C229EE763
:10CC00000004014068500020000400400010004073
:10CC10000000014014AF03082C01000119010001BC
:10CC20002DE9F04F013085B0C3B203930B4602915A
:10CC30008B4C8C4E002B00F09A8032208A4D8B4F0B
:10CC4000DFF82C9227F07CFB4FF4FA7A4FF0100CAF
:10CC50004FF47A70D9F80430C3F30803002B40F086
:10CC6000DE80EFF31183002B40F0D9802968A268A1
:10CC700000BF2B689942F9D1D7F800E000FB0EF312
:10CC80009B1AB3FBFEF300FB01314FF0010E019143
:10CC9000D9F80430C3F30803002B40F08780EFF38A
:10CCA0001183002B40F082802B68A16800BF2A68A6
:10CCB0009342F9D1D7F800B000FB0BF2521AB2FB45
:10CCC000FBF200FB0323019A9B1AB3F57A7FDFD3B3
:10CCD000BAF1010ABED1039B002B40F0BD804FF496
:10CCE0007A7ADFF88C9150464FF0100CD9F8043066
:10CCF000C3F30803002B75D1EFF31183002B71D11F
:10CD00002968A26800BF2B689942F9D1D7F800E0E2
:10CD100000FB0EF39B1AB3FBFEF300FB01314FF057
:10CD2000010E0191D9F80430C3F3080313BBEFF3EC
:10CD30001183FBB92B68A16800BF2A689342F9D11F
:10CD4000D7F800B000FB0BF2521AB2FBFBF200FB6B
:10CD50000323019A9B1AB3F57A7FE3D3BAF1010A50
:10CD6000C4D1029B013B0293002B7FF466AF05B058
:10CD7000BDE8F08FEFF311888CF31288A168236867
:10CD8000DB0344BFC6F800E0A1682B6832685FFA95
:10CD900088F888F31188D7F800801A4400FB08F35C
:10CDA0005B1AB3FBF8F300FB0233D2E7EFF3118811
:10CDB0008CF31288A1682368DB0344BFC6F800E047
:10CDC000A1682B6832685FFA88F888F31188D7F871
:10CDD00000801A4400FB08F35B1AB3FBF8F300FB76
:10CDE000023370E7EFF311828CF31288D4F808E075
:10CDF0002368D90303D501233360D4F808E02B68F6
:10CE00003168D2B282F311883A68194400FB02F308
:10CE1000A3EB0E03B3FBF2F300FB01317FE7EFF36B
:10CE200011828CF31288D4F808E02368D90303D563
:10CE300001233360D4F808E02B683168D2B282F362
:10CE400011883A68194400FB02F3A3EB0E03B3FB0D
:10CE5000F2F300FB013118E7184627F01FF93EE70F
:10CE600010E000E02C6A0020306A0020346A0020C4
:10CE700000ED00E0204B5B68C3F3080330B4BBB99E
:10CE8000EFF31183A3B91D4B1D4C1868A16800BFB7
:10CE90001A689042F9D11B4B1C684FF47A7202FB5E
:10CEA00004F3591AB1FBF4F130BC02FB00107047D7
:10CEB000EFF31182102383F3128811498C680B68F9
:10CEC00013F4803F104B02D0012018608C680B498E
:10CED000D2B20D68186882F311880A4B19684FF4B2
:10CEE0007A72284402FB01F31B1B30BCB3FBF1F345
:10CEF00002FB0030704700BF00ED00E0306A002008
:10CF000010E000E0346A00202C6A00202DE9F84F80
:10CF10008046FFF7AFFF254E2549DFF8A0E0254A00
:10CF2000254D844610274FF47A740120DEF8043032
:10CF3000C3F30803D3B9EFF31183BBB90B68D2F87D
:10CF400008A000BFD1F800904B45F7D1D6F800B04B
:10CF500004FB0BF9A9EB0A09B9FBFBF904FB0393EA
:10CF6000A3EB0C034345E1D3BDE8F88FEFF3118A3F
:10CF700087F31288D2F808B01368DB0344BF286037
:10CF8000D2F808B00B68D5F800905FFA8AFA8AF3F5
:10CF90001188D6F800A0994404FB0AF3A3EB0B0315
:10CFA000B3FBFAF304FB0933DAE700BF346A00206D
:10CFB000306A002010E000E02C6A002000ED00E064
:10CFC0002DE9F04FDFF830C1474A4849484E494DF6
:10CFD0008046102718F1FF38C0F08480DCF8043058
:10CFE000C3F30803002B5CD1EFF31183002B58D15E
:10CFF0000B68946800BF08688342F9D1D6F80090A6
:10D000004FF47A7000FB09FEAEEB040EBEFBF9FE96
:10D0100000FB03EEDCF80430C3F308034FF47A742A
:10D020000120FBB9EFF31183E3B90B68D2F808A034
:10D0300000BFD1F800904B45F7D1D6F800B004FB03
:10D040000BF9A9EB0A09B9FBFBF904FB0393A3EB6A
:10D050000E03B3F57A7FBDD2DCF80430C3F30803C6
:10D06000002BDFD0EFF3118A87F31288D2F808B0D3
:10D070001368DB0344BF2860D2F808B00B68D5F80A
:10D0800000905FFA8AFA8AF31188D6F800A09944D2
:10D0900004FB0AF3A3EB0B03B3FBFAF304FB093322
:10D0A000D5E7EFF3118487F31288D2F8089013685C
:10D0B000D80303D501232B60D2F808900B682868A9
:10D0C000E4B284F31188D6F800A04FF47A7400EB30
:10D0D000030E04FB0AF3A3EB0903B3FBFAF304FB0F
:10D0E0000E3E97E7BDE8F08F10E000E0306A0020C8
:10D0F000346A00202C6A002000ED00E030B4EFF329
:10D100001183102282F312880649074C0A680748E7
:10D11000013200250A602560DBB2026883F31188C2
:10D1200030BC7047306A00202C6A002010E000E01C
:10D1300038B5264B9C68636B73B1A36DA26BD2B1FB
:10D14000998A1A88C90592B201D5D20700D438BD90
:10D150004FF6F7721A8038BDA36D99891A8889062F
:10D1600092B2EBD59206E9D5E26AD2B19888216BEA
:10D1700080B29047E1E799891A880D0692B2DFD50F
:10D180001006DDD5A26A616A8A4219D0A1692569B3
:10D19000885C98800132B2FBF5F105FB1122A26296
:10D1A000CEE79B88E2696169DBB28B54E269E06893
:10D1B000A36D0132B2FBF0F100FB1122E261BDE789
:10D1C000DA6822F08002DA60BAE700BF302F002070
:10D1D00038B5264B5C68636B73B1A36DA26BD2B19B
:10D1E000998A1A88C90592B201D5D20700D438BDF0
:10D1F0004FF6F7721A8038BDA36D99891A8889068F
:10D2000092B2EBD59206E9D5E26AD2B19888216B49
:10D2100080B29047E1E799891A880D0692B2DFD56E
:10D220001006DDD5A26A616A8A4219D0A169256912
:10D23000885C98800132B2FBF5F105FB1122A262F5
:10D24000CEE79B88E2696169DBB28B54E269E068F2
:10D25000A36D0132B2FBF0F100FB1122E261BDE7E8
:10D26000DA6822F08002DA60BAE700BF302F0020CF
:10D2700070B4EFF31186502383F31288836B1A681E
:10D28000D20720D45D686DB9446A826A944217D08F
:10D2900081691144D9600ED9A21A5A6084620022B1
:10D2A00080F85C201A6842F00102F1B21A6081F342
:10D2B000118870BC704701698A1A5A608562EEE76E
:10D2C000012380F85C30F3B283F3118870BC70479F
:10D2D00003682DE9F041DF691FB13B46BDE8F0412D
:10D2E0001847002A164611DD04460D460E4400E09C
:10D2F00023689B68204698470028F9D0236815F8D2
:10D30000011B1B6820469847AE42F1D1BDE8F08171
:10D3100003689B69184700BF03685B69184700BF33
:10D3200003681B69184700BF0368DB68184700BF24
:10D3300003685B68184700BF03681B68184700BF95
:10D3400038B50C46097849B1054601342B682846A2
:10D350001B68984714F8011B0029F7D138BD00BF9E
:10D36000064B53F820302BB11A689B8851690B4249
:10D3700001D1138370475383704700BF206A002098
:10D38000026802F13F4303F57E032DE9F04F9B0A4B
:10D39000544DEB5C03F01F055B090124032B04FAD9
:10D3A00005F400F09980042B00F09180022B3ED010
:10D3B00001F00306731E012BC1F3810CC1F30018A9
:10D3C0008588C1F3411137D90024234601274FF046
:10D3D000030E03E0102B04F1020426D007FA03F039
:10D3E000A84303F10103F5D1D2F800C00EFA04F00E
:10D3F000C04300EA0C0CC2F800C0D2F8008006FA64
:10D4000004FC4CEA080CC2F800C0D2F80CC000EAD8
:10D410000C00D060D2F80CC001FA04F040EA0C0015
:10D42000102BD06004F10204D8D1BDE8F08F2E4B50
:10D430005D6C2C435C64BBE7002003464FF0010E9B
:10D440004FF0030904E00133102B00F102003CD03F
:10D450000EFA03F737EA0504F5D1D2F800A009FA6D
:10D4600000F4E4430AEA040AC2F800A0D2F800B0CB
:10D4700006FA00FA4AEA0B0AC2F800A0D2F808A09D
:10D4800004EA0A0AC2F808A0D2F808B00CFA00FAB6
:10D490004AEA0B0AC2F808A0D2F804A02AEA070751
:10D4A0005760D2F804A008FA03F747EA0A07576062
:10D4B000D7683C40D460D76801FA00F401333C439C
:10D4C000102BD46000F10200C2D1BDE8F08F064BF2
:10D4D0001D6B2C431C636BE7034B1D6C2C431C64BE
:10D4E00066E700BF8CAF0308003802402DE9F04F1B
:10D4F0004A484B494B4B4C4C4FF0010A4FF0020944
:10D500004FF004084FF0080C4FF0100E2027402673
:10D51000802530F8022B12F0010F03D01960A3F818
:10D5200004A0083312F0020F03D01960A3F804908E
:10D53000083312F0040F03D01960A3F804800833F5
:10D5400012F0080F03D01960A3F804C0083312F0DA
:10D55000100F03D01960A3F804E0083312F0200F75
:10D5600002D019609F80083312F0400F02D019607A
:10D570009E80083312F0800F02D019609D8008331E
:10D5800012F4807F05D04FF4807B1960A3F804B0BB
:10D59000083312F4007F05D04FF4007B1960A3F824
:10D5A00004B0083312F4806F05D04FF4806B19601B
:10D5B000A3F804B0083312F4006F05D04FF4006BE9
:10D5C0001960A3F804B0083312F4805F05D04FF45B
:10D5D000805B1960A3F804B0083312F4005F05D033
:10D5E0004FF4005B1960A3F804B0083312F4804FC5
:10D5F00005D04FF4804B1960A3F804B00833D20B68
:10D6000004D04FF4004219609A80083301F580611C
:10D61000A1427FF47EAFBDE8F08F00BF3CB50308A8
:10D6200000000240EC6A002000100240002855D0A3
:10D63000026802F13F4303F57E032DE9F04F9B0A98
:10D64000544DEB5C03F01F055B090124032B04FA26
:10D6500005F444D0042B00F09780022B44D001F055
:10D660000306731E012BC1F3810CC1F300188588DA
:10D67000C1F341113DD90024234601274FF0030E89
:10D6800003E0102B04F1020426D007FA03F0A843AC
:10D6900003F10103F5D1D2F800C00EFA04F0C04343
:10D6A00000EA0C0CC2F800C0D2F8008006FA04FCB4
:10D6B0004CEA080CC2F800C0D2F80CC000EA0C001A
:10D6C000D060D2F80CC001FA04F040EA0C00102B34
:10D6D000D06004F10204D8D1BDE8F08F70472E4B22
:10D6E0001D6C2C431C64BAE72B4B5D6C2C435C64B3
:10D6F000B5E7002003464FF0010E4FF0030904E0A8
:10D700000133102B00F102003CD00EFA03F737EA88
:10D710000504F5D1D2F800A009FA00F4E4430AEABE
:10D72000040AC2F800A0D2F800B006FA00FA4AEAE9
:10D730000B0AC2F800A0D2F808A004EA0A0AC2F84C
:10D7400008A0D2F808B00CFA00FA4AEA0B0AC2F8AC
:10D7500008A0D2F804A02AEA07075760D2F804A06C
:10D7600008FA03F747EA0A075760D7683C40D460D5
:10D77000D76801FA00F401333C43102BD46000F168
:10D780000200C2D1BDE8F08F034B1D6B2C431C631C
:10D7900065E700BF8CAF03080038024010B1036892
:10D7A00082885A83704700BF10B1036882881A8349
:10D7B000704700BF18B10368828809B95A8370475F
:10D7C0001A83704710B40A4B0A4A1C78012383401D
:10D7D000234052F8200029B9B3FA83F149095DF8D2
:10D7E000044BE7E7191C18BF01215DF8044BE1E782
:10D7F0001C6A0020206A002008B501210220FFF7E2
:10D80000E1FF094B1B7803F00503052B08D000212D
:10D810000120FFF7D7FF00210846FFF7D3FFFEE7FF
:10D8200015F090FFF3E700BF2C2F00202DE9F04109
:10D830000B4E346873691C400FD0DFF82880012735
:10D84000B4FA84F3C3F11F0307FA03F558F8230071
:10D8500003689847AC437561F2D1BDE8F08100BF21
:10D86000003C0140BC1D00202DE9F0410B4E346806
:10D8700073691C400FD0DFF828800127B4FA84F3C5
:10D88000C3F11F0307FA03F558F82300036898470C
:10D89000AC437561F2D1BDE8F08100BF003C0140AE
:10D8A000BC1D00202DE9F0410B4E346873691C400B
:10D8B0000FD0DFF828800127B4FA84F3C3F11F03E7
:10D8C00007FA03F558F8230003689847AC437561DD
:10D8D000F2D1BDE8F08100BF003C0140BC1D00203A
:10D8E0002DE9F0410B4E346873691C400FD0DFF80E
:10D8F00028800127B4FA84F3C3F11F0307FA03F564
:10D9000058F8230003689847AC437561F2D1BDE82D
:10D91000F08100BF003C0140BC1D00202DE9F0411A
:10D920000B4E346873691C400FD0DFF82880012744
:10D93000B4FA84F3C3F11F0307FA03F558F8230080
:10D9400003689847AC437561F2D1BDE8F08100BF30
:10D95000003C0140BC1D00202DE9F0410B4E346815
:10D9600073691C400FD0DFF828800127B4FA84F3D4
:10D97000C3F11F0307FA03F558F82300036898471B
:10D98000AC437561F2D1BDE8F08100BF003C0140BD
:10D99000BC1D00202DE9F0410B4E346873691C401A
:10D9A0000FD0DFF828800127B4FA84F3C3F11F03F6
:10D9B00007FA03F558F8230003689847AC437561EC
:10D9C000F2D1BDE8F08100BF003C0140BC1D002049
:10D9D000084A536C10B5084C43F480435364204606
:10D9E000402200212BF044FB4FF0FF332364C4F8A6
:10D9F000433010BD00380240BC1D00202DE9F0412D
:10DA0000044618460D461646984629F0F9FA276846
:10DA1000E6722844A07229467D6943463246204674
:10DA2000AC46BDE8F0416047036810B504461B688A
:10DA30009847236820469B689847A37B0133A373CC
:10DA400010BD00BF2DE9F04FBB4B1E788BB0002EF0
:10DA500040F08180B94BBA4C1D78BA4FDFF808B35B
:10DA600005F00105A4F10A0954F80A0CB8B14FF009
:10DA7000CC0808FB0698FFF75BFC80B154F80A0C51
:10DA8000FFF752FC14F8023C024683B924283BD02D
:10DA900075B354F80A0CFFF74BFC0028EED10136A1
:10DAA000032E04F1CC04DFD10BB0BDE8F08F012BC5
:10DAB0002ED0022B33D0032B40D0042B00F06781F3
:10DAC000052B00F05581062BE3D114F801ECBEF1D3
:10DAD000000F00F0D881BEF1010F00F01B8201366B
:10DAE0000023032E04F8023C04F1CC04BCD1DBE794
:10DAF000232A54F80A0C00F08081934B93F82A30C3
:10DB00009342B8D1FDF792FA012304F8023CC0E732
:10DB10004D2800F06581002304F8023CB9E700239A
:10DB20003C2804F8023C00F055813E28B1D1012286
:10DB3000032304F8012C04F8023CAAE7C028EAD821
:10DB40000021042304F8050C04F8040C04F8061C56
:10DB500004F8023C9DE77D4B18680028A4D0FBF731
:10DB600041FFDFF808A27A4DDFF8F491DAF80000FF
:10DB7000FFF7DEFB002897D0DAF80000FFF7D4FBB0
:10DB800009281BD03F2819D02B68002B66D1042808
:10DB900000F0BA810C2800F0C8807F28E6D0A0F100
:10DBA0002002D2B25E2AE1D80BB92028DED05A1C5E
:10DBB00009F803002A6020F0D9FCD7E72C68002C74
:10DBC00059D1644B264603F5047B002E08BF1E4640
:10DBD00010335B45F9D1002E00F04F81A3F11008FE
:10DBE0003068D8F80020075D135D9F42204402EBA7
:10DBF000040140F04081671E4F4422460BB9FD2AC4
:10DC00005BD907F8013F01322A6010F8013F11F893
:10DC100001EF9E45F2D00AB1B04512D04E4820F037
:10DC2000ADFCB04508D356F8100B20F0A7FC092036
:10DC300020F09CFC4645F6D9484820F09FFC2A6815
:10DC40000024944292D2661E4E4416F8010F20F032
:10DC50008DFC2B6801349C42F7D387E70C2864D0F5
:10DC60000A2833D00D2831D07F2800F0BD80FF2B4B
:10DC70003FF67CAF93E7374F4FF0000807F5047B82
:10DC8000464602E010375F450DD0224639684846C7
:10DC9000FCF71EFA0028F5D1B846002EF2D13E4618
:10DCA00010375F45F1D1002E9AD1B8F1000F3FF443
:10DCB0005DAF294820F062FCB5E7511C202009F82F
:10DCC0000200296009F801300A46A5E720F0D7FCD8
:10DCD000232123482BF0E3F9002800F01381A0EB67
:10DCE0000900286090B1431E19F80310202940F064
:10DCF0002E8109EB030243B112F8011D202903F123
:10DD0000FF304FD10346002BF6D12B604FF48072C9
:10DD1000002148462BF0ACF9074B1B78002B3FF451
:10DD2000C3AE0E4820F02AFC20E70E4820F026FC67
:10DD30000A4820F023FC19E716490020C4360020C9
:10DD40003A830020BC1D0020F069002034350020FB
:10DD500070360020A898030844BB03084CBB030896
:10DD60007035002054BB0308589203086C3500201E
:10DD700014F8063C14F8051C994270D814F8043CB9
:10DD800083427FF4C8AE062304F8023C9DE614F8F3
:10DD9000043C04F8030C5A40052304F8042C04F84E
:10DDA000023C76E62B606B4C002204F5047B09F8FC
:10DDB000032002E010345C454DD02168484613F042
:10DDC00091F80028F6D05C4545D2E36898470023D7
:10DDD0002B609BE7032204F8013C04F8022C58E670
:10DDE000022304F8023C54E6013B00225A482B600F
:10DDF00009F8032020F0C2FBB8E6584B5849DB78FD
:10DE0000584ADFF88CE11060003318BF01230B7013
:10DE1000554B564ACEF80030554BFA644FF0400E41
:10DE2000012187F854E0B864386587F855505148A7
:10DE3000197021F011F8504820F0A0FB4FF4006059
:10DE40000CF0C0FF4D4B93F82A30232B3FF45AAE11
:10DE500014F8023C37E64A4820F090FBB7E714F884
:10DE6000041C08EB03005140013304F8041C04F8BF
:10DE7000063C82720DE62246CDE64248A3F1100828
:10DE800020F07CFBCFE69BE80F000DF1280C0DF194
:10DE9000080888E80F004CF824ED14F8053C14F845
:10DEA00003AC0694624623444FF0010C414606A899
:10DEB000ADF822E00793ADF820A08DF824C00AF059
:10DEC00047FB40B1029A304B03924146A4F10A004D
:10DED00002930FF0FBF9DDF80480002304F8023C04
:10DEE000B8F1000F3FF4DBAD54F80A0C0FF090FAD4
:10DEF000013654F80A0CC047032E04F1CC047FF419
:10DF0000B3ADD1E52868EDE6204812F08BFA0BB0EE
:10DF1000BDE8F08F14F8053C14F8032C0694234454
:10DF200007936E2A4FF0000308930993ADF8202061
:10DF30007FF4D5AD06A8FCF74DF906A8FCF73EF92D
:10DF400006A8FCF73BF906A8FCF738F9C7E5034635
:10DF500029E700BFA89803087CBB0308B04700204E
:10DF60004C2600206C350020081E0020E5B8000873
:10DF70001649002080BB03084CBB0308F069002051
:10DF800060BB030844BB03083887002070350020BD
:10DF9000343500202DE9F04F2DED068B824B834A5E
:10DFA0001C7897B000F59C41203181460B9111609F
:10DFB000002C00F0A2877E4A1268904240F28D80C9
:10DFC0007C4A079216687C497C4A0691013C1C7089
:10DFD0007B4B049206F480560993002E40F08B8010
:10DFE000784B0893784B1B78022B00F09280042B1F
:10DFF00001F03D82012B01F0F181744B9945099BA1
:10E000009B7800F2AF80002B40F0AF80079B1E682A
:10E0100016F4805740F03887DFF8EC81049BB3F9A1
:10E020000610069B5D8BA942B4BF00250125DFF8D1
:10E03000C491D9F8003013F0805300F0E780089ABB
:10E04000127812F0010200F0E8800698408C8842B5
:10E0500041F34682002D40F0E7805D4C94F88C102F
:10E06000002940F0E1805B485B49006890F82D0092
:10E0700000240C604C608C605849002840F0D5802A
:10E080000870002A00F0D680F00640F1D380544A90
:10E090001278D10600F1CE80002F40F0CB80002B0B
:10E0A00040F0C880720200F1C5804E4B1B78002BF7
:10E0B00002F084814C4B9B78002D42F011823BB1E1
:10E0C0004A4A4B4B12681B689B1A002BC2F2EF8125
:10E0D0003F4C012384F88D30ACE0364B07931E682B
:10E0E000364B354A049306F48056354B0692099315
:10E0F000002E3FF475AF00213E48FCF7F5FC314B94
:10E10000002801F0678408932F4B1B78022B7FF4C3
:10E110006EAF069A0499537DD27D013B31F91330DD
:10E120001AB1C3F53B6308331BB2A3F57A7307EE4C
:10E13000903A9FED317A314AF8EEE77A40F2FF31BA
:10E1400067EE877AFCEEE77ACDED057ABDF81430FC
:10E150008B4228BF0B4613801C4B9945099B9B782B
:10E160007FF651AF002B01F03582089B244E1C78BE
:10E17000099BDFF8709093F82150224F1B2023F069
:10E18000F5FF099904F0010491F820308046A24679
:10E190008B46052B3FF63AAFDFE813F062065706D1
:10E1A000DA0599069B068E06E05F0020E85E0020F7
:10E1B000DC5F00206C580020C46900203C4900202E
:10E1C0000C410020C43600204A5F0020404B4C0028
:10E1D000541E0020904200209C40002098230020E4
:10E1E0008E420020380B002020630020306A00207F
:10E1F00014250020B06200206F12833FC44000202D
:10E20000FC68002088420020A032002074023FF504
:10E2100016AF089A127802F001026A4C002184F8C5
:10E220008C10002D3FF41FAF674901200870002AB1
:10E230007FF42AAF654B1A78002A40F0A780069930
:10E24000049C488BB4F90070898BB4F90240B84241
:10E25000B4BF8026002646F04003B942D8BF3346FB
:10E260009B0843F08006A042B8BF3346049F43F0AA
:10E270004006A142C8BF33469B08B7F90440B7F92E
:10E28000066043F08007A042B8BF3B4643F040071A
:10E29000A142C8BF3B469B0843F08007494C8642D9
:10E2A000C8BF3B4643F0400794F88EE08E42B8BFAB
:10E2B0003B469E4501F05083A4F8902084F89220BC
:10E2C000434884F88E300678002E01F051825F2B8F
:10E2D00001F0C3826F2B01F02A83089B1B78DE07B5
:10E2E00054D494F89210002950D1B4F99030322BC4
:10E2F0004CDD94F88E200120572A84F8920001F01A
:10E30000AF86079B1B6813F0040301F06E815A2A45
:10E3100041F06B8194F89430002B42F0A78094F880
:10E3200096302C4A059283F001032B4A0A9284F816
:10E3300096305BB1089B1B78D90707D5049BB3F9CE
:10E340000620069B5B8B9A4201F35F8411212348D0
:10E35000FCF7CAFB002801F0B18094F89A302BB981
:10E3600094F8943013B93223A4F89830012384F838
:10E370009A3016E01A4A1278940741F18486194AB5
:10E38000127D042A41F27F861DF046FA079B114A4E
:10E390001B680592104A0A9203F00403002B40F018
:10E3A0000E87114E0B960DF1500B0023CBF8043065
:10E3B0003546149340F6330A192740F28334049EFD
:10E3C00017E000BF541E0020982300203A49002087
:10E3D000380B00208C42002094420020B0620020C4
:10E3E0008E420020F0820020503200200435454546
:10E3F00020D0A978EB78994217FB0140F6D26978D2
:10E40000043117FB034336F911105145A8BF51469B
:10E41000B1F5617FB8BF4FF461718142E6DD994289
:10E42000E4DC29782729E1D858460435FCF74CFB71
:10E430004545DED13F4B0B9E1B789BE8030089E8E6
:10E440000300002B00F0408601213B48FCF74CFB09
:10E45000002840F09C82099BDB78002B40F09782DB
:10E46000364C059A3448178827F00107BFB20221BD
:10E470001780FCF739FB002800F09282BA0741F1BF
:10E48000AE802F4B2F4A19780C93BB0708BF81F041
:10E49000020150680B92C1F34001FFF78BF9242170
:10E4A0002548FCF721FB30B9089A13785F0744BF71
:10E4B00023F004031370276817F00A0F40F07682E8
:10E4C000059BB3F80080B80600F159851E4F1A4825
:10E4D0000C21FCF709FB002800F0218348F480742C
:10E4E0001A4B059A1B781480082B00F0F4840E2B2D
:10E4F00000F0F184079BD3F8008018F4806F61D09E
:10E50000134B1B79002B00F0248214210A48FCF7DE
:10E51000EBFA002840F0228217F038FD012022F0AB
:10E52000C3FD002849D0DFF82CA000244FF0CC0B0D
:10E53000A94614E016490020B062002038420020AD
:10E540001C6A0020206A0020C045002000410020F5
:10E55000B045002030830020DCB2022C2CD80BFB0D
:10E5600004F8631C5AF80850002DF5D1032290F9E5
:10E57000023002950192C278E34951F822200092BC
:10E5800018462A462B46012122F0F0F9034604EBF7
:10E59000440000EB00100D9353B129460AEB8000B4
:10E5A000CC222AF065FD0D9B4AF808300134E4B214
:10E5B0001BF0D8FC0028D0D14D46059B1C88079B3A
:10E5C000D3F80080089B1B7813F0010BCF4B00F0B1
:10E5D000C48201221A700A9B04991B68B1F90610C3
:10E5E0005A89CB484FF0010E914280F800E080F24A
:10E5F0009A82C84B4FF07E521A60C74A069B049815
:10E60000B3F81890B0F900E092F90430107892F85D
:10E6100001C0002BAEEB090314BF01224FF0FF3203
:10E62000002BB8BF5B42B3F5FA7FA8BF4FF4FA7373
:10E63000984280F23E831B1A07EE903AF8EEE77A92
:10E64000F145C7ED007A03DDF1EE677AC7ED007A98
:10E65000049BB3F902E0AEEB0903002BB8BF5B42A9
:10E66000B3F5FA7FA8BF4FF4FA73984280F21E8385
:10E670001B1A07EE903AF8EEE77AF145C7ED017AFA
:10E6800003DDF1EE677AC7ED017A049BB3F904006C
:10E69000A0EB0903002BB8BF5B42B3F5FA7FA8BF1C
:10E6A0004FF4FA736345CCBFA3EB0C03002302FBCA
:10E6B00003F207EE902AF8EEE77A4845C7ED027AB2
:10E6C000BCBFF1EE677AC7ED027A18F4805800F00B
:10E6D000CA82B1F5FA6F914BA8BF4FF4FA61B1F558
:10E6E0007A7F1A78B8BF4FF47A71A1F57A71002A4F
:10E6F00041F064808A4ADFF840E282FB0130CB17A8
:10E70000C3EB6013581C6FF0630C3EF910003EF928
:10E7100013E00CFB0313A0EB0E0003FB00F382FBE2
:10E720000312DB17C3EB62139E440FFA8EFE07EE53
:10E7300090EAB8EEE78A87ED038AB8F1000F40F05F
:10E740005984630640F1FA80764A774B92ED018A4C
:10E75000D3ED019A93ED026A92ED034A93ED030A19
:10E7600092ED029A93ED007AD2ED005AD7ED011A9C
:10E7700097ED002A6D4B6E4A38EE445A79EEC63A50
:10E7800077EE007A65EE233A75EEC96A75EE890A6E
:10E7900037EE401A66EEA76AB0EE633AA0EE813A11
:10E7A00014F00304B0EE665A78EE044A79EE867AE5
:10E7B000A0EE815AF0EE638AA4EEA73AD4EEA78ABF
:10E7C000A4EEE75A33EE263AF0EE687AF0EE674AA6
:10E7D000F6EE008A35EE88AAE0EEC14A28EEC33A8A
:10E7E00035EE635A77EE293A77EEE67AAAEE233AC7
:10E7F00025EE285A76EE403A34EE49AAE0EE817AC8
:10E8000074EEA64AAAEE235A34EE094A37EE697A24
:10E8100064EEA84A63EE036AE4EE074A75EEC85A4E
:10E8200036EE006A67EEA87AB0EE667A95EE057A63
:10E83000E5EE056AE5EE867AB1EE648AF0EE665A98
:10E84000F0EE476AB1EE674AE8EE246A63EE270A03
:10E8500067EEA43AE4EE275AB1EE450AB0EE609AAC
:10E86000B0EE631AA4EE277A23EE244AE7EEA76AF5
:10E87000A5EE249AA0EE031AE8EE245AB0EE448ADC
:10E8800031EEA16AE0EE240AA5EE278A66EEA16ABF
:10E8900072EE028AE5EE033A61EE211A26EE096A6B
:10E8A000A4EEA47AA0EE274A0CBFD7ED022ADFED32
:10E8B000212A83ED005AA2EE256AE0EEA86AE2EE74
:10E8C000081A73EEA33A27EE227A34EE044AF0EEE9
:10E8D000005AE3EEA26AA2EE846AA1EEA57AC7ED21
:10E8E000016AC2ED376A82ED366A87ED006A82ED11
:10E8F000387A83ED013AC3ED027AC3ED034AECB9ED
:10E9000087ED027A1AE000BF24AE0308C536002066
:10E91000D023002048230020F8620020CC250020CE
:10E920001F85EB51A0000020F00A0020280B0020DA
:10E93000541E00200000000004690020BBF1000FFD
:10E9400040F0BA8123F064FE17B0BDEC068BBDE841
:10E95000F08F089B1B78DA077FF5DEAD4FF40F7060
:10E9600027F038FD00283FF428AE0EF017FE4FF4D4
:10E970000F7027F0DBFC00283FF41FAE0EF00EFEF8
:10E980004FF40F7027F0D2FC0028EED115E6D14CE1
:10E99000236899077FF565AD059B1F8847F0010740
:10E9A00027F00207059BBFB21F806AE50521CA4810
:10E9B000FCF79AF8002800F07485059BB3F80080F6
:10E9C00018F0040F00F0E8860621C348FCF78CF825
:10E9D000002800F05D8518F0400F00F0D686072172
:10E9E000BD48FCF781F800283FF46DADBB4AB2F991
:10E9F0000030002BB8BF5B42B3F5E17FBFF663ADDB
:10EA0000B2F90230002BB8BF5B42B3F5E17FBFF62D
:10EA10005AADB34BD3ED096A93ED057AD3ED077A7E
:10EA200093ED030A77EEA67A30EE070AF7EE000AB6
:10EA3000B0EE007AE7EEC70A30EE000AFBF7A0FD61
:10EA4000F6EE007A20EE670ADFEDA67A30EE277A3E
:10EA5000FDEEC76A16EE903A2033402B41F28D80CE
:10EA60009FEDA17AA14ADFEDA07A82ED007ABDEE9A
:10EA7000C07AC2ED017A17EE103A2033402BC2ED76
:10EA8000027A49D8DFED9A7AB4EEE70AF1EE10FA8D
:10EA900041F3E484DFED976A9FED977A01E0B0EEF1
:10EAA000670AB4EEC70AF1EE10FA70EE667AF6DC89
:10EAB0009FED927AF4EEC77AF1EE10FA41F17A8482
:10EAC0009FED8C6ADFED8E6A01E0F0EE477AF4EE9E
:10EAD000E67AF1EE10FA37EE867AF6D4DFED817A37
:10EAE000B4EEE77AF1EE10FA41F3FD82DFED807AC1
:10EAF00037EEC77A27EE076ADFED825ADFED826ACA
:10EB0000DFED827AE6EE256A67EE065AE6EE267AB1
:10EB1000A5EEA77AF0EE477AC2ED037AD3E428F4A3
:10EB20008074A4B2DCE4B1F5FA6F80F22C84187A18
:10EB30008B1A03FB00F3C2F5FA6293FBF2F3C3F105
:10EB4000640307EE903AF8EEE77A9FED717A714B25
:10EB500067EE877AC3ED007A4FE593F800A0BAF12B
:10EB6000000F7FF438AD6C4B1B68002B3FF433ADC6
:10EB70006A4B6B4A13F8030C127807931946A3F1FA
:10EB80000309059223F0C8FA079B002800F0C3840C
:10EB9000059A002A5AD109F1080199F8050023F0D5
:10EBA000BBFA002841F0C9835E4999F80A0023F0B6
:10EBB000B3FA002800F0C484059B022B41F0F583D2
:10EBC000594999F80F0023F0A7FA002841F0E8838B
:10EBD000564999F8140023F09FFA002800F0C484E5
:10EBE000059B042B41F0D783514999F8190023F074
:10EBF00093FA002841F0CA834E4999F81E0023F089
:10EC00008BFA002800F0C484059B062B41F0B483E6
:10EC1000494999F8230023F07FFA002841F0A7839F
:10EC2000464999F8280023F077FA002800F0C484B8
:10EC3000059B082B41F0A583414999F82D0023F04D
:10EC40006BFA00283FF4C7AC4FF0090A534603EBB8
:10EC500083034B443B4A324859789B7880F800A0A4
:10EC600011705370B7E4069B5A8B9142C0F28983AE
:10EC7000B1F5FA6FD4BFC2EB0101C2F5FA614FF4EE
:10EC80007A7303FB01F130480378C2F5FA62B1FBF5
:10EC9000F2F1002B3FF42EAD43782C4A01FB03F137
:10ECA00082FB0123C917C1EB631123E5DFED0E7A67
:10ECB000E3E4DFED0D7AC3E40C9B19780B9B01F0C4
:10ECC00001011868FEF776FD17B0BDEC068BBDE8B4
:10ECD000F08F00BF38420020B06200203C4200208C
:10ECE000000B0020DB0FC93F00000000A000002047
:10ECF000DB0F4940DB0FC940E4CB1641DB0F49C0B5
:10ED0000E4CB16C192E741B99730083C15A82ABE5A
:10ED10000AD7233C48230020C8360020FA330020BD
:10ED20001C00002004340020093400200E34002090
:10ED300013340020183400201D3400202234002019
:10ED400027340020CC360020CC2500201F85EB5135
:10ED5000012D04BF05238BF82030BAF1000F10D02D
:10ED6000069B3088B3F918100022134661F30F0296
:10ED700060F31F4261F30F03049861F31F43426085
:10ED80000360BD4CDBF8142023689A4280F0E084D5
:10ED900047F230520323CBF81C208BF8203002209E
:10EDA0000CF010F80CF0C0FC2268DBF81C301344A7
:10EDB0000422CBF818308BF82020012D40F09E86DD
:10EDC0002368DBF818209A42BFF420A999F80000C4
:10EDD00020B923F0CBF900287FF418A93B6823F071
:10EDE00002033B6022687388642101FB03234FF414
:10EDF00080600022CBF810308BF820208BF80320A5
:10EE00000BF0D0FF9BF82030FFF7C3B923F0B4F923
:10EE1000012807D1984C73882268642101FB0323E1
:10EE2000CBF81030B8F1000F02D0B379002B45D1E8
:10EE3000012D3FF4EBA8904CDBF8102023689A4298
:10EE4000C0F0638601238BF82030012D34D0F37994
:10EE5000012B47D023F01EF99BF82030FFF799B91A
:10EE6000BAF1000FD2D14FF48060B8F1000F00F07A
:10EE70000C830BF09FFF099A00231361079B1E6808
:10EE800016F480573FF4C8A81D217C48FBF72CFEE0
:10EE900000287FF4C1A87A4B03F1500803E0043343
:10EEA000984500F0C1851A78262AF8D19978DA7841
:10EEB0009142F4D2FFF7B2B86F4C93E723F0EAF82F
:10EEC00003224FF47A738BF82020CBF81C306A4C65
:10EED00065E7694C71E724F04004059BA4B21C80EF
:10EEE000FFF708BB23F0D6F8032240F6B8338BF8BF
:10EEF0002020CBF81C30604C51E7624F3B78002B50
:10EF000001F0FE80604BDFF8B481DFF8B4B1DFF8C8
:10EF1000B4A1069345465E46049099460EE019F862
:10EF200004109847032C28DC88B93B782AF8020F94
:10EF300001349C4205F1040580F24981072CE1B2BD
:10EF40003046DBF80430EADD984700B2EDE738F8E8
:10EF500024206B88801A4FF47A719B1A01FB00F011
:10EF600040F6CA0290FBF3F00844904240F2EE23D0
:10EF7000A8BF10469842B8BF184600B2D5E7434B29
:10EF80001B78990704D5424C237D042B00F2C885D9
:10EF900018F0300F3FF49AAA10200BF003FF202046
:10EFA0000BF000FF059A3B4BB2F800803A4F00226D
:10EFB0001A703A493A4A3B4C3B4800230B603B49A4
:10EFC00023604FF0000E036053609361C2F800E0CD
:10EFD000C2F808E0C2F814E0C2F81CE0C1F800E092
:10EFE0004B60C1F808E0C1F814E08B61C1F81CE087
:10EFF000FFF76DBA1D212148FBF776FD28B100F01F
:10F00000C3BC0436AE423FF49CAB31782629F8D11C
:10F01000B278F3789A42F4D2099BDB78002B7FF424
:10F0200090AB1648FBF760FDDFED217A002801F078
:10F030006B8038EE678A1F4A1F49FDEEC87ACDED16
:10F04000047ABDF910301B0382FB0302DB17C3EB0C
:10F05000A212C9F57A731BB203FB02F343F30F3319
:10F060004B4407EE903AF8EEE77A0123C7ED037AB6
:10F070000B70FFF766BB00BF306A0020B062002053
:10F080005032002030350020C46900208E4200201C
:10F09000F0820020A05B0020C04500208C5C002096
:10F0A0003C5C00206C2300202C240020645C0020A9
:10F0B00000007A44D34D6210C4230020A433002002
:10F0C000D45E0020521E0020DFF804B3DFF8049362
:10F0D000B04C98460BF15A074FF0010A59461BF8FD
:10F0E000010C23F019F8F8B19BF804009BF80230EA
:10F0F0009BF803E000EB400104EB8101013BD1F8F8
:10F10000A02003EB43034B4493420DD094F8CC2052
:10F1100081F89CE00AFA00F022EA0000C1F8A03071
:10F12000C1F8A48084F8CC000BF1060BBB45D5D107
:10F13000994B9A4A1B780B930A9B994C1B68D2F8FF
:10F1400000B00C93A4F19C0A4FF0000963686BB304
:10F150001F785FB3A168ABEB010100290BDB9AF8C4
:10F16000CC10012000FA09F021EA00010BF5FA7039
:10F170008AF8CC10A0600B9AC2B12178587804317B
:10F18000C9B2002840F0B281069A108B049A32F975
:10F19000111000F1C80E714540F386849AF8CC1026
:10F1A0009B7841FA09F1CA0740F13D8509F101094F
:10F1B000B9F1040F04F10C04C8D1FFF745B9754C3F
:10F1C00094F89630002B3FF4C1A8FFF7B3B8DDF8F0
:10F1D0001090744A07927449126842F2010AA1FB26
:10F1E000091B12EA0A0A4FEA9B1B00F064816F4D6B
:10F1F0006F48694C6F492E780078267008701EB1F0
:10F200006C490E7886F00106624C0F2184F82410B8
:10F21000002B00F0D682069D674BB5F826C0B5F8E6
:10F2200024E0069D109318462D8B0078634B1295B1
:10F2300094F825500995624D0495A3FB00535B0893
:10F2400003EB4303C31ADBB20F90CDF834C002F4D2
:10F2500080520C9304F128000BF59673CDF844907E
:10F2600097F80080DDF82490DFF86CC10994544CC5
:10F270000E91139200210A930896CDF814E0089B92
:10F28000002B00F0D981099B059D33F911201FFA4D
:10F2900082FEAE454FEA410303D30D9DAE4540F2D9
:10F2A00010825CF82120934580F0D081E25EBAF1B3
:10F2B000000F40F0E58101314145E25200F10600C6
:10F2C000DDDB0E9A099C3F4B84F824200F2A494627
:10F2D0000CBF01220022DDF8449084F825101A703A
:10F2E00000F07682384B3249324ADFF8B0A00993F9
:10F2F0001C46042001230B7013700BF063FDDAF839
:10F300000030A1686268E3605B1A934284BF002307
:10F3100084F82130079B3C781E68002C00F0188789
:10F32000069A2A4DB2F824E0178B254916F4805628
:10F33000284640F0748232460EE0437803EB8303A4
:10F3400003EB830303F2EE239BB20132944221F8D4
:10F35000023B00F102000ED015F81230002B00F035
:10F36000B481022BE9D001320B8821F8023B944290
:10F3700000F10200F0D1109A137801331370FEF7F8
:10F380002CBE41467FE41B7AC3F1640307EE903A3A
:10F39000FFF7D9BB541E002030410020306A002006
:10F3A000F01E00206C580020D34D6210B05E00208B
:10F3B000E00A0020E10A002072340020ABAAAAAAC9
:10F3C0003C490020314100200C4100204E340020F7
:10F3D000F13200206892030874340020C54CD4F840
:10F3E0008830A9EB0303002BFEF607AEC24AC34BDD
:10F3F000527C069933F812308A7DDFEDC16A9FEDA9
:10F40000C16AC97D9BB207EE102A07EE903AB8EEAA
:10F41000C77AF8EEE77A27EE267A67EE867A0B9AB5
:10F42000C4F88820C7EE876A40F2FF32FCEEE67A25
:10F43000CDED057ABDF81430934228BF134609B1CB
:10F44000D31A9BB2B048B14D0178B14C35F8116078
:10F45000226825F81130921B13440131AD4D236011
:10F4600001F00F021B0902702B80FEF7C6BDFDF7ED
:10F4700001FDA94BA94A1B68C31A93427EF7BDAD93
:10F48000A44B00221A80FEF7B8BD0BF08BFCF2E40F
:10F4900028F04004059B1FFA84F8A3F80080FFF7CA
:10F4A0009EBA059A148824F004041FFA84F8A2F87E
:10F4B0000080FFF789BA9A490E78A0E694F8943054
:10F4C000002B3EF46EAF089B1B7813F001037EF413
:10F4D00068AF012284F8943084F89520FEF761BF6C
:10F4E000844C012184F88C10FEF79EBE012800F0A8
:10F4F00084859AF8CC20012303FA09F309F1010964
:10F500001343B9F1040F8AF8CC3004F10C047FF4F2
:10F510001DAEFEF799BF591D99F8050022F0FCFDBC
:10F5200000283FF441AB059B012B40F0068709F111
:10F530000D0199F80A0022F0EFFD002840F0358710
:10F54000784999F80F0022F0E7FD00283FF440AB1E
:10F55000059B032B40F02487734999F8140022F08F
:10F56000DBFD002840F01787704999F8190022F058
:10F57000D3FD00283FF440AB059B052B40F00687E8
:10F580006B4999F81E0022F0C7FD002840F0F48670
:10F59000684999F8230022F0BFFD00283FF440ABF2
:10F5A000059B072B40F0E386634999F8280022F079
:10F5B000B3FD002840F0E586604999F82D0022F05F
:10F5C000ABFD00283FF407A8059B092B3FF403A8D7
:10F5D000FFF73ABB099A01239370FEF7C6BD059B5E
:10F5E00047F002071F80FEF74CBF5D2A00F01D8325
:10F5F0005B2A00F0AA855E2A00F03C86562A00F0BD
:10F600003C86972A00F0A586A72A00F024864C4B5A
:10F6100005931B88980740F0AE85A2F1B703072B2E
:10F6200000F22F83DFE813F025032D032D032D03B4
:10F630001D032D030D030D03059B002B3FD05CF82C
:10F64000212093454FEA4103FFF430AE3D4A3D4D42
:10F65000D25C05EB030E002A00F0D380022A47D1CA
:10F660009EF8012002EB820202EB820202F2EE22FD
:10F6700092B2032933DD12B2BAF1000F3FF41BAE90
:10F680000C9D20F81520B9F1000F03D10F9D022D1C
:10F690007FF611AEB0F802900288B0F804E04A4458
:10F6A0009644294A0FFA8EFE82FB0E52274DA2EB9A
:10F6B000EE7225F803E012B24FF00109FBE51A469D
:10F6C0004B000A9D4CF82150F1E5D3B2022B04D92E
:10F6D000032B7FF448AE734637E63B4635E60125FB
:10F6E00005FA01FE0E9D25EA0E0512B20E95DEE525
:10F6F000E25ABEE7541E0020746C0020946C002077
:10F700000000C842000080444B5F0020505F002092
:10F710004C5F0020C44000206024002060E31600FD
:10F7200030410020093400200E3400201334002022
:10F73000183400201D3400202234002027340020FB
:10F740008C4200204E34002056555555C41E0020D2
:10F75000BE4B1B78002B7FF41BABBAF1000F3FF4BC
:10F7600017AB012D7EF452AC9BF82030FEF711BD93
:10F770003146B748FBF7B8F9002800F0B48084F8A8
:10F7800093600CF0ABFBFEF7A8BD059B48F040086A
:10F79000A3F80080FFF723B9AE4BAF4AB3F90430AA
:10F7A000AE4982FB0302DB17C3EBA203059A0B8071
:10F7B00048F00408A2F80080FFF706B95B78FFF76D
:10F7C0006CBAA74BA74A109201221A70A64B049359
:10F7D0001B219F48FBF788F900287FF483ADA34BDA
:10F7E000DFF898A209931946DAF80030CA688B60EE
:10F7F0009B1AC82B00F2B084079B1E6806F4805643
:10F80000B9E5CAB2022A40F2F583032A7FF470AF49
:10F81000129A139D059E002D08BF324629E700224B
:10F820000FE0437803EB830303EB830303F2EE2340
:10F830009BB20132A24221F8023B00F102003FF4E8
:10F840009AAD15F812301BB1022BEAD00B88F0E705
:10F85000D3B2032BFAD83B46EBE7B2F5FA7FFEF6BC
:10F8600095AD94F89230002B7EF490AD089D2B78E6
:10F87000012113EA010084F8921000F00C847C4A04
:10F88000927823F001032B70002A3EF47FAD794C6F
:10F8900023780B2B17D8994040F6030211427EF4CF
:10F8A00075AD11F4C06F0ED0093B012B0BD845206C
:10F8B00023F006FEFF2023F003FE6F4823F0ECFD4B
:10F8C000002023F0FDFD6D496D4A079B09685160DA
:10F8D0000B221B6822706B4A05926B4A0A9203F056
:10F8E0000403FEF75BBD089B684A1B781060DB07CA
:10F8F0007EF5F7AC664B1B78002B3EF447AD099BB9
:10F90000DB78002B7EF442AD94F893300133DBB208
:10F91000032B84F893307EF639AD5E4B5B7813B9D8
:10F92000002D7EF433AD0BF0FFFEFEF7D6BCB2F532
:10F93000FA7FFEF62BAD94F89220002A7EF426ADD5
:10F94000089B1B780121DF0784F8921000F1C68321
:10F950000CF0C4FAFEF71ABD4F4A50491068B4F9CA
:10F960009020C66981FB06018911F617701A00F50F
:10F97000FF407F3082423EF7A3AC891B0A4412B29B
:10F98000A4F89020FEF79CBC099BDB78002B7FF449
:10F990003CABDFED437A414938EE678AC9F5FA633B
:10F9A000FDEEC87A1BB2CDED047ABDF9102012032A
:10F9B00081FB0201D217C2EBA11203FB02F343F356
:10F9C0000F334B4407EE903AB8EEE78A87ED038A8F
:10F9D000FFF71BBB194608931B78DD077EF502ABCA
:10F9E000234A927823F001030B70002A3EF4FAAA0E
:10F9F000204C23780B2B0DD801229A4040F60305AA
:10FA000015407EF4EFAA12F4C06F03D0093B012B1E
:10FA100040F23F85DFF864A0194BDAF800205A6005
:10FA20000B232370FEF7DEBA1E4A069BD588049A84
:10FA30001B8BB2F906105A1B914240F39B802B445A
:10FA40009942B4BF00250125FEF7F1BA88230020B2
:10FA5000B06200203C42002067666666AC5C002015
:10FA600031410020723400203C4900200C4100202C
:10FA70000E4900200C490020B8BB0308306A002062
:10FA8000D06200208C4200209442002018250020E3
:10FA9000304100202063002074440020D34D6210C8
:10FAA00000007A44E03C0020C838814254DA9AF8D9
:10FAB000CC109B7841FA09F1C8073FF577ABC3F149
:10FAC0000008791E162900F28781DFE811F0310263
:10FAD00045021702670159026A020402F101B201EC
:10FAE0009D0188018501670177016A020402F10125
:10FAF00053013F012B017D02150100010999226884
:10FB0000CB6913448B61FEF781BA22F0C3FA03225A
:10FB100040F6B8338BF82020CBF81C30FFF73FB904
:10FB20000A2022F023FB8146002800F0BC8218F056
:10FB3000100F00F0F383C94C94F8D490B9F1000F82
:10FB40007EF4C4ACC64F012384F8D430B9F1000F61
:10FB50007FF42FAAFEF7BBBC9AF8CC30012202FA40
:10FB600009F223EA02030BF5FA728AF8CC30A2609C
:10FB7000FFF71CBB0125FEF75ABAB4EEE70AF1EE17
:10FB800010FA40F382849FEDB76ADFEDB76A01E0B7
:10FB9000B0EE677AB4EEE67AF1EE10FA77EE467AD6
:10FBA000F6DC9FEDB27AF4EEC77AF1EE10FA40F18E
:10FBB00059849FEDAC6ADFEDAE6A01E0F0EE477A62
:10FBC000F4EEE67AF1EE10FA37EE867AF6D4DFED4F
:10FBD000A97AB4EEE77AF1EE10FA40F33083DFED64
:10FBE000A67A37EEC77A27EE076ADFEDA45ADFED73
:10FBF000A46ADFEDA47AE6EE256A67EE065AE6EE21
:10FC0000267AA5EEA77AFEF72DBF00219E48FAF7C7
:10FC10006BFF00287EF49AAB322384F89600A4F898
:10FC20009830FEF793BB98464BE7984A00219848D6
:10FC3000984C0260984A0592984A21700A92FEF701
:10FC4000ADBB964A0A921146924B954A0A6002222F
:10FC50005A7022F0EDFA079B1B6803F00403FEF7CD
:10FC60009DBB8E4A0A9211468E4A0A60894B002239
:10FC7000EEE78A4A0A9211468B4A0A60854B0122B6
:10FC8000E6E79E2A00F0DA839D2A00F0D083AE2AB0
:10FC900000F0C683AD2A00F0BC83EF2A00F0B683E3
:10FCA000FD2A00F09F83FB2A00F02C84FE2A00F03E
:10FCB0002684F72A00F020847B2A00F08D83079B9E
:10FCC000764A1B680A9203F00403FEF767BBDAF872
:10FCD000D000764B90F836109A7841446429A8BF3A
:10FCE000642121EAE17180F83610002A40F0EE83A9
:10FCF00013F0BEFAFFF7FDBBDAF8D0006B4B90F8BB
:10FD000037109A784144FE29A8BFFE2121EAE1710B
:10FD100080F83710002AEBD0162022F06FFADAF8BC
:10FD2000D000E5E7DAF8D0008178604B4144C8297B
:10FD3000A8BFC82121EAE17181709B78002BD7D040
:10FD4000142022F05BFADAF8D000D1E7DAF8D0001C
:10FD50004178564B4144C829A8BFC82121EAE17126
:10FD600041709B78002BC3D0132022F047FADAF8B9
:10FD7000D000BDE7DAF8D00001784C4B4144C829E7
:10FD8000A8BFC82121EAE17101709B78002BAFD098
:10FD9000122022F033FADAF8D000A9E70C9A434B8C
:10FDA0009179987841446429A8BF642121EAE171DE
:10FDB0009171002840F0BC830D2F0DD00C983B4B67
:10FDC00041799A7841446429A8BF642121EAE1710C
:10FDD0004171002A40F09983DAF8D00088E7DAF818
:10FDE000D000324B017A9A784144C829A8BFC82173
:10FDF00021EAE1710172002A3FF47AAF0B2022F070
:10FE0000FDF9DAF8D00073E7DAF8D000274BC179B2
:10FE10009A784144C829A8BFC82121EAE171C1717B
:10FE2000002A3FF465AF0A2022F0E8F9DAF8D000A2
:10FE30005EE7DAF8D0001D4B81799A784144C829F1
:10FE4000A8BFC82121EAE1718171002A3FF450AFB7
:10FE5000092022F0D3F9DAF8D00049E7541E002037
:10FE6000C0450020DB0FC940E4CB1641DB0F49C081
:10FE7000E4CB16C1DB0FC93FDB0F494092E741B924
:10FE80009730083C15A82ABEB0620020CA4700205F
:10FE900090420020B04700208C4200209442002075
:10FEA000EE480020D6480020E24800200E490020FD
:10FEB000DAF8D000C74B41799B784144C829A8BFE4
:10FEC000C82121EAE1714171002B40F02B83112FF1
:10FED0007FF42AAF0CE7DAF8D000BE4B01799B78AB
:10FEE0004144C829A8BFC82121EAE1710171002B52
:10FEF00040F01283102F7FF42BAFF9E60C9A1179A2
:10FF00008844B8F1640FA8BF4FF0640828EAE87885
:10FF100082F8048022F08CF9AE4B9B78002B3FF4E2
:10FF20005BAF0320414622F069F9DAF8D000DFE642
:10FF30000C9AA84B11784144FA29A8BFFA2121EA6A
:10FF4000E17111709B78002B3FF446AF012022F045
:10FF500055F9DAF8D000CBE60C9A9E4B91784144E3
:10FF60006429A8BF642121EAE17191709B78002B7C
:10FF70003FF432AF022022F041F9DAF8D000B7E6C0
:10FF80000C98944BC1799A78414481F30801C1716E
:10FF9000002A3FF421AF052022F030F9DAF8D00032
:10FFA000A6E6DAF8D0008B4BC1789B784144C8298B
:10FFB000A8BFC82121EAE171C170002B40F08A82FC
:10FFC0000F2F7FF4D9AE93E60C9A824B51784144BF
:10FFD000B1F5967FA8BF4FF4967121EAE171517097
:10FFE0009B78002B3FF4F8AE152022F007F9DAF8E1
:10FFF000D0007DE6129AFFF73CBB049A987832F95C
:020000040801F1
:10000000111040F633039942A8BF1946B1F5617F3C
:10001000B8BF4FF461710C2FA1F561714FF4966375
:1000200093FBF0F391FBF3F100F0F480182F7FF4D1
:1000300060AADAF8D030C9B2C82993F817E00846A8
:10004000A8BFC82086453FF454AA624AD875927862
:10005000002A3FF44EAA384622F0D0F8FFF749BAFA
:100060005D4B5E491A684FF47A73B3FBF2F3C3EB4E
:10007000431203EB8202079B1B68D2001D06A1F806
:10008000A8203EF577A9564A0592564A0A9203F0EF
:100090000403FEF783B9079B84F89200FA3A1B68C1
:1000A000A4F89020EFE718F0100F40F02B810B2000
:1000B00022F05CF8002840F0EC804B4F18F0200F45
:1000C00040F04081494C94F8D430002B3FF43BADD4
:1000D000B9F1000F7EF46DAFFEF7F9B94449079B03
:1000E0000A601B68CFE7DFED437AB4EEE77AF1EE02
:1000F00010FA44BFDFED407A37EEC77AFEF7FABC5C
:100100003E4A0692FFF765B838EE678A3C4B3D4998
:100110001870FDEEC87AC9F5FA63CDED047ABDF921
:100120001020120381FB0201D217C2EBA1121BB2F5
:1001300003FB02F343F30F334B4407EE903AF8EE20
:10014000E77AC7ED037AFEF7FCBA2F4A01216EE584
:1001500006F48056FFF70FB92C4A079B1E681368F8
:1001600023F004031360099A012306F4805682F8F1
:100170002130FFF700B90023BB2A149300F06B81F4
:10018000B72A00F06481BE2A00F05F81BD2A7FF4A7
:1001900078AD4FF6FE711E4A1248D5890A909089B3
:1001A0002B4401449181D3811DF0FCFDFBF70BF83A
:1001B0001DF0E0FDFBF7C2FD079BB4F890201B6823
:1001C000FA3A0021A4F8902003F0040384F8921076
:1001D000FEF7E4B80E4900205C5800206C50002067
:1001E0008C42002094420020C0450020541E002074
:1001F00018250020DB0FC9BFDB0F49C0C4690020F0
:10020000C4230020D34D62101848002088420020EB
:1002100000630020C84B5B785FFA81F843453FF4E8
:1002200068A940460CF0CEFDC44B9B78002B3FF4F0
:1002300060A94146384621F0E1FFFFF75AB9DFEDEA
:10024000C07AB4EEE77AF1EE10FA44BFDFEDBD7A82
:1002500037EEC77AC7E4BC49079B0A781B68BB48DE
:10026000059042F004020A70B94A0A9203F00403AE
:10027000FEF794B8B74A0221D9E41DF093FDFAF7CE
:10028000A2FF1DF077FDFBF759FD94F88E20FFF7D4
:10029000B8B9B14BB14F5B8997ED007A07EE903A50
:1002A000F8EEE77AB0EEC77AB4EEE77AF1EE10FA3C
:1002B0007FF504AF97ED017AB0EEC77AF4EEC77A16
:1002C000F1EE10FA7FF7FAAE18F0200F7FF4FAAED5
:1002D00020200AF06FFD94E80C00A1490A6008464E
:1002E00041F8043F18F0EEF89E4B01221A709E4C24
:1002F00094F8D430002B00F0E280059BB3F8008026
:10030000FEF757BE10200AF04DFD964B059A83F874
:100310000090B2F800804FF00109C8E610200AF002
:1003200049FD20200AF03EFD90498C4F081F18F02F
:10033000C9F88C4B02221A70D9E74FF0010A5346D4
:10034000FEF785BC20200AF02DFD864B00221A7096
:10035000CDE7079B864A7D491B6805914FF4C8711C
:1003600011807B4A0A9203F00403FEF717B84FF09E
:10037000070A5346FEF76BBC4FF0060A5346FEF7DA
:1003800066BC4FF0080A5346FEF761BC4FF0050A01
:100390005346FEF75CBC4FF0040A5346FEF757BCC9
:1003A0004FF0030A5346FEF752BC4FF0020A534681
:1003B000FEF74DBCB0EE677AFEF790BB002D3DF422
:1003C00087AE694C94F88D30002B3DF433AF002399
:1003D00084F88D30FDF72EBF4FF4FA6102200CF047
:1003E00017FC6CE4002101200CF012FCB4F8902002
:1003F000079B57491B680A91963AA4F8902000225F
:1004000003F0040384F89220FDF7C8BF00210846DA
:10041000EAE7FF21002011F080FE94F88E203CE4F2
:100420000121002011F079FE94F88E2032E40021A1
:10043000FF2011F072FE94F88E2028E400210120A4
:1004400011F06BFE94F88E201EE40221A3E61946FB
:100450004FF6FE739FE6194602239CE6F0EE407AC3
:10046000FEF726BBB0EE677AFFF7B1BB374A94F8C8
:1004700096300592364A84F8941084F895000A92D2
:10048000002B3DF463AFFDF755BFF0EE477AFFF761
:1004900088BB452023F014F8FF2023F011F83548DD
:1004A00022F0FAFF284623F00BF8FFF7B3BA2E4CE0
:1004B0000BF03AF9002384F88D30FDF7BBBE059BA5
:1004C0004FF00109B3F80080FFF73DBB172021F082
:1004D00095FE81E40F2021F091FEDAF8D0006FE55F
:1004E000002B3FF46EAF2449244A09684FF47A7018
:1004F00000FB0313136064E70021042074E700216C
:10050000032071E7002102206EE70E2021F076FE25
:10051000DAF8D000FFF7ECBB102021F06FFEDAF81C
:10052000D000E7E4112021F069FEDAF8D000CEE433
:100530000D2021F063FE3FE4B04700200E4900206B
:10054000DB0FC9BFDB0F49C08E4200208C42002068
:100550009442002066480020305C0020C045002006
:1005600040240020A05B0020541E0020985B002047
:100570001E690020B8BB0308306A00201425002043
:100580002DE9F843C74C636820469847002800F0DF
:10059000C380C54B1B780122042B84F83C2000F05B
:1005A000BD80B4F91610B4F91820B4F91A302163DB
:1005B0006263A363BD4B1B88002B69D0BC4DD4ED97
:1005C0000C7AD5ED004A95ED050A95ED015A95EDA9
:1005D000067AD5ED035A95ED026AF8EEE76AD5ED95
:1005E000047AA4EEA60AA5EE267A67EEC07AA5EEF6
:1005F000C07AE6EE267A85ED057AC5ED067A27F013
:1006000071FDD4ED0D6AD5ED094A95ED0E0A95ED13
:100610000A5A95ED0F7AD5ED0D7AD5ED0C5A95ED78
:100620000B6A2063F8EEE66AA4EEA60AA6EE857AC7
:1006300067EEC07AA5EEC07AE6EE267A85ED0E7AF0
:10064000C5ED0F7A27F04EFDD4ED0E6AD5ED124AB6
:1006500095ED170A95ED135A95ED187AD5ED167AA2
:10066000D5ED155A95ED146A6063F8EEE66AA6EECC
:10067000A40AA6EE857A67EEC07AA0EE657AE6EE69
:10068000867A85ED177AC5ED187A27F02BFDA063E1
:10069000884EA17F884814F087FC3388002B40F0F7
:1006A0008180864DD5F8E400854B1B685B0743D4F9
:1006B00004F130012AC9B0F90060824A824F92EDFC
:1006C000026AD2ED006AD2ED015A891B2163B0F9AA
:1006D00002609B1B6363B0F904003E68281A07EEB2
:1006E000900AB8EEE75A07EE901AB8EEE77A07EEEE
:1006F000903AF8EEE77A36EE056A36EE877A77EECC
:10070000A57A0136A06382ED026A82ED007AC2ED1D
:10071000017A3E60BDE8F883BDE8F8836B4BB4F91D
:100720001600B4F91810B4F91A2018802063598003
:1007300061639A80A2633DE7B5F89830322B00F0F0
:100740008580002B63D195F89530002BB0D0D5F87B
:1007500000215F4E5F4986FB0273D217C2EB231262
:100760000280D5F8042186FB0273D217C2EB231254
:100770004280D5F80831A78A86FB0362DB17C3EBFA
:100780002213DB1B83800023CB6085F895301DF09E
:1007900009FBFAF718FD1DF0EDFAFBF7CFFAD5F8D3
:1007A000E40085E7454D216BD5F8E400B3F5C87F3B
:1007B0004FF0000323630380328814BFD5F8E8703C
:1007C0000027B2F5C87F18BFD5F8EC30328839441D
:1007D000676BC5F8E8104FF0000E3B44B2F5C87FD8
:1007E000C4F834E0C5F8EC30A0F802E051D0D4F8F9
:1007F00038C0D5F8F070C4F838E06744012AA0F892
:1008000004E0C5F8F07069D0013A32804CE7D5F8C1
:100810000061216B00223144C5F80011226302807F
:10082000D5F80461616B62633144C5F804114280FC
:10083000A16BD5F80861A2633144012BC5F80811FA
:10084000828073D0013BA5F898307CE7028822496A
:10085000204E276BA5F8F4200022B0F802E0B0F893
:1008600004C0F6684A608A602263C5F8007102809D
:10087000616BC5F8041162634280A16BC5F8081171
:10088000A263A5F8F6E0A5F8F8C0C5F8FC60828080
:10089000D8E7A36BC5F8F030C4F838E0A0F804E05E
:1008A000B2E700BF44420020CC440020043D0020B9
:1008B000083D00201E69002074420020541E0020C4
:1008C0006C580020D4680020D0680020D04400205C
:1008D0001F85EB5100630020541F00201D4ADFF8E4
:1008E00078C0C83182FB0198C833C917C1EBE81141
:1008F00082FB0398DB17C3EBE81343800180C83702
:1009000082FB0732A18AFB17C3EBE2135B1A8380D9
:10091000CCF80CE01DF046FAFAF755FC1DF02AFA67
:10092000FBF70CFA3288D5F8E4006DE70A49B5F810
:10093000F4E0B5F8F67085F89A20B5F8F860D5F8C7
:10094000FC20A0F800E04780868085F89430CA60DB
:1009500078E700BF1F85EB51006300202DE9F047C9
:10096000894B1B78DB07064641D5884B884D1C78A0
:10097000884F012C56D01CD3022C07D18649874AB8
:1009800009881288914201D901241C70EB7AE3B1E5
:100990002B89D3B1824B1B78BBB10CF035FA002800
:1009A00000F093802B7B83422CBF01210021397002
:1009B0000CE079497B4A098810886A7B801A884252
:1009C000E2DAEB7A0024002BE2D139782A79632A23
:1009D00006D8022C744D00F0B2802B78002B51D138
:1009E000724B8C4238BF0C461C70BDE8F0876A4BD6
:1009F000674D19885B88E878CB1A83EAE3728142F5
:100A0000A2EBE3721DD32B788B421AD35F4B1C7879
:100A1000E01E01285CD96649097802294AD0012CD8
:100A20005C4FA8D15D4A5C491288687B0988121A1C
:100A3000914234DD5B4A12888A42A7D200241C709E
:100A4000A4E7B1EB400FE1DC504B1C78E11E01291B
:100A500040F29180022ADEDC55494E4F0878DFF8DB
:100A60004081DFF840C1DFF834E10021032402288F
:100A70003C701C7088F80010ACF80010AEF8001044
:100A800084D11AE06868301A4A4B98425CDD474BC3
:100A90006A708C4238BF0C461C70BDE8F087022497
:100AA0001C7073E7022AD7DD4149097802294FF00B
:100AB000040466D13A49374F09783F48022ACCBF2F
:100AC00000220122C280818053E7022139707DE734
:100AD000022AA0DC95F800C091FBFCFC0CF1010C93
:100AE000BCF1080FDFF8B8A0314FA87895F801E005
:100AF00097F800802B4CDFF8A490264FA8BF4FF04A
:100B0000080C8AF800C01FFA8CFA10FB0AF01EFBD2
:100B10000AFE80B2DFF890A02080A9F800E000244F
:100B20004FF0640EB8F1020F3C701C70CAF804401C
:100B30008AF801E07FF441AF0FFA8CF1BDE7287825
:100B4000B0B901236E602B70C2F164021B4B00FB35
:100B500002F083FB0023C017A0EBA3508C42134B81
:100B600000F1640038BF0C4668701C70BDE8F08767
:100B70006B68F01A88E7032C94D10D490978022993
:100B800098D0044F02E700BFC4360020C4250020DF
:100B900028420020D4250020A8450020C825002098
:100BA000BE450020C6250020CC250020443500206D
:100BB000CC4400207F969800D04400206BCA5F6B25
:100BC0002DE9F04F2DED028B93B0064615F0DEF9BE
:100BD0009A4B1D7825B113B0BDEC028BBDE8F08FA8
:100BE000974B1B685C05F6D5964F3A68002A00F0D3
:100BF0002181954CD4F8283103F5F43348339E42D3
:100C0000C0F01881DFF8888294F82C31D8F80010F1
:100C1000C4F828610133DBB2880784F82C3101F174
:100C2000B886080700F1BE8113F0070901F06C8552
:100C3000282B864B029301F0FA875E209047844B65
:100C40001B78002B6BD0804C824AD4F83431F31AD5
:100C5000934201F21F84DFF83CA29AF80090B9F1A8
:100C6000000F33D1DFF8FC81D8F80000FCF760FBFF
:100C7000C0B201280ED90228774F42F095803B7808
:100C8000002B42F06781D4F83C31F31AB3F57A6F48
:100C900082F0028271480268002A40D09AF800303F
:100CA000BBB96F4BD8F800001B689B781E3B012B2B
:100CB0004FF0020142F2A381043015F01FF8012227
:100CC00000238AF8002084F8483126E0634802684F
:100CD0002AB3D4F8443140F6B731F31A8B421ED907
:100CE00094F84031002B02F05580013BDBB284F8D0
:100CF0004031002B01F0BB8612F8011B94F84871BB
:100D0000026094F849315748CA190133006884F8E1
:100D1000482184F84931FCF70FFBC4F84461524A7A
:100D2000029B12781B68012A03F101030A9301F068
:100D3000DB824E4B1B786BB14D4F3B6853B1029B2E
:100D4000414CD3F800B0D4F85C31ABEB0303632B18
:100D500001F2FF81DFF8408198F80090B9F1020FAD
:100D600001F05F863C4F97F87430032B01F09584B7
:100D7000404B1B7873B1404D2B685BB1324CFCF794
:100D800079F8D4F86831039044F61F62C31A93428D
:100D900000F25C81394B1B78002B7FD1384B1B78DC
:100DA00043B1294CD4F8B83203F50043E8339E42EE
:100DB00081F01083334B1B78002B3FF40CAF224E95
:100DC000314C324D06F2C1272068FCF7B1FA0028F9
:100DD0003FF401AF2068FCF7A7FA2B7880465A1E33
:100DE00033B120682A70FCF7A3FA0028F2D1F2E6AA
:100DF00003223946781E28F021F996F8C03296F879
:100E0000C12286F8C38283F47F4383F0FF039B1AD9
:100E10001FFA88F89BB2B8EB132FD5D196F8C222EF
:100E2000DBB29A42D0D1781E16F05AF92B781844CA
:100E30002870C9E7054B029301E700BF164900205F
:100E40006C580020B0420020601F0020306A002053
:100E5000424300203F0D030020000020A842002054
:100E6000A4420020A0420020434300205043002021
:100E70007C470020584300205C430020C8430020EA
:100E8000D943002062430020684300206C430020C7
:100E900038420020AC420020A23000205E4C227874
:100EA000002A41F018825D4F3C78002C40F0A7806A
:100EB0005B4D2878002841F0CD875A4C5A4DD4F824
:100EC000B0122A78594B93FBF2F30B449E42FFF485
:100ED00065AF574A94F8B432C4F8B062D75CFA07E9
:100EE00002F1FF80BB0702F1A381780702F166815E
:100EF0003A074CD54F4BDFF850810B930DF1480961
:100F0000A3F13D0249F8202D0021A3F1400203F88E
:100F1000401C02231121517093704846D8F80010EC
:100F2000F9F768F94846D8F80410F9F763F9B8F802
:100F30000E30414903EBC3039B00053381FB0321C2
:100F4000DB17C3EBA10189B24846F9F76BF9B8F892
:100F5000103003EB8303590089B24846F9F762F970
:100F6000364B1B789B0743BFB8F8081001F57A7120
:100F700089B24FF47A714846F9F754F90A9B98F808
:100F80001420591C0A9148461A7014F0A5FF94F8D1
:100F9000B4322978013393FBF1F201FB123384F868
:100FA000B432FBE613F0030A7FF43EAE5E209047B6
:100FB0003B6814209847224B1F4AB3F9043082FB48
:100FC00003124FEAE379C9EBA2090FFA89F95FFA34
:100FD00089F014F0E7FEC9F3072014F0E3FE3B6844
:100FE0005E2098473B681C209847504614F0DAFE74
:100FF000504614F0D7FE94F82C313A6814E6114D9F
:10100000286E002841F0EE858146064B87F8009057
:10101000C3F8B062C2E600BF34430020D1430020D1
:10102000D0430020601F0020D8430020A08601008C
:10103000D4430020F4420020676666668E4200209A
:101040003C420020E0430020F082002094F86E3102
:10105000002B41F02485DB4B1A6802F00803002BBB
:1010600048F603414AF60B404BF60F4349F6074753
:1010700004BF03460F4612F0040F4FF0190118BFCA
:101080001F46930684F86E1103D547F4804747F056
:1010900020070BF0ABFEC7F30909002842F01681C8
:1010A000C94B9B79002B42F0F582984664204FF0A3
:1010B000FF3A4FF0000C0A970B97ADF834C0CDF80B
:1010C0003AC0CDF83EC0CDF842C0CDF83090ADF872
:1010D0003680ADF838A08DF846000AAF0FCFDFF8A4
:1010E00000E384F805C0AEE80F0097E80F00AEE813
:1010F00007002EF8023B71464FF0010C1B0CFE2737
:101100001F20C82201F81E39A770A27184F807C0F9
:10111000E07094F87E01207180F0F10383EA0313FC
:10112000DAB2130983F0E70343EA022383EAC20336
:101130001BB283EA0312D2B2C3F3072383EA12136A
:1011400043EA022383EAC2031BB283F0C80282EAA5
:101150000212D2B2C3F3072383EA121343EA022333
:1011600083EAC2031BB283EA0C0787EA0717FFB2C0
:10117000C3F3072282EA171242EA072200EB0C03AC
:1011800082EAC7070EEB0C0084F87E31278011F845
:10119000013B7B4083EA0313DBB21A0982EA172280
:1011A00042EA032282EAC3031BB29FB28142278034
:1011B000EDD183F07C0383EA0313DBB24FEA131E05
:1011C0008EEA172E8EEA032E8EEAC30E0FFA8EFEDB
:1011D0001FFA8EF9DFF80CC2A4F800905FFA8EFEB9
:1011E0004FEA192984F8289084F827E00CF5D37881
:1011F00004F1220ADCF80000DCF80410DCF8082016
:10120000DCF80C3047460FC70CF1100CD445B8463B
:10121000F0D1DCF8000038606C4F9CF8043088F89E
:10122000043007F1270884F8CDE184F8CE9117F84F
:10123000011F2868FCF780F8B845F8D194F86F31A1
:10124000002B41F031846249029A097812680A2021
:1012500084F86F01002901F0BE855E4F01293888AE
:10126000069042F20F820229B7F802E002F00181F3
:10127000B8880590032902F023820429B7F806B044
:1012800002F0198238890490052902F0108206299B
:10129000B7F80A9002F008820729B7F80C8000D04E
:1012A000FB8994F87E110A92084680F0300282EAA7
:1012B0000212D2B217094849079087F07A0747EA25
:1012C00002270988207187EAC202444FC1EB01213D
:1012D00087FB010A06984FF0000C60F30F0C05988D
:1012E0006EF31F4C4FF0000E60F30F0E0498CDF814
:1012F0002CC012B28A440027C917C1EB6A2A60F3D6
:101300000F0782EA02110020C9B268F30F00C2F38E
:10131000072269F31F4782EA11126BF31F4E63F332
:101320001F404FF00009CDF830E00D978DF83DA03B
:101330000E908DF83C9042EA01220DF1280C82EAD1
:10134000C107BCE80F003FB287F0C80888EA081858
:10135000DFF88CE084F805905FFA88F8C7F3072778
:10136000AEE80F0087EA181747EA08239CE8030055
:1013700083EAC8031BB283F023024EF8040B82EA0F
:101380000212D2B2C3F30723079F83EA12137046F7
:1013900043EA022383EAC20207F1010C20F8141980
:1013A0004FF023081621FE27C82384F87EC122802F
:1013B00084F80780A7700EF1020EE170A371114648
:1013C00012E000BF38420020284200200721002000
:1013D000D45E00203C490020C44000200308208047
:1013E000681F0020621F002010F8013B4B4083EA79
:1013F0000313DBB21A0982EA112242EA032282EACB
:10140000C3031BB299B270452180EDD183F0F40380
:1014100083EA0313DBB24FEA131E8EEA112E8EEA23
:10142000032E8EEAC30E0FFA8EFE1FFA8EF8CC4FF3
:10143000A4F800804FEA182C5FFA8EFE84F81EE0B4
:1014400084F81FC07968BA683868FB6807F5D378F4
:10145000A8E80F0038697969BA6904F2A717A8E803
:10146000070004F2C51884F8C5C184F8C4E117F870
:10147000011F2868FBF760FFB845F8D194F8723176
:10148000002B41F00783B74B1B681922980684F89C
:10149000722140F10B83B44BDFF8DC821B78990793
:1014A00041F11C8698F81430042B8CBF03270227C7
:1014B000FBF7E0FCB8F81030B8F808200A9003EB0E
:1014C00083035B00ADF842304FF47A70D8F80030F7
:1014D0000C93B8F80E1098F814C0D8F804308DF8B2
:1014E000447000FB02F24FF0000E4FF0FF300DF1A0
:1014F00028098DF845C0CDF82CE00E920D93ADF87B
:1015000040100F90CC46BCE80F00984F0FC79CE8E6
:101510000F0007C73A46182122F81C39E17194F8E8
:101520007E1184F805E081F0780383EA0313D8B2D2
:10153000030983F0F60343EA002383EAC0031BB2E6
:1015400083EA0310C0B2C3F3072383EA101343EA0C
:10155000002383EAC0031BB283F0C80080EA001EA8
:101560005FFA8EFEC3F3072080EA1E1040EA0E20C9
:1015700080EACE0000B280F0180383EA0313DBB2E6
:10158000C0F3072080EA131040EA032080EAC30377
:1015900001F1010C1E204FF0FE0E4FF0C80AE07062
:1015A0000237217184F87EC1238084F802E084F838
:1015B00006A0184612F8011B414081EA0111C9B288
:1015C0000B0983EA102343EA012383EAC10109B22C
:1015D00088B2BA422080EDD181F0180181EA011170
:1015E000C9B24FEA111B8BEA102B8BEA012B8BEA55
:1015F000C10B0FFA8BFB1FFA8BF3594A23805FFA5A
:101600008BFB1B0A0492059384F8273084F826B0DC
:10161000964602F5D37C04F1220ADEF80000DEF8DB
:101620000410DEF80820DEF80C3067460FC70EF114
:10163000100ED645BC46F0D14D4BDEF800003860A8
:101640001A4603F1260A9DF8143084F8CCB184F8C8
:10165000CD31934617461BF8011F2868FBF76CFE37
:10166000DA45F8D1FBF706FC424BDFF810C1B3F9BD
:101670000410B8F808E00A9098E80C008CFB010C04
:10168000C9174FF47A704FF0000800FB0EF0C1EB61
:10169000AC01ADF83C80ADF83E80ADF84080ADF8CF
:1016A00042100D900E900B920C93CC46BCE80F00AC
:1016B000DFF8B8E084F80580AEE80F009CE807008A
:1016C0004FF021088EE807001C23C8224FF0FE0CC3
:1016D000E370A27184F8078084F802C094F87E1148
:1016E000217181F06A0383EA0313DAB2130983F0EC
:1016F000D50343EA022383EAC2031BB283EA03123F
:10170000D2B2C3F3072383EA121343EA022383EA24
:10171000C2031BB283F0C80282EA0212D2B2C3F340
:10172000072383EA121343EA022383EAC2031BB2AC
:1017300083EA080282EA0210C0B2C3F3072282EAF7
:10174000101242EA0022013182EAC0020EF10C0EB0
:1017500084F87E112280AEF11C01104610E000BF1B
:10176000621F0020384200208E420020681F0020A7
:10177000072100203C420020F08200206766666658
:1017800011F8013B434083EA0313DBB21A0982EAF2
:10179000102242EA032282EAC3031BB298B27145C7
:1017A0002080EDD183F0680383EA0313DBB24FEAB4
:1017B000131B8BEA102282EA032B8BEAC30B0FFA6E
:1017C0008BFB1FFA8BF3DFF800E423805FFA8BFBBF
:1017D0001B0A059384F8253084F824B00EF5D37ADB
:1017E00004F12208DEF80000DEF80410DEF808201C
:1017F000DEF80C30D446ACE80F000EF1100EC645F2
:10180000E246EFD1BEF80030ACF800309DF814305D
:10181000DFF8B88384F8CAB1BA4684F8CB311AF835
:10182000011F2868FBF788FDD045F8D194F87EA108
:10183000E14A84F804A08AF0EB0383EA0313D9B2E7
:101840000B0983F0C50343EA012383EAC1031BB2FA
:1018500083EA0310C0B2C3F3072181EA101141EA01
:10186000002181EAC00109B20CCA81F0C80C8CEADF
:101870000C1C5FFA8CFC4FF0000EC1F307210B9398
:10188000CDF830E081EA1C130A9299E8070043EA98
:101890000C2383EACC03BB461BB2C84F84F805E097
:1018A00083F0310C87E807008CEA0C1C5FFA8CFC93
:1018B000C3F3072383EA1C1343EA0C2383EACC0314
:1018C00094F808C0607AA17AE27A94F80CE094F86F
:1018D00011801BB28CEA030C8CEA0C1C5FFA8CFCA6
:1018E000C3F3072383EA1C1343EA0C2383EACC03E4
:1018F0001BB2584080EA0010C0B2C3F3072383EA4A
:10190000101343EA002383EAC0031BB2594081EA63
:101910000110C0B2C3F3072181EA101141EA00218E
:1019200081EAC00109B24A4082EA0212D2B2C1F38E
:10193000072383EA121343EA022383EAC2031BB29A
:101940008EEA030E8EEA0E1E5FFA8EFEC3F30723A5
:1019500083EA1E1343EA0E23607BA17BE27B94F8AB
:1019600010C083EACE031BB2584080EA0010C0B218
:10197000C3F3072383EA101343EA002383EAC00377
:101980001BB2594081EA0111C9B2C3F3072383EAAC
:10199000111343EA012383EAC1031BB25A4082EACE
:1019A0000212D2B2C3F3072383EA121343EA0223DB
:1019B00083EAC2031BB28CEA030C8CEA0C1C5FFAAC
:1019C0008CFCC3F3072383EA1C1343EA0C2383EA4A
:1019D000CC031BB288EA030888EA08185FFA88F883
:1019E000C3F3072383EA181343EA082383EAC803EF
:1019F000A17CE27C1BB2594081EA0111C9B2C3F358
:101A0000072383EA111343EA012383EAC1031BB2CC
:101A10005A4082EA0212D2B2C3F3072383EA1213B6
:101A200043EA022383EAC2031BB283F0270989EA4F
:101A30000912D2B2C3F3072989EA121949EA022925
:101A400089EAC2090FFA89F90AF101031FFA89F23A
:101A500031205FFA89F94FF0FE0C0C2184F87E31B9
:101A6000C8234FEA122E07F5D0782280E07184F85F
:101A700002C0E170A37184F81490049F84F815E00B
:101A80007968BA68FB683868B7F810C0A8E80F0032
:101A90005F4628F803CB84F8BBE184F8BA9117F8C5
:101AA000011F2868FBF748FCB845F8D194F8767117
:101AB000002F40F0EA87424B94F87EC1B3F9001042
:101AC000B3F90220B3F904309FED3E6A677107EE67
:101AD000103A029B1B680A938CF06A0383EA031393
:101AE00006EE901AD9B20B0983F0D50343EA01231D
:101AF00083EAC1031BB283EA03115242C9B207EE63
:101B0000902AC3F3072383EA111343EA0123F8EE73
:101B1000E77AF8EEE66AB8EEC77A83EAC1031BB249
:101B200067EE867A66EE866A27EE067A002083F0F4
:101B3000C808CDED0C7ACDED0B6A8DED0D7A0E90C7
:101B40000F90109088EA081E0DF128095FFA8EFEAA
:101B5000C3F30728B9E80F0088EA1E1848EA0E28E0
:101B600088EACE08DFF854E00FFA88F8AEE80F00F4
:101B700088F01E0799E8070087EA0717FFB2C8F345
:101B8000072383EA171343EA07238EE8070083EA53
:101B9000C707C8214FF005094FF01E08FE231C207F
:101BA0000CF1010284F8769184F80780A370E0704C
:101BB000A171AEF110010BE0945B0020681F0020C2
:101BC0003C42002088C3E43A621F00202B21002001
:101BD00084F804C00EF10C0E278084F87E2111F8E1
:101BE000013B7B4083EA0313DBB21A0982EA172226
:101BF00042EA032282EAC3031BB29FB271452780E7
:101C0000EDD183F0270383EA0313DBB24FEA131EFF
:101C10008EEA172E8EEA032E8EEAC30E0FFA8EFE80
:101C20001FFA8EF9DFF8DCC3A4F800905FFA8EFE8D
:101C30004FEA192984F8259084F824E00CF5D3782C
:101C400004F1220ADCF80000DCF80410DCF80820BB
:101C5000DCF80C3047460FC70CF1100CD445B846E1
:101C6000F0D1E04FBCF80030A8F8003007F12408AC
:101C700084F8CAE184F8CB9117F8011F2868FBF7B4
:101C80005BFBB845F8D194F877B1BBF1000F40F099
:101C9000F686D54B1B68052284F877219A0641F118
:101CA0009480D24BDFEDD26ADA891B8907EE902A45
:101CB00007EE103AF8EEE77AB8EE477A67EEA67AC2
:101CC00094F87E81CB4BCC4AB3F90410B2F90620CC
:101CD000CA4FCB48CDED0B7A88F0220383EA031379
:101CE0005FFA83FE4FEA1E1383F0590343EA0E2383
:101CF00083EACE03B2F5FA6F1BB2A8BF4FF4FA62C3
:101D000083EA031E5FFA8EFEB2F57A7FC3F30723E0
:101D100083EA1E13B8BF4FF47A724FF0640C43EAA3
:101D20000E23A2F57A720CFB02F283EACE0E87FB39
:101D300002C780FB01C00FFA8EFEC917D217C2EB93
:101D4000A7124FF0000AC1EBA0038EF0C8070DF1F7
:101D500028098DED0C7AADF83A20ADF83830CDF881
:101D600028A0CDF834A0CC4687EA0717BCE80F00BE
:101D7000FFB2CEF3072E8EEA171E4EEA072E8EEA2A
:101D8000C707DFF894E2DCF800C084F80480AEE80E
:101D90000F003FB287F04A0383EA0313DBB2C7F3B5
:101DA000072181EA1311724641EA032108F1010873
:101DB00081EAC303142042F810C9FE274FF04A0CF1
:101DC000002184F87E814FF0C808E07023800EF176
:101DD000040E84F807C0A770617184F80680184665
:101DE00012F8011B414081EA0111C9B20B0983EAD3
:101DF000102343EA012383EAC10109B288B2724584
:101E00002080EDD181F0140181EA0111C9B24FEABD
:101E1000111E8EEA102E8EEA012E8EEAC10E794B2B
:101E20000FFA8EFE1FFA8EFC1F464FEA1C2A5FFA3D
:101E30008EFE84F81DA084F81CE0596838689A6802
:101E4000DB68A4F800C007F5D37CACE80F00386964
:101E50007969B7F818800497ACE8030004F2A71773
:101E6000ACF8008084F8C3A1B84684F8C2E104F25B
:101E7000C31A18F8011F2868FBF75EFAC245F8D1AB
:101E8000614B624A1B781278013B12F00100DBB211
:101E900014BFC0214021172B03D85D4A134493F887
:101EA00014B05C4B1A8893071ABF002341F010014D
:101EB000012312F4027F18BF022312F0100F18BF83
:101EC000062312F0200F18BF1023002841F0D48001
:101ED0004FF0030894F87EE10A938EF0460383EAFC
:101EE0000313DAB2130983F0920343EA022383EA6D
:101EF000C2031BB283EA0310C0B2C3F3072282EA13
:101F0000101242EA002282EAC00212B282F0C80C29
:101F10008CEA0C1C00235FFA8CFC0320C2F307221E
:101F20008DF82CB08DF82F8082EA1C128DF82D30A0
:101F30008DF82E108DF8300042EA0C2899E8070041
:101F400088EACC0C0FFA8CFCDFF8CC80E3718CEAC9
:101F50000C19A8E803005FFA89F9CCF3072C8CEA86
:101F6000191C4CEA092181EAC90994F808C088F8CB
:101F700000200FFA89F98CEA090C8CEA0C1C5FFA34
:101F80008CFCC9F3072282EA1C1242EA0C22607A16
:101F9000A17A94F80B90637182EACC0C0FFA8CFC56
:101FA00080EA0C0080EA0012D2B2CCF3072080EA6B
:101FB000121040EA022080EAC20000B2414081EAE9
:101FC0000111C9B2C0F3072282EA111242EA0122CA
:101FD00082EAC10212B289EA020989EA09195FFAA2
:101FE00089F91BE00721002038420020F082002000
:101FF0000AD7233C3C4200203C490020D34D6210CC
:1020000067666666621F002000410020C43600201B
:10201000B09203088C420020681F0020C2F3072200
:1020200082EA191242EA092294F80CC0607BA17B73
:1020300084F804E082EAC90212B28CEA020C8CEA4B
:102040000C1C5FFA8CFCC2F3072282EA1C1242EAE3
:102050000C2282EACC0212B2504080EA0010C0B2D8
:10206000C2F3072282EA101242EA002282EAC00288
:1020700012B2514081EA0111C9B2C2F3072282EAC9
:10208000111242EA012282EAC102E17B94F8109027
:1020900013B281EA030282EA0212D2B2C3F3072327
:1020A00083EA121343EA022383EAC2031BB289EADA
:1020B000030282EA0212D2B2C3F3072383EA1213A5
:1020C00043EA022383EAC2031BB283F0320282EAAC
:1020D0000212D2B2C3F3072383EA121343EA0223A4
:1020E00083EAC2031BB29AB24FF0FE0C5FFA83FB85
:1020F0000920C8210EF1010E84F802C04FEA122C0B
:10210000E070A17184F87EE1228084F812C084F826
:1021100011B0049B186859689A68B3F80CA008F5C8
:10212000CC7EAEE8070008F5D4788EF80290AEF8C1
:1021300000A084F8B8C184F8B7B117F8011F286867
:10214000FBF7FAF8B845F8D1039BC4F86831FEF7FD
:1021500021BEDFF828A3DFF82883DFF82893412089
:1021600015F03EFABAF9023088FB0320DB17C3EB07
:10217000A00080B215F018FABAF9003088FB0320ED
:10218000DB17C3EBA00080B215F00EFABAF90430E9
:1021900088FB0320DB17C3EBA00080B215F004FA24
:1021A00099F800103868FBF7C7F894F860A11AF0A6
:1021B000010800F0A184A44B1B689A067AD5A34BB2
:1021C000DFF8C4821B789B0740F11D8798F8143014
:1021D000042B8CBF4FF0030A4FF0020A472015F082
:1021E000FFF9D8F8000015F0ABF9D8F8040015F0A5
:1021F000A7F9B8F80E30964A3868A2FB0323C3F358
:10220000471319460393FBF797F8B8F8082099F895
:102210000010039B64204B4000FB02F089F8003063
:1022200015F08EF998F8148038684AEA88085FFA41
:1022300088F84146FBF780F899F80030386888EA5A
:102240000308414689F80080FBF776F894F860A10E
:10225000BAF1000F2ED1DFF834824F2015F0C0F90B
:10226000D8F8000015F06CF9D8F8040015F068F9FA
:10227000504615F065F901213868FBF75DF8734A9F
:1022800099F8003092F80080386808F0010883F06F
:102290000103414689F80030FBF74EF899F8003009
:1022A000386888EA0303194689F80030FBF744F8D8
:1022B00094F860A1674AC4F85CB10AF10103DBB28B
:1022C000A2FB0312D20802EB8202A3EB420384F8C2
:1022D0006031FEF73FBD604B60491868FAF7F8FFC0
:1022E00000232370FEF7DFBD5D4F386800283EF401
:1022F00020AD4FF0000ADFF898815A4CAB465546A6
:10230000FBF716F8F8B1F5B94FF00109AA4638689D
:10231000FBF70AF883B27E2B00F09A8398F801202D
:10232000002A49D194F84C11B1B11B2B84F84C21EF
:1023300000F066830D2B45D0386888F80190FAF7D5
:10234000F7FF0028E3D1AA4650460AAA46495D464F
:1023500013F074F9FEF7EDBC7D2B00F0468594F880
:10236000502122B180F02003DBB284F8501194F8A0
:102370004B21062A10D8B4F84E1138681944A4F835
:102380004E11A118013281F8543184F84B21FAF72B
:10239000CFFF0028BBD1D6E7B4F84E2188F80190D2
:1023A00013449BB21A0A52FA83F3FF2BA4F84E315E
:1023B000386802D12D4DA3E73868FAF7B9FF002835
:1023C000A5D1C0E73868A4F84E21FAF7B1FF00287C
:1023D0009DD1B8E794F8BC32C4F8B862012B40F242
:1023E000DD8494F8BD222249981801EB8001013266
:1023F00002F00102CF6A84F8BD22BFB11D4D0B95DA
:102400000DF14809123DA52349F8205D802284F88A
:10241000103115233146484684F8112184F81231D1
:10242000B847002840F03B8494F8BC32124A01338C
:1024300082FB0312A2EBE37202EB42029B1A84F8C6
:10244000BC32FEF7B7BC00BF384200208E420020ED
:102450001F85EB51CDCCCCCCCC430020F4420020E6
:102460009C420020601F0020AA200020B4200020F1
:10247000B092030885200020565555553C42002057
:102480006766666680470020F0820020945B00202B
:10249000200000208B4A8C4B92F80BC0029A1B88BC
:1024A0001168D4F83801894A5FFA83FE1F0A4FF495
:1024B0007A73091A03FB0CF30020994282F81EE09C
:1024C000D77782F814E057759070107180F05284BD
:1024D0007F49DFF81CE20B688F687E49DFF81482C1
:1024E000087898F814908EFB03C1DB17C3EBA101A9
:1024F0008EFB07CE1177FF170912C7EBAE07517796
:10250000F4214FEA272E82F820709176012730219E
:10251000D77682F82210704B82F821E07527782157
:1025200082F8237082F82410820783F81A9040F111
:102530001E84D8F800E0694AD8F80470DFF8B8B112
:10254000DFF8B8C182FB0E1A4FEAEE7082FB071269
:10255000C0EBAA50F917C1EBA2510BFB00E202EB52
:10256000420252000BFB017B00EB8000049201EB66
:10257000810100EB80000BEB4B0B4FEA4B0B0590FE
:1025800001EB8100049907908CFB022A8CFB0B2C39
:102590004FEAAC424FEAAA4AC9174FEADE7E0692DA
:1025A00083F809E04E4AB8F80EC0B8F80880AAEBE4
:1025B000010E0499F24602FB1A1A05994FFA8EFE93
:1025C0000EEB810E06994FEAEB7008F5FA780A1ABD
:1025D0001FFA88F8FF0F4249CDF80C8010469F7310
:1025E0000CEBCC0C079FDFF8188101FB12B24FEA0D
:1025F0008C0C3C4940B200EB870088FB0C789DF8BE
:102600000C705F754FEAEC7CCCEBA81C81FB0A7860
:1026100081FB0271D217B9F1050FC2EB6112DFF82D
:10262000E4900399B9F800B05A744FEAEA7ACAEB19
:10263000681A1FFA8EFE80B24FEA11282A4983F8E1
:102640000AE04FEA1E294FEA102E4FEA2A2783F8A4
:102650000CA0098883F80B90D87383F810E04FEA38
:102660002229CCF307204FEA1B2E34BF4FF0320A49
:102670004FF0330A5F7383F8129083F8168083F863
:1026800007C0187283F813B083F814E083F81BA016
:102690001977C4F83461FEF7DEBA144B0393186857
:1026A000FAF73AFE00283EF463AB039B0121186859
:1026B000FAF72EFE0222002387F8742088F80030F3
:1026C000FEF756BBB0450020A8450020704300200F
:1026D000104200208E4200209C4300206BCA5F6B9A
:1026E00040420F001F85EB51E45B002008350020BD
:1026F00067666666F0820020806967FF83DE1B43A1
:10270000D34D6210984200205E2090473B68022023
:102710009847FF2014F066FC0378FF2B00F06C84D0
:1027200090F901304FEAE3795FFA89F9D8B213F0F2
:1027300039FB484613F036FB3B685E2098473B6800
:1027400003209847FF2014F04DFC0378FF2B00F086
:102750000784B0F90830D8B2C3F3072913F022FB7D
:10276000484613F01FFBD34B1B78042B75D0DFF8C2
:102770006CB3B4F82E319BF80010DFF864A393FB20
:10278000F1F201FB123292B2BAF80030A4F82E2115
:102790001201642092B200FB03134900B3FBF1F372
:1027A00042EA03295E20C3F303221FFA89F93B683A
:1027B00049EA020998473B68062098475FFA89F082
:1027C00013F0F0FA4FEA192013F0ECFABA49B4F812
:1027D0002E214B7ABAF800900132012BA4F82E2159
:1027E00000F05F864A7B09EB89031FFA83F9002A10
:1027F00040F04C843B685E2098473B683A209847FD
:10280000AE4BA3FB09234FEA531A1FFA8AFB5FFA68
:102810008BF013F0C7FA4FEA1B2013F0C3FA3B68A2
:102820005E2098473B683B209847642303FB1A933C
:102830009BB2A348053380FB0320DB17C3EBA0004A
:10284000C0B213F0AFFA002013F0ACFADFF89492A4
:1028500099F80630002B40F0DA83D8F8003099065A
:1028600040F1B381DFF8809299F800309A0700F1C7
:102870007C83DFF878824FF0000BDA463B685E20FD
:1028800098473B6801209847504613F08BFA58460A
:1028900013F088FA3B685E2098473B680920984708
:1028A000002013F07FFA002013F07CFAB8F8123001
:1028B00098F814B0B3F5967F0AD994F82C2102F059
:1028C0000F02072A04D842F20F7B9B4528BF9B4684
:1028D0003B68DFF8E4A15E2098473B6805209847F5
:1028E0009AF80830002B00F0E784ABF1200307EEE4
:1028F000903A9FED747AF8EEE77AF6EE006A67EEAA
:10290000877ABEEE007AF5EEC07AF1EE10FA58BF83
:10291000B0EE667A77EE877AFDEEE77ACDED027A51
:10292000BDF908B05FFA8BF013F03CFACBF3072047
:1029300013F038FA99F800200023900708930993C0
:1029400000F1FD8294F83031012B00F0F882BAF9E1
:102950000030DFED5D6A07EE103ABAF9023007EE9B
:10296000903AB8EEC77AF8EEE77A27EE267A67EE65
:10297000A67ABDEEC77AFDEEE77A0AA88DED0A7A4F
:10298000CDED0B7A13F030FA94F82C313A68FEF75B
:102990004FB9DFF85C919FED4D8A4FF0240B5E201C
:1029A000904758463B689847494BF9EC016A9B8A27
:1029B00007EE103AF8EEE66AB8EEC77A0BF1010BB3
:1029C000C6EE877A5FFA8BFB67EE887AFDEEE77AD0
:1029D000CDED027ABDF908A05FFA8AF013F0E2F9B2
:1029E000CAF3072013F0DEF9BBF1270F01D03A68D4
:1029F000D5E794F82C31D8F800103A68FEF711B9F1
:102A00003868FAF795FC00287FF496AC386884F8AB
:102A10004A9188F80190FAF78BFC00287FF477AC94
:102A200091E4FAF727FA2B4B1B68A0EB030A40F658
:102A3000B8339A4500F2BE81DFF8B8B09BF8043095
:102A40003A2B00F05B84002388F80030FEF790B941
:102A5000386884F84AA184F84BA184F84C9188F82E
:102A600001A0FAF765FC00287FF451AC6BE494F800
:102A7000481194F8493118484A1CFEF746B90BF141
:102A8000FF3B84F877B1FFF75FBB013F84F87671B5
:102A9000FFF7F9B8013B84F87231FFF707B8013B43
:102AA00084F86E31FEF7CABB013B84F86F31FEF744
:102AB000E5BC00BF44350020B04500201F85EB5128
:102AC00067666666E4380E3F0050C34700007A44EC
:102AD00044420020A8300020A0420020BE45002033
:102AE000A8450020284200208E420020F0820020CD
:102AF0007442002090300020C54B1B88D80515D4A7
:102B0000D90600F1B6829A0600F1BA84580600F19F
:102B1000E684190700F1E784DA0700F1248513F051
:102B2000020F0CBF4FF004084FF00C08B94BBA4A23
:102B30001B78D27803F001030AB143F0020353205B
:102B4000039314F04DFDB54A128802EB820202EBAA
:102B50008202900080B214F027FD002014F024FDC2
:102B6000AF49B04AB1F800A03868CAEBCA1A4FEAB8
:102B70004A0A82FB0A3252444FEAEA7ACAEB622AD4
:102B80005FFA8AFA5146FAF7D7FB99F80020039BBF
:102B9000386848EA03088AEA020A002189F800A096
:102BA000FAF7CAFB41463868FAF7C6FB99F80030D5
:102BB000386888EA0303DBB2194689F80030FAF76F
:102BC000BBFB94F860A1FFF743BB19077FF5DCAEB0
:102BD000954B93E803000AAB83E80300184613F013
:102BE00003F9D1E60024DFF86482A1464FF0500AD1
:102BF00002E0DBB283F3118815F804B0601C59467B
:102C0000284414F09BFB002840F0F9800BF10103ED
:102C10001C44EFF311838AF312882A6E9442E8DB96
:102C20000022DBB22A6683F31188FEF7EEB94FF07B
:102C3000000A5E20D3F8008084F82CA190473B68FE
:102C4000DFF80C9217209847504613F0ABF8774BFB
:102C5000A3FB08239B0BA9FB03125209C2EB021230
:102C6000A3EB8203D8B213F09DF83B685E2098472F
:102C70003B68182098476E4BA3FB08239B09A9FBD0
:102C800003125209C2EB0212A3EB8203D8B213F073
:102C900089F8504613F086F83A68FDF7CEBF0A9ED1
:102CA000AE424FF000014FD941F2210015F8013B2F
:102CB00081EA03235A0013F4004F80EA020192B222
:102CC00089B208BF11464B0011F4004F80EA03029D
:102CD0009BB292B208BF1A46530012F4004F80EA2A
:102CE00003019BB289B208BF19464B0011F4004F93
:102CF00080EA03029BB292B208BF1A46530012F454
:102D0000004F80EA03019BB289B208BF19464A000E
:102D100080EA020311F4004F99B293B218BF0B4638
:102D2000590013F4004F80EA010289B292B208BF41
:102D30000A46530080EA030112F4004F9BB289B2A5
:102D400008BF1946B542B1D14846F7F791FA39495B
:102D50000A9D39486D1A152DA8BF15252A4626F05B
:102D600062F9364A94F8BC321570FFF75FBB2D222A
:102D7000DA768EE4324B02991B780968C4F8381170
:102D8000013B012B3FF6A4AB10210223917013717C
:102D9000FFF79EBB12F0E8FFFDF7BFBF224A02EB30
:102DA0008302D76AFFF729BB12F0CEFF01233B70E5
:102DB000FDF770BF234AB2F8623100210133A2F857
:102DC000623188F80010FDF7D3BFDFED1F7AB0EE57
:102DD000677AFEF775BF8846894604918B46059150
:102DE0008E4606910B46FEF75CBA386884F850911F
:102DF000FAF79EFA00287FF48AAAFFF7A4BA4146A0
:102E00003A2014F0F7F940EA09095FFA89F9FDE67A
:102E10008C420020C43600200C410020A845002030
:102E2000C440002003082080B092030873B2E74535
:102E3000D34D621070200020E05D0020F55D002081
:102E400044350020601F0020000000000D5F0208D4
:102E500089888888C949CA4B0093A1F13F07C94BAB
:102E6000C94A099101F8404C0AA8C8490897F7F7E0
:102E7000D7FA089F7B1C08933C70089B2922591C99
:102E800008911A70089BEA22591C08911A70089B35
:102E9000C822591C08910AA81A7024F0B1F800F150
:102EA00001080AA94246089826F0BDF8089A02EBE4
:102EB00008030133089302F80840089B5A1C089243
:102EC0001C70089B5A1C08921C70089B5A1C089284
:102ED0001C70089B5A1C08921C70089B5A1C089274
:102EE0001C70089B5A1C08921C70089B5A1C089264
:102EF0001C70089B5A1C08921C70089B5A1C089254
:102F00001C70089B5A1C08921C70089B5A1C089243
:102F10001C70089B5A1C08921C70089B012299186F
:102F200012A808911A7050F8283DDB1B3B7012F074
:102F3000D3FF974B2C70C3F8B062FDF72FBF98E812
:102F40000C00012108A884F830110892099312F0AE
:102F50004BFF19E5C4F83C6187F80090FDF79ABE75
:102F60004FF000094846FFF7F9BBDFF83C823B68A9
:102F7000DFF838B25E2098473B6811209847B8F8D0
:102F80000E304FF4F36A0AFB03F38BFB032BDB17C2
:102F9000C3EB6B3B5FFA8BF012F004FFCBF307201F
:102FA00012F000FF3B685E20984719203B68984765
:102FB000B8F80E30774A0AFB03F382FB0301DB17F4
:102FC000C3EB611382FB0321DA17C2EB61126421A8
:102FD00001FB1233D8B212F0E5FE002012F0E2FE3F
:102FE00099F80030B8F808B09B077FF544AC5FFA59
:102FF0008BFA4FEA1B2B41E44846FFF798BBFAF7E0
:1030000087F9FDF75CBE4FF0010AFFF7E7B83B68B0
:10301000DFF89CA1DFF89CB15E2098473B68282030
:103020009847DAF800308BFB032BDB17C3EBAB0BB5
:103030005FFA8BF012F0B6FECBF3072012F0B2FE6F
:103040003B685E2098473B6804209847B9F80830F1
:10305000002B40F01982DAF8083083F310095FFA88
:1030600089F012F09FFEC9F3072012F09BFEFFF7D4
:10307000F4BB4FF0340859E5474AD278002A0CBF18
:103080004FF004084FF00508FEF724BF9BF800300E
:1030900099FBF3F9FFF7AEBB0123D8F800003B70B2
:1030A000FAF742F90746D8F80000FAF73DF97B062F
:1030B0007DF4F0AD8A2800F041828E287DF4EAADDF
:1030C0009AF80030002B7DF401AE3448344B036095
:1030D0002D2384F840310268FDF7E0BD0127FEF79B
:1030E000E7B9DFF8D4909FED2F8AB9F90230234A6F
:1030F0000B9207EE903AF8EEE77A0DF1480867EE8A
:10310000887AA2F14003FDEEE77AA2F13D0148F88A
:10311000201D02F8400C0822CDED027A5A701E22C2
:103120009A70BDF808104046F7F77CF8B9F90030FE
:1031300007EE903AF8EEE77A404667EE887AFDEEC1
:10314000E77ACDED027ABDF80810F7F76BF8B9F918
:10315000043007EE903AF8EEE77A404667EE887A58
:10316000FDEEE77ACDED027ABDF80810F7F75AF8D0
:10317000404612F0B1FEFDF7B5BE00BFF44200209C
:10318000B6470020E0BB0308E8BB0308F4BB030814
:10319000601F00201F85EB510C410020A842002039
:1031A0007043002058A08B41F082002089B5F814AC
:1031B00010420020676666663C420020CC4ACD4B38
:1031C00012680B930021A3F1400903F8401C21234E
:1031D000D10089F8023040F17481C7494FF00308EB
:1031E000C64B1B885A0500F15881D80700F1B781FA
:1031F00003F00203C24A002B1CBF4FF00308114624
:10320000DFF82CA34246504625F00DFF08EB0A03D9
:1032100012A80133AAF1020140F8203D00225B1AF6
:1032200008F80A2089F8013012F056FEFDF760BE5A
:10323000B04AB44B0B920DF14808A2F13D0048F89A
:10324000200D1988DFF8C892A2F1400300204FF04A
:103250000A0E02F8400C082283F801E040469A70FA
:10326000F6F7E0FFD9F80030A749DA1781FB03131E
:10327000C2EBA30399B24046F6F7D4FF09F0C4FDB0
:10328000D9F808900A9B4FEA1942591C0A911A7002
:103290000A9B4FEA1922591C0A911A700A9B5A1C60
:1032A0000A9283F800900A9B5A1C0A9218704046B2
:1032B00012F012FEFDF719BE5FFA8BF012F072FDEC
:1032C0004FEA1B2012F06EFDFFF734BB8D4B8F4A87
:1032D0001B88927903EB830303EB83034FEA830894
:1032E0001FFA88F8002A00F04281894B1B680FFA08
:1032F00083FA09F089FD40B2FDF7DBBE9BF80210AE
:1033000058460CF015FA00287FF49DAB7D4A814F9A
:103310007F4B1288FA61804C1A688049FA627F4AB2
:1033200003919B68B4F86211F863C7F86CA0106849
:10333000FB64F965F8F7AAFA824600287DF413AD1C
:10334000764B49461868F9F7E3FF94F864319BF827
:1033500003200492642B4FF0040287F8742040F09D
:10336000098194F86531DFF8CCB1072B08BF84F8E8
:1033700065A194F86531079307EB0319D9F8041098
:103380000691084623F03CFED9F8083005935FFA11
:1033900080F9184623F034FE5FFA80FA079B0699FD
:1033A00009EB0A0208320AEBC9008BF8072023F068
:1033B0000F0203F00F038BF80A208BF80D304A46FA
:1033C0008BF80E000BF10F0025F02DFE0BF106031C
:1033D00009F1090018445246059925F024FE9BF88E
:1033E000073003F10109D3B1013B5FFA83FC0CF113
:1033F000080CDFF844E1DC440BF10700002310F86F
:10340000012B5A409300D10883EA420301F01801CE
:1034100053404EFA01F253408445DBB2EFD1404AAB
:10342000049809F8023024F005FD94F86531002273
:10343000013384F8653184F864219BF802305BB174
:10344000039B1BF805101868F9F776FF01359BF808
:103450000230EDB2AB42F3D894F864310322013369
:1034600084F8643187F8742088F80020039BFFF704
:1034700016B99846994604939B460593FDF711BFEC
:103480004FF02408FFF752BB09F0BEFC12F08AFC93
:10349000002012F087FCFFF7E0B94FF00308214944
:1034A000AEE63B685E2098473B68392098475FFA54
:1034B00089F012F077FC4FEA192012F073FCFFF745
:1034C000C5B9194B0C4A1B68184903F48003002B3B
:1034D00016BF11464FF004084FF0030880E64FF086
:1034E0001008FFF723BB4FF02008FFF71FBB00BFFA
:1034F000B0620020F4420020CCBB03088C420020C4
:10350000DCBB0308A84500206766666628420020E9
:103510001042002020000020601F002008350020FD
:103520000E830020D0BB03086C580020C4BB0308E6
:10353000B7420020088300200007090E634B1B6878
:1035400099067DF5A7AB9AF80030002B7DF4BEAB51
:103550005F48604B03602D2384F84031BBE55E4932
:103560004FF004084CE64FF00808FFF7DFBA4FF0C1
:10357000FF33BCE697F87590DFF870B119F00F0FC4
:1035800004BF09F101095FFA89F9B9F1070F28BFF2
:103590004FF001094FEA091A07EB0A035FFA8AFCA8
:1035A000187C4E4B1A180023117A8BF80A300BF155
:1035B0000D0307EB0A024CEA000001291870D268DB
:1035C00003F1010E0CD90239C9B2881C18447346A4
:1035D00003F8012B83424FEA1222F9D101318E44C4
:1035E000BA4422F0600309F101099AF811205FFA48
:1035F00089F91343B9F1080F8EF800300EF1010379
:103600004FD04FEA091A07EB0A01354A087C3349C3
:1036100001449A1A097A02EB010E0CF1100CBEF16A
:10362000130F5FFA8CFCC4DDD2B2931DDBB243F002
:1036300040018BF8071003F1010CDFF8B4E0CBB1C7
:1036400005325FFA82FA0AF1080ADA440EF1010043
:10365000002310F8011B59408B0083EA4103CA087C
:103660004B40204902F0180241FA02F253408245D1
:10367000DBB2EED104980CF80E3087F8759024F088
:10368000D9FBDAE69846994604939B4605939E46F5
:10369000FDF707BE144B8046B3F900A06420FDF788
:1036A00008BD0F4A9A1ABFE79846FDF7FABD98463B
:1036B0009946FDF7F6BD984699460493FDF7F1BD8E
:1036C0009846994604939B46FDF7EBBD384200208F
:1036D000A84200209C430020D4BB0308B0920308FA
:1036E000158300200007090E1042002008830020E7
:1036F0000E8300202DE9F04F2DED0C8BDFF8A09309
:1037000095B0D9F80420069048469047002875D017
:10371000B9F8A850002189F85110002D41F05084CB
:10372000D9F84820B9F93C70B9F93840D9F8206087
:10373000B9F93A00D9F82450DFF868B3BB1A83EA24
:10374000E371A1EBE371A41BB1F5804FC9F82C40E4
:10375000D9F8284099F85210DCBFC9F848703A46A9
:10376000401B121BC9F83000B248C9F8342011F0D0
:103770001BFCDBF80020940041F11485D9ED0C5AB4
:10378000DFF824A3D9ED0B7AAB499AED406ADAED64
:10379000416A9AED427ADAF80C210968A74B049342
:1037A000B8EEE58AD9ED0D5AF8EEE77AF8EEE58A3B
:1037B000013277EE867A38EE268A78EE878A8A4258
:1037C000CAED407A8AED418ACAED428ACAF80C21D4
:1037D00002F02E821F78142F03F0C9810023DAF83B
:1037E00014410593062C01F27D81DFE814F00A15DF
:1037F00048164614DF15EB085916A6148F4BDFF850
:10380000A8A21C780493072C01F0BF819AF82031FC
:10381000089353B1013B8AF82031012C01F09F84B9
:1038200015B0BDEC0C8BBDE8F08F854A5279002AAB
:1038300001F01F82834A1278013AD2B2072C8AF82B
:10384000202102F0C38200230A937F4BDAF82C2157
:10385000D3F800B07D4B0793069B9FED7D6ADAEDB0
:103860004A9A7C497C4FD1ED006ACAF82C319A1AE9
:1038700007EE902AF8EE677AB7EE007AC6EE278A4E
:1038800007F11C0300240993DFF82082734B744E68
:103890000593254677EE69BA9AED49CA9FED719A6C
:1038A000DFED71AA9FED71BA9FED71AA6BEEA6BA1A
:1038B000F4EEC7BAF1EE10FA88BFF0EE47BA6D4BDE
:1038C00097ED008A2344D3ED007AF5EE407AF1EECD
:1038D00010FA17D0684B234493ED007A78EE476ACC
:1038E000B0EEE66AF4EEC67AF1EE10FA08D5F5EE1F
:1038F000C06AF1EE10FACCBF37EE878A37EE678ADE
:1039000083ED008A5D4B1A8891073FD0022D3DD090
:103910005B4B9BF82E1033F9153007EE103A099BDC
:1039200007EE901A2344F8EEE76AB8EEC77AD3EDB3
:10393000007A4B42A6EEA77A680007EE903AF8EEBE
:10394000E77AB4EEE77AF1EE10FA0AD407EE901AAD
:10395000F8EE677AF4EEC77AF1EE10FA88BFF0EE6F
:10396000477A484B48490344085EB3F90C30C01A03
:1039700007EE100AB8EEC77AD307E7EE497A41F1AD
:103980000E81424B93ED008A27EE888A079B9AF8B6
:103990006421234493ED01DA78EE4DCA002A00F049
:1039A000C4803B4BDAF8682106991B688A1A9A4250
:1039B00040F3BB80022D04F04185364B1B6898070D
:1039C00076D4354B86ED00BA1B689342C0F2AA80CC
:1039D000F7EE007AF4EEE79AF1EE10FA40F1A580E6
:1039E00007992E4BD1ED017A93ED007AF0EEE77A4C
:1039F000F4EEC77AF1EE10FA40F19780D1ED027A39
:103A0000F0EEE77AB4EEE77AF1EE10FA40F38D804B
:103A1000D1ED037AF0EEE77AB4EEE77AF1EE10FA40
:103A200040F383801B4B1B6899077BD51649154BC8
:103A30005FE000BF985000207C3D0020CC44002077
:103A400048580020F4620020904200205C5800207A
:103A5000002474492C3C0020542300209040002076
:103A60009C400020CDCCCC3DAE47813F0000000003
:103A70000000C842203C0020602300208C4200202F
:103A80006C230020006300203C420020083C002002
:103A9000343C002038420020303C00203C3C0020D8
:103AA0006C5000206C58002024220020A8400020E8
:103AB000D44BD549DFF8BCE331F915C09EED008A3F
:103AC000DFF8B4E386ED00BA03EB450028EE098A7F
:103AD000B0F90C00A0EB0C0007EE900AF8EEE77AC4
:103AE000DEF8000027EE888A824278EE4DCA7FF722
:103AF0006FAFB3F90C20B1F900E0C448AEEB020E91
:103B000000688EEAEE72A2EBEE7282420DDAB3F931
:103B10000E30B1F90220D21A82EAE273A3EBE2730B
:103B2000984202DD00238AF86431B94B234493EDB7
:103B3000000A059B2CEE000A022D20EE2C0AA3ECB5
:103B4000010A059304F03784B24BD6ED006A93ED79
:103B5000007AB14BD3ED007AB04B93ED006AB04BD5
:103B600067EE277A234427EEAB7AD3ED007A67EE2F
:103B7000277AF0EE665AECEEA75AB1EE467AB4EE2A
:103B8000E57AF1EE10FA08DCB4EEE56AF1EE10FA2F
:103B90008CBFB0EE657AB0EE467A9AED4A6AF7EEDF
:103BA000007AB4EEE76AF1EE10FAACBF012300230D
:103BB00043B1F0EEE66AF0EEC77AF4EEE67AF1EEA3
:103BC00010FA01D586ED007A022D04F09E83954A05
:103BD000954B52F825001B68B0EE4D0A9847934A62
:103BE000934B52F825001B6898479BF8373023B158
:103BF000904B1B88002B01F0D580B0EE4B8A8E4B8A
:103C000038EE400A234493ED008A83ED000A9BF8C6
:103C1000483030EE480A20EE280A3BB3874B1B7829
:103C2000DA0740F1C586F7EE007AF4EEE79AF1EE96
:103C300010FA9AF86431C1F27985002B01F068819D
:103C4000DAF86831069AD31A7D4A12689A420DDD75
:103C50007C4BD3ED007AF0EEECCAF4EEE7CAF1EE5D
:103C600010FA42F1D38500238AF86431764B9AF832
:103C700074212344D3ED007A6CEE277A27EE800A74
:103C800088ED000A32B9059B86ED00BA03ED01BA52
:103C900088ED00BA0135032D07F1040708F1040887
:103CA00006F1040604F104047FF409AE049B1A78BB
:103CB000072A01F05185012A02F07680002307933C
:103CC0009AF87C21002A41F05782DFF8B0B15F4BAF
:103CD000DBF800201968D30491F82C0001F18E80E4
:103CE000DFF89C815A4AB8F81A30D2ED005A594A86
:103CF000594CD2ED004AD4ED036A584ACAED635AD2
:103D000007EE103A564B92ED005AD3ED007AD3ED00
:103D1000013A93ED026ACAED615AB8EEC77A34EE01
:103D2000E54A012236EEC77A8AED604ACAED644A56
:103D30008AF89421C7EE055A0A8D534206EE903A4E
:103D4000484BDFED494A93ED005A484B93ED004A4A
:103D5000B7EE007AF4EEC75A35EE045AF1EE10FAD7
:103D600088BFF0EE475A35EE275AF8EEE66AF4EED1
:103D7000E45AF1EE10FA07EE902AB4EEE65AB8BF14
:103D8000F0EE645AF1EE10FACAED675AB8EE677AAF
:103D900001F15683B4EEC75AF1EE10FA88BFB0EEC7
:103DA000475A304BDFED324AD3ED017A2F4B93ED7A
:103DB000014A77EE847A25EE245A77EEA37AF4EE60
:103DC000E76AF1EE10FA08DCB4EEE77AF1EE10FAE9
:103DD0008CBFF0EE676AF0EE476A224B4A8DD3ED56
:103DE000027A9FED237A534204EE103A76EE277A58
:103DF000B8EEC44A66EE876AF4EEC47AF1EE10FAC1
:103E00004BD43FE0006300203C420020383C0020BF
:103E1000DC3B00209800002080370020503C002030
:103E2000E83B00208837002084370020DC37002062
:103E3000D83700208C42002090230020C436002078
:103E4000343C0020403C0020F43B00209042002005
:103E500050610020CC620020C0450020E83C0020DA
:103E60009C4000209040002000000000A84000205E
:103E70006F12833A083C0020303C00206C58002030
:103E8000C469002007EE102AB8EE474AB4EEE74AAC
:103E9000F1EE10FA88BFB0EE674AEB4ADFEDEB7A3D
:103EA000527824EE274A0AB9B1EE444A002841F07C
:103EB0008386B7EE003AE64D2A78002A02F0E186C2
:103EC000E4499FEDE56AD1ED024A91ED017AD1ED29
:103ED000037A66EEA44AE5EE074AE4EE274A63EE6B
:103EE000244AF4EEC64AF1EE10FAB4BFF0EE463AB8
:103EF000F0EE643A98BFB0EE646A012ACDED0C4A48
:103F000002F00E87D1ED067AD1ED052A91ED077A00
:103F100066EEA77AE5EE227AE4EE077A23EE277AB8
:103F2000B4EEC67AF1EE10FAB4EEE37A8CBFF0EE9E
:103F3000467AF0EE477AF1EE10FA98BFB0EE676A73
:103F4000B4BFF0EE637AF0EE477A022A8DED0D7A77
:103F500000F0DE8091ED0A7AD1ED092AD1ED0B3A1D
:103F600026EE877AA5EE227AA4EE237A23EE077A4C
:103F7000B4EEC67AF1EE10FAB4EEE77A8CBFF0EE4A
:103F8000463AF0EE473AF1EE10FA98BFB0EE636AA7
:103F9000A8BFF0EE477A032A8DED0E7A00F0B880C4
:103FA00091ED0E7AD1ED0D2AD1ED0F3A26EE877AFA
:103FB000A5EE227AA4EE237A23EE077AB4EEC67A2F
:103FC000F1EE10FAB4EEE77A8CBFF0EE463AF0EE7E
:103FD000473AF1EE10FA98BFB0EE636AA8BFF0EE70
:103FE000477A042A8DED0F7A00F09280D1ED123AD3
:103FF000D1ED112A91ED137A66EEA33AE5EE223A5D
:10400000E4EE073A63EE233AF4EEC63AF1EE10FA24
:10401000F4EEE73A8CBFB0EE467AB0EE637AF1EE9A
:1040200010FA98BFB0EE476AA8BFF0EE637A052A8F
:10403000CDED103A6CD0D1ED163AD1ED152A91EDB7
:10404000177A66EEA33AE5EE223AE4EE073A63EE1B
:10405000233AF4EEC63AF1EE10FAF4EEE73A8CBFEA
:10406000B0EE467AB0EE637AF1EE10FA98BFB0EE99
:10407000476AA8BFF0EE637A062ACDED113A47D021
:10408000D1ED1A3AD1ED192A91ED1B7A66EEA33AD9
:10409000E5EE223AE4EE073A63EE233AF4EEC63A4E
:1040A000F1EE10FAF4EEE73A8CBFB0EE467AB0EEDD
:1040B000637AF1EE10FA98BFB0EE476AA8BFF0EE4F
:1040C000637A072ACDED123A22D091ED1E7AD1ED16
:1040D0001D2AD1ED1F3A26EE877AA5EE227AA3EEAD
:1040E000847A27EE037AB4EEC67AF1EE10FAB4EED3
:1040F000E77A8CBFF0EE466AF0EE476AF1EE10FA0E
:104100008DED137A98BFB0EE666AA8BFF0EE477ADD
:1041100077EEC67AF7EE006AF4EEE67AF1EE10FA80
:10412000CAED4A7A43F3248786EEA77A022ADDEDA8
:104130000D7A67EE244A67EE877ACDED0C4ACDED15
:104140000D7A2DD0DDED0E7A67EE877A032ACDED5C
:104150000E7A25D0DDED0F7A67EE877A042ACDED51
:104160000F7A1DD0DDED107A67EE877A052ACDED46
:10417000107A15D0DDED117A67EE877A062ACDED3B
:10418000117A0DD0DDED127A67EE877A072ACDED30
:10419000127A05D0DDED137A27EE877A8DED137A4A
:1041A0002E49096811F08053059301F07682F6EEEE
:1041B000005ACAED675A002A02F05D859AF99431D7
:1041C0009AED646A2649274E9AED635A264FB6F94E
:1041D0000660C878DBF80010099607EE103ABDEECD
:1041E000C66A224BB8F81A601C78214BD7ED004AFA
:1041F0000A9616EE10EABDEEC56A01F0100601F44B
:10420000805701F480010B911B78DAED606ADAEDDA
:10421000617AB8EEC77A04F0010C16EE101A002885
:1042200040F0EC870B4C9DED0C5A94ED006A002E8B
:1042300041F0978325EE866A0E48A5EE076AB0EE38
:10424000675AA6EE265A17E0004100206F12833A03
:1042500014860020583C002000000000B0620020BE
:104260000C4100203C490020543C0020C436002072
:10427000D04B0020D8400020BDEEC56A16EE107A63
:1042800016EE106A7745A8BF7646B942C8BF0E46FB
:1042900006EE106AB8EEC66A012A80ED006A00F0E8
:1042A000DC8094ED046A9DED0D5A25EE866AA5EE3C
:1042B000076AB0EE675AA6EE265ABDEEC56A16EE3C
:1042C000107A16EE106A7745A8BF7646B942C8BF85
:1042D0000E4606EE106AB8EEC66A022A80ED016A42
:1042E00000F0BB8094ED086A9DED0E5A25EE866ABB
:1042F000A5EE076AB0EE675AA6EE265ABDEEC56A6D
:1043000016EE107A16EE106A7745A8BF7646B942C7
:10431000C8BF0E4606EE106AB8EEC66A032A80EDE4
:10432000026A00F09A8094ED0C6A9DED0F5A25EE1A
:10433000866AA5EE076AB0EE675AA6EE265ABDEE6B
:10434000C56A16EE107A16EE106A7745A8BF764653
:10435000B942C8BF0E4606EE106AB8EEC66A042A15
:1043600080ED036A79D094ED106A9DED105A25EE28
:10437000866AA5EE076AB0EE675AA6EE265ABDEE2B
:10438000C56A16EE107A16EE106A7745A8BF764613
:10439000B942C8BF0E4606EE106AB8EEC66A052AD4
:1043A00080ED046A59D094ED146A9DED115A25EE02
:1043B000866AA5EE076AB0EE675AA6EE265ABDEEEB
:1043C000C56A16EE107A16EE106A7745A8BF7646D3
:1043D000B942C8BF0E4606EE106AB8EEC66A062A93
:1043E00080ED056A39D094ED186A9DED125A25EEDC
:1043F000866AA5EE076AB0EE675AA6EE265ABDEEAB
:10440000C56A16EE107A16EE106A7745A8BF764692
:10441000B942C8BF0E4606EE106AB8EEC66A072A51
:1044200080ED066A19D094ED1C6A9DED135A65EE75
:10443000865AE7EE055AE6EEA57AFDEEE77A17EE24
:10444000904AA645A8BFA646A142D8BF714607EE2E
:10445000901AF8EEE77AC0ED077ABCF1000F00F091
:10446000DA87CF4A1268002A40F0E287CD4A1278F4
:1044700082B1287858B1CC4ECC4F0024E0B23B68D2
:10448000B6EC010A9847287801348442F6DBC84A22
:1044900012689047049B1A78072A01F04C81002388
:1044A0000593DBF80020540501F19980C14B1D688C
:1044B000280701F13980C04B1B78BBB1BF4AB8F85F
:1044C0001A30B2F906209A4210DCBD4B1B78012B42
:1044D00001F08184192B01F07E840E2B06D0082B6D
:1044E00004D0B84C0023A360CAF838319AF8A6412A
:1044F00024B1B54B1B889B0741F02E849AF8AC6120
:10450000002E40F0A18798F81E70002F00F01E8644
:10451000022F01F08683032F41F07F8398F820302B
:10452000C3EB431203EB8202D20092B298F81F3021
:104530000233DBB2002E00F03A86002A00F0378604
:10454000A2490F68B2FBF7F217B2AAF8DC71002B90
:1045500003F0E88107EE907AF8EEE77AF7EE006A6A
:1045600086EEA77A974C012BDAED7C6AD4ED007ABF
:1045700077EEE67A67EE877ACAED787A21D0D4EDC5
:10458000017ADAED7D6A77EEE67A022B67EE877ABA
:10459000CAED797A15D0D4ED027ADAED7E6A77EE3B
:1045A000E67A032B67EE877ACAED7A7A09D0D4EDE2
:1045B000037ADAED7F6A77EEE67A67EE877ACAEDFC
:1045C0007B7A049A1278092A03F0F982002F40F3CB
:1045D000C3859BB39AED7C7ADAED787A77EE877AA9
:1045E000012BCAED7C7AC4ED007A21D09AED7D7A58
:1045F000DAED797A77EE877A022BCAED7D7AC4ED0F
:10460000017A15D09AED7E7ADAED7A7A77EE877AAA
:10461000032BCAED7E7AC4ED027A09D0DAED7F7AF7
:104620009AED7B7A77EE877ACAED7F7AC4ED037ACA
:10463000013B022BB8BF0223DBB20893002E089D7A
:1046400018BF0225624BDFED676A1A68049B9178F8
:104650001878137807EE903AF8EEE77AB0EE007A21
:1046600067EEA67AF4EEC77AF1EE10FA40F3E4862C
:10467000DFED596A37EEC77AB0EE676AA7EE266AB1
:10468000F0EE466A94ED007A9FED546A27EE066AD2
:10469000F0EEC65A8AED536ACAED565A99B107EE42
:1046A000101AB8EEC75A9FED4F7A66EE064A25EE0D
:1046B000075AB7EE007A37EE457A64EEA54AA4EEC3
:1046C000857A26EE076A9FED467A537926EE877A39
:1046D00027EE067ACBB1DFED436A9FED436A65EEC4
:1046E000A65A06EE903AF8EEE66A65EEA65AF4EEA1
:1046F000C65AF1EE10FA01F34982B7EE006A76EE7F
:10470000655AC6EE256A27EE267A0C289FED378A71
:10471000DFED376A00F0C887B4EEC87AF1EE10FA20
:1047200098BFB0EE478AB4EEE68AF1EE10FAB8BF51
:10473000B0EE668A8AED4C8A002D00F00981B0EE59
:10474000007AF4EEC77AF1EE10FA05DD37EEC77A9B
:10475000DFED216AE7EE267A94ED017ADFED1F6A3C
:1047600027EE267AF0EEC75A8AED547ACAED575AE8
:1047700000293FD006EE901A9FED1A6AF8EEE66A1D
:1047800027EE075A66EE866AB7EE006A36EE666A6C
:1047900025EE255AA5EE266A27EE067A2AE000BF06
:1047A0007C370020F84E0020D8400020C44B002069
:1047B000CC4B002038420020380B00203C49002020
:1047C00000410020C04500208C420020FC40002019
:1047D000944200200000C842D7A368416F12033BF7
:1047E000000048430AD7233CA4707D3F00C0F94431
:1047F00000C0F9C45FED066A937967EEA67A67EEAA
:10480000877AABB107EE103AB8EEC77A1FED0B6AA4
:104810005FED0B6A27EE257A27EE067AB4EEE67A8C
:10482000F1EE10FA41F3A4815FED166A67EEA67A05
:104830000C2800F054875FED136A1FED137AF4EE35
:10484000E67AF1EE10FA88BFF0EE667AF4EEC77AF7
:10485000F1EE10FAB8BFF0EE477A012DCAED4D7AAD
:1048600076DD53785FED216A07EE903AF8EEE77A4D
:10487000B0EE007A67EEA67A537AF4EEC77AF1EEDC
:1048800010FA05DD37EEC77A5FED2D6AE7EE267A7E
:1048900094ED027A5FED2F6A27EE267AF0EEC75A82
:1048A0008AED557ACAED585A9BB106EE903A1FED43
:1048B000336AF8EEE66A27EE075A66EE866AB7EEC6
:1048C000006A36EE666A25EE255AA5EE266A27EEC0
:1048D000067A5FED3D6AD37967EEA67A67EE877A4E
:1048E000FBB107EE103AB8EEC77A1FED426A5FEDF2
:1048F000426A27EE257A27EE067AB4EEE67AF1EEE2
:1049000010FA01F33181B5EEC07AF1EE10FA02F13E
:10491000BD83B7EE006A36EE477AC6EE076A67EEE9
:10492000A67A0C2800F0FA865FED506A1FED507AE7
:10493000F4EEE67AF1EE10FA88BFF0EE667AF4EE65
:10494000C77AF1EE10FAB8BFF0EE477ACAED4E7AA8
:10495000092800F0958698F82140002C40F04A86FE
:10496000C54B1D6800238AF8AC31AC0609D5C34B92
:104970001B8803F0300323B1C14B1B78D80702F129
:104980000581C04B1B7823B9BF4CA378002B41F0A5
:10499000F981049B1C78072C7EF43FAFF8F76AFA84
:1049A000049ABA4B1478059A801AD880FEF735BF5E
:1049B0009AF86431002B3FF459A900238AF8643136
:1049C000FFF754B9B24A1178DAF81861B14B9FED8C
:1049D000B27AF5005A1982ED007A002978D0AF48F2
:1049E000B0EE476AF0EE476A0022F0EC017A01323D
:1049F00067EEA77A05EE902AB4EEE77AF1EE10FAA8
:104A0000F8EEE55AB8BFB0EE677A8A4276EEA76A4A
:104A1000A7EEA56AE9D1F5EEC06A5A19F1EE10FACF
:104A200082ED007A54DDC6EE265A9D4A9D490988DA
:104A3000F7EE007A75EEE75AD2ED007A65EEA77AC6
:104A4000FDEEE77A17EE902A812A42F3A3828A428A
:104A5000A8BF0A4607EE902AF8EEE77A924AA8190C
:104A600002EB800292ED057AD2ED003A92ED066AF1
:104A700092ED014AD2ED046AD2ED034A92ED025A58
:104A8000A3EEA77AA4EE276A66EEC76AA7EE646A69
:104A9000BDEEC77AE5EE276A17EE100A812882ED8F
:104AA000056AC2ED066A42F372828142A8BF0146DE
:104AB00007EE901AF8EEE77AFCEEE77ACDED077A8A
:104AC000BDF81C2059198A8016B9132F03F03E82B5
:104AD000152F41F025831D446C4BAA8823F816201E
:104AE000DAF81441714A013482FB04321119E217D9
:104AF000C2EBA102C2EBC202A41ACAF814416C486C
:104B0000DAF81C21069B6B4C01682478CAF81C312A
:104B10009A1A11440160002C40F0E08007EE902AC0
:104B2000654DDFF8B481654EB8EEE78A05F244744E
:104B300005F5F667F5EC017A99ED070AD9F86C37B7
:104B4000F8EEE77A204627EE800A9847A4F1E000C5
:104B5000D9F88C369847A4F17000D9F8FC369847FC
:104B6000D5F85006D9F8AC309847D6ED007AA8ECC5
:104B7000010AE0EE087A2434A742E6EC017AD9D1A2
:104B8000049B1C78072C7EF441AEF8F773F9049A65
:104B90003E4B1478069A801A1880FEF737BEB1F99A
:104BA00000209AED567AB1F90200DAED576A4449CD
:104BB00082EAE273A3EBE273F4EEC76A80EAE07282
:104BC000F1EE10FAA2EBE072B4BFB0EE476AB0EEBD
:104BD000666A9342B8BF134607EE103A0B78B8EEF8
:104BE000C77A27EE097A002B40F06381354BD3ED6D
:104BF000005AF4EEEA5AF1EE10FA41F1A880B7EE4D
:104C0000005A75EE654ADFED306A9FED305A304B41
:104C100036EEC77A24EE855AD3ED006AE7EE055AE0
:104C200065EEA65AF5EEC05AF1EE10FA40F2318563
:104C3000CAEE256AB7EE007AF0EE475AE6EE665AFB
:104C4000F0EE656AF4EEC76AF1EE10FA88BFF0EE96
:104C5000476AF5EEC06AF1EE10FAB8BFF0EE4B6AA3
:104C60001C4B93ED007A67EE877AA7EEA68AFEF7D3
:104C70008DBE0122FEF7E2BD384200208C420020AA
:104C80008E420020164900200E490020D04400200A
:104C9000823D0020784000200000000024220020F7
:104CA000843D0020803D0020A03F002093244992B5
:104CB000C0680020743D002098500020C468002087
:104CC000143C00201C3C002000003443610BB63B28
:104CD000103C00200C3C00206058002007EE902A79
:104CE000A14BA24CA249A34FCDF81CA0F8EEE78A35
:104CF000059304F2D465984600268A46049BD9EDB4
:104D0000077A1B78172B6DD094ED007AB8EEC78A1E
:104D1000082B28EE278A07D1B0EE480A089323F023
:104D2000E1F9089BA8F80000DBF8002090000BD503
:104D3000002E03F0AB83B0EE480AD9F86C3705F1CA
:104D400070009847B0EE408AB0EE480AD9F88C3629
:104D5000A5F170009847D9F8FC3628469847049B7F
:104D60001B78032BB0EE408A37D0D4F85406D9F81C
:104D7000AC30B0EE480A9847D7ED007AAAEC010AA9
:104D8000E0EE287A0136032E05F1240508F1020829
:104D900004F10404E7EC017AB0D1049BDDF81CA017
:104DA0001C78EFE6744B754A234493ED007AD2EDFC
:104DB000007A734B67EE277AF7EE006AF4EEE67A34
:104DC000F1EE10FA93ED007A88BFF0EE667A67EEA6
:104DD000877A27EE888AFEF712BF23F083F9A8F8B6
:104DE0000000C2E794ED007A09EB4602B8EEC78AEC
:104DF000128FA8F8002028EE278A95E7614BDFF88C
:104E0000BC811A78604CD7075CBFB8F81820AAF8A4
:104E100088215E4AD4ED037A128807EE102AB8EE94
:104E2000C77AF4EEC77AF1EE10FA41F25D86584C7B
:104E3000238807EE103AB8EEC77AF4EEC77AF1EE9F
:104E400010FAC0F2D487534A534C92ED006AD4ED65
:104E5000006A9AF99421CAED636A76EE665A012ACD
:104E6000CAED616ACAED605A8AED646A01F02E8566
:104E7000069BCAF89831002437EEC77AFCEEE77A31
:104E8000464D8AED677A17EE902AAAF8882101220A
:104E900095ED005A8AF89421414A944241F2548691
:104EA000404BD3ED007AD3ED013A93ED026AFEF761
:104EB00041BF3D4B93ED005AB5EEC05AF1EE10FAEA
:104EC00040F3E783394BD3ED006AF5EEC06AF1EEAB
:104ED00010FA40F3DE8336EEC77A66EE4A5A87EE62
:104EE000266AC5EE856AB7EE007AB4EEC76AF1EEBF
:104EF00010FA88BFB0EE476AB5EEC06AF1EE10FA5C
:104F000076EE876AB8BFB0EE4B6A66EE266A99E61F
:104F1000274AD2ED007AB0EEC07AB4EEE77AF1EE2D
:104F200010FA7EF7A3AE234AD2ED007AB0EEEC7A07
:104F3000B4EEE77AF1EE10FA7EF798AE1E4AD7ED9E
:104F4000007A92ED007AF0EEE77AF4EEC77AF1EEAD
:104F500010FA7EF58BAE01220699CAF868118AF81C
:104F60006421FEF771BE00BFD0440020985000209D
:104F700060580020C46800207C230020043C0020EE
:104F8000003C0020C4360020C0450020EC3C00203E
:104F9000EE3C0020CC620020D83C0020F43C0020F5
:104FA0008FD003009C400020103C0020183C0020C3
:104FB000443C0020403C0020483C0020C4690020C4
:104FC000804C814B81481A68477807932646804B6E
:104FD000B6F9060005944FF47A76B6FBF2F2C2EB0E
:104FE000421602EB8602D600B6B2B54204931C7894
:104FF00001F0D487D9F87C30B9F93810D9F860209D
:1050000003F1010E07EE901A0A44BEF1010FC9F830
:105010007CE0C9F86020F8EEE77A01F0CC87D9EDA2
:105020001B5AD9ED1D6A07EE10EA37EEE56AB8EEB5
:10503000C75A012D86EE057A37EE257A77EEC77AC4
:1050400089ED1C7AE7EE866A89ED1B7AF0EE667AC6
:10505000C9ED1E6AC9ED1D6A02F02784D9F89030A7
:10506000B9F93A10D9F8642003F1010E07EE901A4D
:105070000A44BEF1010FC9F890E0C9F86420F8EEC7
:10508000E77A01F0B387D9ED205AD9ED226A07EE0D
:1050900010EA37EEE56AB8EEC75A012D86EE057ABA
:1050A00037EE257A77EEC77A89ED217AE7EE866AC0
:1050B00089ED207AF0EE667AC9ED236AC9ED226A9D
:1050C00002F0CA83D9F8A430B9F93C10D9F86820A5
:1050D00003F1010E07EE901A0A44BEF1010FC9F860
:1050E000A4E0C9F86820F8EEE77A01F09A87D9EDD4
:1050F000255AD9ED276A07EE10EA37EEE56AB8EED1
:10510000C75A012D86EE057A37EE257A77EEC77AF3
:1051100089ED267AE6EE276A89ED257AF0EE667A41
:10512000C9ED286AC9ED276A02F0E883059BD8809B
:10513000049B013D1C78A9F8A8500799DFF8B0A09E
:1051400000224A608A60CA60FEF75DBBAAF8DC7183
:10515000002E3FF40AAC1F4C0225FFF773BA1E4B1A
:105160001E4A19681288174BC96919805A8015B0F0
:10517000BDEC0C8BBDE8F08F194B1A4D1A7812F06C
:10518000010F2A7840F01C83002A00F0038592006A
:1051900015491648DFF85CB0DFF85C8023F043FF68
:1051A000FFF75FB90A4B0493DFF844A0A7E4BAF80D
:1051B000DC71013F3FB2002FAAF8DC71C8DD054C5D
:1051C000FFF707BAD04400205C5800204858002060
:1051D000CC440020C0450020744400204835002005
:1051E000C4360020148600204C350020D840002012
:1051F000242200206C580020C4690020002E01F0F9
:105200009E81BCF1000F42F09583BD4C002B42F013
:10521000D58194ED006A9DED0C5ABA4825EE866A58
:10522000FDEEE44AA5EE076AB0EE675AA6EE265AEE
:1052300014EE901ABDEEC56A16EE107A16EE106ADC
:105240007745A8BF7646B942C8BF0E4606EE106A3B
:10525000B8EEC66A012A80ED006A00F0DF8094EDA6
:10526000046A9DED0D5A25EE866AA5EE076AB0EE3A
:10527000675AA6EE265ABDEEC56A16EE107A16EEED
:10528000106A7745A8BF76468F42B8BF0E4606EE35
:10529000106AB8EEC66A022A80ED016A00F0BE808C
:1052A00094ED086A9DED0E5A25EE866AA5EE076A12
:1052B000B0EE675AA6EE265ABDEEC56A16EE107A13
:1052C00016EE106A7745A8BF76468F42B8BF0E46E5
:1052D00006EE106AB8EEC66A032A80ED026A00F094
:1052E0009D8094ED0C6A9DED0F5A25EE866AA5EE21
:1052F000076AB0EE675AA6EE265ABDEEC56A16EEEC
:10530000107A16EE106A7745A8BF76468F42B8BF6E
:105310000E4606EE106AB8EEC66A042A80ED036AED
:105320007CD094ED106A9DED105A25EE866AA5EEAC
:10533000076AB0EE675AA6EE265ABDEEC56A16EEAB
:10534000107A16EE106A7745A8BF76468F42B8BF2E
:105350000E4606EE106AB8EEC66A052A80ED046AAB
:105360005CD094ED146A9DED115A25EE866AA5EE87
:10537000076AB0EE675AA6EE265ABDEEC56A16EE6B
:10538000107A16EE106A7745A8BF76468F42B8BFEE
:105390000E4606EE106AB8EEC66A062A80ED056A69
:1053A0003CD094ED186A9DED125A25EE866AA5EE62
:1053B000076AB0EE675AA6EE265ABDEEC56A16EE2B
:1053C000107A16EE106A7745A8BF76468F42B8BFAE
:1053D0000E4606EE106AB8EEC66A072A80ED066A27
:1053E0001CD094ED1C6A9DED135A65EE865AE7EECB
:1053F000055AE6EEA57AFDEEE77A17EE904AA64545
:10540000A8BFA646A142D8BF714607EE901AF8EE93
:10541000E77AC0ED077A002A3FF423A892003A49C0
:10542000384823F000FE394A1268002A3FF41EA8CB
:105430000CF0F6FEFFF71AB8F0EE676AFFF722B934
:10544000B0EE665AFEF7ADBC314A324BD2F8EC20D2
:105450001B6844F620618A42A8BF0A46B2F57A7FEB
:10546000B8BF4FF47A7292B213F0100FAAF8AE21BF
:10547000DBF8003000F0B684DB0441F1E086264B17
:105480001F68788E4008254C2549DAF8B031D4EDF4
:10549000037AA1FB02129109642292FBF1F2142A11
:1054A000BDEEE77A0AEB4304A8BF142201339A4207
:1054B000CAF8B03117EE10EADCBF0023CAF8B031E9
:1054C0000AEB4303A4F8B4E1B3F9B43107EE103AA0
:1054D000B8EEC77A77EEC77AFDEEE77ACDED077AB8
:1054E000BDF91C2082EAE273A3EBE273834202F36C
:1054F0001E800C4A4FF07E531360FFF704B800BFC4
:10550000583C0020D84000204C3500207C3700203B
:1055100024010020B062002090420020C0450020FD
:10552000D34D621098000020954CD4ED027AB2EE73
:105530000E7AF0EEE76AF4EEC76AF1EE10FA41D5A2
:10554000904B1B8859073DD58F4B904AB3F90430D7
:105550008F4982FB03020988DB17C3EBA2035B1AA6
:105560009BB219B211F1B30FBCBF03F5B47319B2FA
:10557000B329C4BFA1F5B47319B2864B864A1B790F
:105580001278002B4FF6FF7318BF012312077EF528
:1055900092AF824A126811FB03F3117E804A9BB2DC
:1055A00011FB03F382FB03121A44DB17C3EB221334
:1055B00007EE103AB8EEC77A77EEC77AC4ED027AF2
:1055C000FEF779BF704B714AB3F90430704982FB22
:1055D0000302DB17C3EBA2030B80FEF76CBFD9F805
:1055E0000830002B3EF462AF6E49A1F14C009847A1
:1055F000FEF75CBF1E216C48F5F776FA00283FF4F1
:10560000AFA9604B1B885D063FF5AAA99AF8003246
:10561000A34242F0F082654BDAED817AD3ED016A64
:105620009AED4E5ADFED625A9FED626A27EEC57A17
:1056300068EE277AA8EE267AE5EE267AB4EEE57AC9
:10564000F1EE10FA88BFB0EE657AB4EEC67AF1EEEC
:1056500010FAF4EEE57AB8BFB0EE467AF1EE10FA41
:1056600088BFF0EE657AF4EEC67AF1EE10FAB8BFB4
:10567000F0EE467A8AED4C7ACAED4E7AFFF770B9B1
:10568000FDEEC87A4C4A17EE903A9780D380FFF728
:1056900062B9DFED4A6AFFF7E3BADBF800104E02A9
:1056A0003EF585ADFEF787BDB4EEC87AF1EE10FA8F
:1056B00098BFB0EE478ABDEEC77AB4EEE68A3E4E9A
:1056C000F1EE10FA17EE103AB8BFB0EE668A8AED26
:1056D0004C8A3380002D7FF432A8FFF73CB99FED50
:1056E000347ADFED346A3449F4EEC77AF1EE10FA19
:1056F00098BFB0EE677AFDEEE77AB4EEE67AF1EEA7
:1057000010FA17EE903AB8BFB0EE667A012D8AED26
:105710004D7A4B803FF7A5A8FFF71DB9BDEEE77A9C
:10572000254B17EE102A9A80FFF7FEB8002B3EF4A7
:105730009DAAFEF785BAF7F79DFB049B1E491A78D0
:10574000079B072AA0EB030088807EF4A8AEF7F73A
:1057500091FB0590FEF7A5BEF7F78CFB049A0A991A
:105760001278154B0593401A012A588000F01E83C9
:10577000072A7EF4A3AAF7F77DFB0790FEF7A0BAED
:10578000C04500208C4200203C42002067666666CF
:10579000AC5C0020F86200208E4200209042002085
:1057A00089888888B8500020B062002098000020C6
:1057B00000C0F94400C0F9C4D0440020000000003B
:1057C000002A00F0E781DAED573A9AED566ADAEDF1
:1057D000617AF3499AED607AD1ED005A9AED544A14
:1057E000DAED534AEF4CF048F4EEC63AF3EE046AB1
:1057F000F1EE10FA37EEA65A00F18C8394ED026AAE
:1058000026EE446AF0EE674AE6EE074AF4EEC54A31
:1058100034EEE66AF1EE10FA48BFB0EE656A012A8E
:1058200080ED006A00F0B68194ED066A26EE446AC7
:10583000F0EE674AE6EE074AF4EEC54A34EEE66A51
:10584000F1EE10FA48BFB0EE656A022A80ED016AF7
:1058500000F0A08194ED0A6A26EE446AF0EE674AF1
:10586000E6EE074AF4EEC54A34EEE66AF1EE10FAC7
:1058700048BFB0EE656A032A80ED026A00F08A81B3
:1058800094ED0E6A26EE446AF0EE674AE6EE074AA9
:10589000F4EEC54A34EEE66AF1EE10FA48BFB0EE17
:1058A000656A042A80ED036A00F0748194ED126A3F
:1058B00026EE446AF0EE674AE6EE074AF4EEC54A81
:1058C00034EEE66AF1EE10FA48BFB0EE656A052ADA
:1058D00080ED046A00F05E8194ED166A26EE446A5B
:1058E000F0EE674AE6EE074AF4EEC54A74EEE66A61
:1058F000F1EE10FA48BFF0EE656A062AC0ED056ABF
:1059000000F04881D4ED1A6A66EEC46AF0EE674A88
:10591000E6EE874AB3EE046AF4EEC54A74EEC66A50
:10592000F1EE10FA48BFF0EE656A072AC0ED066A8C
:1059300000F03081D4ED1E6ADFF874B2DFF87482B3
:1059400026EEC44AE4EE077AF4EEC57A77EEC67A1C
:10595000F1EE10FA48BFF0EE657AC0ED077AFEF777
:1059600080BDBCF1000F41F00F8225EE866A8E48A3
:10597000A5EE076AB0EE675AA6EE265ABDEEC56AD6
:1059800016EE107A16EE106A7745A8BF7646B94231
:10599000C8BF0E4606EE106AB8EEC66A012A80ED50
:1059A000006A3FF43BAD94ED046A9DED0D5A25EE7F
:1059B000866AA5EE076AB0EE675AA6EE265ABDEED5
:1059C000C56A16EE107A16EE106A7745A8BF7646BD
:1059D000B942C8BF0E4606EE106AB8EEC66A022A81
:1059E00080ED016A3FF41AAD94ED086A9DED0E5A00
:1059F00025EE866AA5EE076AB0EE675AA6EE265A2D
:105A0000BDEEC56A16EE107A16EE106A7745A8BF8D
:105A10007646B942C8BF0E4606EE106AB8EEC66AB0
:105A2000032A80ED026A3FF4F9AC94ED0C6A9DED17
:105A30000F5A25EE866AA5EE076AB0EE675AA6EE03
:105A4000265ABDEEC56A16EE107A16EE106A774534
:105A5000A8BF7646B942C8BF0E4606EE106AB8EE39
:105A6000C66A042A80ED036A3FF4D8AC94ED106A4C
:105A70009DED105A25EE866AA5EE076AB0EE675ACC
:105A8000A6EE265ABDEEC56A16EE107A16EE106A1C
:105A90007745A8BF7646B942C8BF0E4606EE106AE3
:105AA000B8EEC66A052A80ED046A3FF4B7AC94EDFF
:105AB000146A9DED115A25EE866AA5EE076AB0EECE
:105AC000675AA6EE265ABDEEC56A16EE107A16EE95
:105AD000106A7745A8BF7646B942C8BF0E4606EEA3
:105AE000106AB8EEC66A062A80ED056A3FF496ACE5
:105AF00094ED186A9DED125A25EE866AA5EE076AA6
:105B0000B0EE675AA6EE265ABDEEC56A16EE107ABA
:105B100016EE106A7745A8BF7646B942C8BF0E4652
:105B200006EE106AB8EEC66A072A80ED066A3FF4F0
:105B300075AC94ED1C6A9DED135A65EE865AE7EE3E
:105B4000055AE6EEA57AFDEEE77A17EE904AA645ED
:105B5000A8BFA646A142C8BF8E4607EE90EAF8EE5F
:105B6000E77AC0ED077A56E4DFED106AFEF7D7BE9C
:105B7000B5EEC07AF1EE10FA01F18482B7EE006A58
:105B800036EE477AC6EE076AFEF750BEDFED076ACB
:105B9000FEF7B9BDDFF818B0DFF81880FEF761BC7A
:105BA000543C0020583C0020D84000200000C8424F
:105BB0006C580020C4690020BE494A79002A3EF48E
:105BC00078A9BD4A1278002A3EF473A90B78BB4924
:105BD000DFEDBB4A07EE903A0B88B8EE677A07EE26
:105BE000902A06EE103AF8EEE77AB8EE466A67EECB
:105BF000277AB7EE007A87EE863AB4EEE43AF1EE11
:105C000010FA88BFB0EE643AB4EEC73AF1EE10FA7B
:105C1000B8BFB0EE473AFEF74EB9AA4B5A88FEF726
:105C200085BCBAF8AE2102F57A7292B2FEF77EBC5C
:105C3000A549059107EE102A08461978B0F9040025
:105C400099ED070ABAF81041B8EEC77AF7EE006A84
:105C50000022132986EE879ACAF80C2101F02282CD
:105C60009A4A9B4901EB84060025CAF80051CAF8FC
:105C7000045167EE897A92ED001AD2ED053A92ED61
:105C8000122A92ED173AD2ED091AD2ED0E4A92ED90
:105C9000016A92ED064A92ED0A7AD2ED0F5AD2EDE0
:105CA000132AD2ED186A92ED045AD2ED030A69EE76
:105CB000288A29EE088AE1EE273AA2EE283AE1EE98
:105CC000884AA6EE274AE7EE085A92ED167A92ED38
:105CD0000D6A92ED021AD2ED0C1AC6ED003AE2EE10
:105CE000A86A25EE635A27EE437A92ED0B2AD2ED8D
:105CF000152AC6ED204AA0EEE34A26EE646AD2EDEC
:105D0000143A82ED054AA1EE275AF0EE477AE1EE09
:105D1000E45AA2EE086AE2EEC36AE3EEA87A82EDE4
:105D2000065AC2ED0E5A82ED0F6A86ED403AC2ED78
:105D3000176AC2ED187ACAF80851059B621C02F076
:105D40001F029880AAF81021049BFDF743BD614B08
:105D5000D3ED005AFEF766BF5F4B9FED607AD3ED3F
:105D6000087AF4EEC77AF1EE10FA00F2F3849FEDB0
:105D70005C7A5C4CD4ED037A77EE877AC4ED037AD3
:105D8000FEF7BCBB584D2A78013A0A2A7ED8DFE8D4
:105D900012F069067F06A3050606EE05D4054C053C
:105DA00056065C0042062706474B0593F7F762F854
:105DB0004E49DAF8782109680790821ACAF8780102
:105DC0000598511A8280C180FDF77ABFF7F752F823
:105DD0000A90FDF73ABD464B9B7B002B3EF481AB0E
:105DE000FEF784BBDF003FF547ABFEF78CBBBAF88C
:105DF0008841944240F2F9849AF8A041002C40F086
:105E000065873C4A3C4D92ED007AD5ED007A9AF9CF
:105E10009421CAED637A77EE676A012ACAED617A46
:105E2000CAED606A8AED647A02F0AB80069BCAF81C
:105E30009831324A9FED2A7A92ED005A8AED677ABC
:105E400001228AF89421FFF727B81A201CF08EF956
:105E5000D0B12B4B1B88BBB92A4B45201E681DF0C7
:105E60002FFB0E201DF02CFB304619F0A5FB069EE3
:105E7000304619F0A1FB244A244B12681A603046C0
:105E80000A232B7019F012FC19F024FF2379012B3F
:105E900000F0E384022B7EF47CAD2B78012B7EF4A2
:105EA00078AD1B4B1B78002B7EF473AD19F096FB7D
:105EB000FEF76FBD28420020BE450020A845002007
:105EC000713DAA3FD45E0020D04400200C40002049
:105ED000A03D0020103C0020986800208FC2753C37
:105EE00000000000C04500200C490020FC400020BC
:105EF000984F0020CC620020D83C0020F43C0020C9
:105F000028610020246100203861002030610020D9
:105F10002061002094ED016A26EE646AB0EE674AC3
:105F2000A6EE074AB4EEC54A34EE666AF1EE10FA00
:105F300048BFB0EE656A012A80ED006A3FF42AAEE0
:105F400094ED056A26EE646AB0EE674AA6EE074A4B
:105F5000B4EEC54A34EE666AF1EE10FA48BFB0EE10
:105F6000656A022A80ED016A3FF414AE94ED096A75
:105F700026EE646AB0EE674AA6EE074AB4EEC54A5A
:105F800034EE666AF1EE10FA48BFB0EE656A032A95
:105F900080ED026A3FF4FEAD94ED0D6A26EE646A70
:105FA000B0EE674AA6EE074AB4EEC54A34EE666A1A
:105FB000F1EE10FA48BFB0EE656A042A80ED036A7C
:105FC0003FF4E8AD94ED116A26EE646AB0EE674ADC
:105FD000A6EE074AB4EEC54A34EE666AF1EE10FA50
:105FE00048BFB0EE656A052A80ED046A3FF4D2AD81
:105FF00094ED156A26EE646AB0EE674AA6EE074A8B
:10600000B4EEC54A74EE666AF1EE10FA48BFF0EEDF
:10601000656A062AC0ED056A3FF4BCADD4ED196A85
:1060200066EEE46AB0EE674AA6EE874AB3EE046A0B
:10603000B4EEC54A74EE466AF1EE10FA48BFF0EECF
:10604000656A072AC0ED066A3FF4A4ADD4ED1D6A67
:10605000DFF850B3DFF8508366EEE44AE4EE877A67
:10606000F4EEC57A77EEC67AF1EE10FAB8BFF0EE2C
:10607000657AC0ED077AFEF7F4B9C34DDAED017A1F
:106080009AED006A29886A6977EEA77AF0EE006ACD
:10609000B0EE677AA6EE267A4D1E0AEBC501D6EE63
:1060A000267A08391032F6EE003A27EE237A67EEA8
:1060B000A37A8AED207ACAED217ADFF8E4A2564667
:1060C0000AF1800091ED027A91ED036AD6ED036A40
:1060D000D6ED027A52ED014A12ED025A37EE674AC6
:1060E00076EEC65A77EE277AE4EE845A013DA1F1A6
:1060F0000801E5EE047A06F1080602F1080236EE20
:10610000267A00F10800E4EE877AE5EE475A67EE5A
:10611000A37A25EEA37AC0ED007A80ED017AD1D181
:10612000142F7EF4DFACF6F7A5FE059A974B801A84
:106130005880DAF81441FEF7D5BCDAF818E1BAF85D
:106140001031C3F120025FFA82F8914A03EB4E1638
:1061500002EB86065FEA980201F00587013215011D
:106160008C488D4906EB050C06F1100212ED024A2F
:1061700012ED035A12ED016A12ED047A50ED024A53
:1061800050ED035A50ED016A50ED047A64EE244A52
:1061900065EE255A66EE266A67EE277A1032944538
:1061A00041ED024A41ED035A41ED016A41ED047AA5
:1061B00000F1100001F11001D8D17848A5F11001CB
:1061C0000E4400EB010C514418F0030209D0B6EC68
:1061D000017AFCEC017A67EE277A013AE1EC017A68
:1061E000F5D1002B40F0D787142F7EF47BACF6F767
:1061F00041FE059A654BDAF81441801A5880FEF783
:1062000071BC614D29886B684FEA51084FEA8800DC
:106210005FEAD10E0AEB00020AEB810400F0A180D4
:1062200000F110010EF1010E5B4E02EB0E1E214437
:10623000103203F1100704F1100050ED032A50ED65
:10624000043A16ED043A16ED032A50ED026A10EDF9
:10625000016A16ED020A16ED018A11ED044A11EDEC
:10626000035A52ED044A52ED035A12ED027A52EDEE
:10627000017A51ED020A11ED011A73EE238A72EED2
:10628000221A46ED048A46ED031A70EE268A78EE4D
:10629000061A46ED028A46ED011A74EE848A75EEFE
:1062A000851A42ED048A42ED031A77EE208A77EED2
:1062B000811A42ED028A42ED011A73EE633A75EEDD
:1062C000655A17ED035A32EE623A74EE644A65EE8F
:1062D000631A17ED044A23EE052A64EE652AE3EEFD
:1062E000041A1032964524EE843AA3EE842A06F16D
:1062F000100607F11007A5EE853A00F1100001F134
:106300001001E4EE852A40ED071A00ED082A01EDA0
:10631000073A41ED082A57ED055A17ED065A70EE77
:10632000666A38EE466A30EEC77A71EE677A26EE14
:10633000253A65EEE63A25EE674A67EE054AE6EE4F
:10634000053AA6EE853AA7EE254AE7EEA54A00ED06
:10635000063A40ED053A01ED064A41ED054A7FF463
:106360006CAF1FFA88F81A4641460D481FF092F9A3
:106370006A68414620461FF08DF9049B1A78142A5A
:106380007FF4D7AECFE600BF883D0020D044002088
:10639000A03D0020303F002034220020203F00207C
:1063A000242200206C580020C4690020DFF8848378
:1063B00098F800108E0801F06686D54D06F1010CA4
:1063C0004FEA4C1C05EB0C0E05F12002A5F1700004
:1063D00012ED076A52ED056A12ED037A52ED017A69
:1063E00052ED025A12ED084A52ED064A12ED045AD5
:1063F00026EE066A66EEA66A27EE077A67EEA77AA9
:10640000A4EE046A20329645E4EEA46A00F110007E
:10641000A5EE057AE5EEA57AF1EEC65AB1EEE66A8A
:10642000F1EEC76AB1EEE77A40ED085A00ED076A6F
:1064300040ED066A00ED057ACAD1ACF120022A448B
:106440000AEB061611F0030018BF08320FD052ED08
:10645000017A12ED027A67EEA77A0138E7EE077A41
:1064600002F10802B1EEE77AA6EC017AEFD1142F1F
:1064700001F0A6850134CAF81441FEF7A5BAA54D6E
:10648000A548AA68A98920F05BFD049B1F78142FFA
:1064900001F08285DAF814410134CAF81441EDE5BF
:1064A000DAF818019D499E4C9E4BC20011441044DD
:1064B0008A88196800EE102A643AC82AA8BFC82240
:1064C000782AB8BF782207EE902AB8EEC07AF8EEA4
:1064D000E77A04EB800477EE670A77EE876A67EE67
:1064E000877A20EEA67AB8EE400AC7EE870A2046E1
:1064F000D4F81880E669256A94ED058A1DF096FAAD
:10650000049B84ED058A1F78C4F81880142FE66177
:10651000256201F04B85DAF818218349DAF8144135
:10652000013281FB0213A3EBE27E0EEB4E03A2EBE2
:10653000030E0134CAF818E1CAF81441FFE57B4C98
:10654000002B40F0938694ED006A9DED0C5A78483C
:1065500025EE866AFDEEE44AA5EE076AB0EE675ABC
:10656000A6EE265A14EE901ABDEEC56A16EE107A03
:1065700016EE106A7745A8BF7646B942C8BF0E46E8
:1065800006EE106AB8EEC66A012A80ED006A3DF494
:1065900064AF94ED046A9DED0D5A25EE866AA5EE72
:1065A000076AB0EE675AA6EE265ABDEEC56A16EE29
:1065B000107A16EE106A7745A8BF76468F42B8BFAC
:1065C0000E4606EE106AB8EEC66A022A80ED016A2F
:1065D0003DF443AF94ED086A9DED0E5A25EE866AB0
:1065E000A5EE076AB0EE675AA6EE265ABDEEC56A5A
:1065F00016EE107A16EE106A7745A8BF76468F42DF
:10660000B8BF0E4606EE106AB8EEC66A032A80EDE1
:10661000026A3DF422AF94ED0C6A9DED0F5A25EE0F
:10662000866AA5EE076AB0EE675AA6EE265ABDEE58
:10663000C56A16EE107A16EE106A7745A8BF764640
:106640008F42B8BF0E4606EE106AB8EEC66A042A3C
:1066500080ED036A3DF401AF94ED106A9DED105A90
:1066600025EE866AA5EE076AB0EE675AA6EE265AB0
:10667000BDEEC56A16EE107A16EE106A7745A8BF11
:1066800076468F42B8BF0E4606EE106AB8EEC66A6E
:10669000052A80ED046A3DF4E0AE94ED146A9DEDA8
:1066A000115A25EE866AA5EE076AB0EE675AA6EE85
:1066B000265ABDEEC56A16EE107A16EE106A7745B8
:1066C000A8BF76468F42B8BF0E4606EE106AB8EEF7
:1066D000C66A062A80ED056A3DF4BFAE94ED186ADD
:1066E0009DED125A25EE866AA5EE076AB0EE675A4E
:1066F000A6EE265ABDEEC56A16EE107A16EE106AA0
:106700007745A8BF76468F42B8BF0E46FDF783BED9
:10671000A4220020883D0020242200207840002070
:10672000DC5700205C58002056555555583C002039
:10673000D8400020823D0020306E99BC2716983D3D
:10674000A40DC93F843459BEDB0F4940D06D393A9E
:1067500000000000F0EEE76AB7EE005A35EE665A28
:106760001FED0B4A5FED0B5A1FED0A6A1FED0C7A05
:106770009AED6A0AF1EEC54AE6EE845AF5EEC07A61
:10678000A6EEA56AF1EE10FAA6EE867A48BF5FED96
:10679000127A27EE247A48BF37EEC77A27EE000A2E
:1067A00021F0A0FCB0F5617F00F3DC8607EE900AD3
:1067B000F8EEE76A5FED1B7A66EEA76A07EE904A8D
:1067C000BDEEE67AF8EEE77A17EE103A2033402B6A
:1067D00041F2DF841FED220A21F084FC00B207EEB3
:1067E000900AB8EEE77AFFF7C4BAAF4A02F1500454
:1067F00003E00432944200F069821378262BF8D12A
:106800009578D3789D42F4D2FFF7F6BAA74BD7ED2F
:10681000007A93ED007AF0EEE77AF4EEC77AF1EEC3
:1068200010FA7DF723AAFDF71EBA1CF003FEA04B59
:10683000002105208DE80300A3F1080202915320F6
:1068400019F068FF00287FF421AB9A4A08231060F2
:106850002B702379012B7EF49CA8974E974B1B78C5
:10686000DA0740F10881DAF80C2233689A423FF6E1
:1068700014AB2B78012B3EF48CA8914F3A78002A68
:106880003EF487A80B2B18D801229A4040F603014A
:1068900012EA010416D112F4C06F0ED0093B012B8D
:1068A0000BD845201CF00CFEFF201CF009FE85488B
:1068B0001CF0F2FD20461CF003FE7E4B32685A604D
:1068C0000B232B7000233B70FEF763B8DAF8984176
:1068D000069B1C1BFEF7D0BA764F774E1CF0AAFD24
:1068E0007B68326864339342BFF4D0AA40201CF026
:1068F00085FD00287FF4CAAA3B68734EDFF8E49157
:106900004FF040080DE01CF0DBFDD9F800203B689B
:10691000013A0133B8F10108C9F800203B6001F0E9
:10692000EE84F35C1846002BEDD100234FF0FF32CC
:106930003B6004237A602B708BE71CF07BFD634A7D
:106940000292A2F10C03072601930096A2F108031C
:106950000021143A472019F0DDFE00287FF496AAA2
:10696000544B2E704FF0FF3283E8050071E71CF0A6
:1069700061FD574B002102208DE80300A3F10802BE
:106980000291482019F0C6FE00287FF47FAA494BE7
:106990004FF0FF310622186059602A7059E71CF049
:1069A00049FD4C4A0292A2F10C0328210193009167
:1069B000A2F10A035021163A492019F0ABFE002833
:1069C0007FF464AADBF8003013F0800301F08B84BD
:1069D000384B4FF0FF310522186059602A7038E7B4
:1069E000344A354E52683168C8328A4205D31CF0A9
:1069F00043FD00283FF44AAAA378032B01F08F84BB
:106A00002379012293422A703FF428AF022B7DF4B0
:106A1000C0AFFFF746BA304B1B78002B01F0B782AE
:106A20001A201BF0A3FB002841F0B182244B1B78F5
:106A3000002B41F0AC8209232B70FFF725BA1CF024
:106A4000F9FC19F06FF900283FF420AA1CF014FD9E
:106A500000283FF41BAA214A214B12681A600A231E
:106A60002B70F6E6154B1B78D90701F1E7832379E4
:106A7000012BCBD1104E0DF0EBF900283FF4F3AE13
:106A8000336803F59C530833CAF80C32FFF705BA94
:106A9000094E084A336853601249002313600322E9
:106AA0000B602A70D5E600BF50320020483C002021
:106AB00088950308D0620020306A0020C436002088
:106AC00020610020B8BB0308EC920308409503083E
:106AD00024950308529303080241002038610020E6
:106AE00030610020B8690020964A974CD2ED006AC8
:106AF000964A94ED006A1278CAED636A8AED646A78
:106B0000002A00F0438376EE665A9AF99421CAED82
:106B1000605A0132CAED616A00F0FE86069BCAF82F
:106B20009831002437EE677AFCEEE77A884D8AEDDB
:106B3000677A17EE902AAAF88821FF2295ED005A6D
:106B40008AF89421FEF7A8B9DFED827A824B9AED9C
:106B5000677AC3ED007AC3ED017AC3ED027A7F4B09
:106B6000B0EE676AF0EE673A1968FDF7E3B8F6F73A
:106B700081F9049B05901F78142F05BF784BDAF834
:106B80001441DAF814411C80FCF72CBE754B764A90
:106B9000B3F90430DFED757A82FB0312DB17C3EB28
:106BA000A2031BB208EE103AB8EEC88A28EE278A74
:106BB000B0EE480AF3F7CCFDF0EE408AB0EE480A9A
:106BC000F3F74CFD6A4BD878002800F08D84694AB1
:106BD000BAF90A12B2F9023044F250645B1AA342C5
:106BE00040F3DD87A3F50C43A03B44429C4200F3F5
:106BF000D3878342A8BF0346B2F90020BAF90852EE
:106C00000B4419B2531B44F250629342AAF80A1281
:106C100040F3CD87A3F50C43A03B9C4203DC984294
:106C2000A8BF184604462B191BB207EE903A07EE90
:106C3000101AF8EEE77AF8EEC76A27EEE87A60EE07
:106C4000277AA0EE267AAAF80832E8EEA67ADFEDD7
:106C50004A6A27EE267A67EEA67ABDEEC77AFDEE7F
:106C6000E77A17EE102A17EE903AAAF84821AAF808
:106C70004A31FDF786BE414B1C7804F0010CFDF74C
:106C8000ECBB3F49DFED3F7A0968CAED4A7A11F063
:106C90008053059340F05984DBF8001011F4800311
:106CA000059300F0D28200230593B6EE007A67EEDA
:106CB000877AF4EEE57AF1EE10FAC8BFF0EE675A83
:106CC00040F34384CAED675AFDF775BA1D4A1E4C5E
:106CD000D2ED007A1D4A94ED007A1278CAED637AFB
:106CE0008AED647A002A00F01C8477EE676A9AF9CC
:106CF0009421CAED606A0132CAED617A00F04687DC
:106D0000069BCAF8983100249FED127A104D8AED47
:106D1000677AFF2295ED005A8AF89421FEF7BCB8F5
:106D200073EEC67AB7EE007AF4EEC77AF1EE10FA97
:106D3000CAED4A7A41F31C8184EEA77A8DED0C7A74
:106D4000FDF72EBA50610020DC3C0020D04B002023
:106D5000F03C0020000000009C40002090420020F9
:106D6000D04400203C4200206766666635FA8E3CBF
:106D7000305C00208C5C0020CDCCCC3DC4360020A3
:106D8000B062002000000080002F00F0C78725EED1
:106D9000866AC048A5EE076AB0EE675AA6EE265A84
:106DA000BDEEC56A16EE107A16EE106A7745A8BFDA
:106DB0007646B942C8BF0E4606EE106AB8EEC66AFD
:106DC000012A80ED006A3DF44CAB94ED046A9DED20
:106DD0000D5A25EE866AA5EE076AB0EE675AA6EE52
:106DE000265ABDEEC56A16EE107A16EE106A774581
:106DF000A8BF7646B942C8BF0E4606EE106AB8EE86
:106E0000C66A022A80ED016A3DF42BAB94ED086A54
:106E10009DED0E5A25EE866AA5EE076AB0EE675A1A
:106E2000A6EE265ABDEEC56A16EE107A16EE106A68
:106E30007745A8BF7646B942C8BF0E4606EE106A2F
:106E4000B8EEC66A032A80ED026A3DF40AAB94EDFF
:106E50000C6A9DED0F5A25EE866AA5EE076AB0EE24
:106E6000675AA6EE265ABDEEC56A16EE107A16EEE1
:106E7000106A7745A8BF7646B942C8BF0E4606EEEF
:106E8000106AB8EEC66A042A80ED036A3DF4E9AAE6
:106E900094ED106A9DED105A25EE866AA5EE076AFC
:106EA000B0EE675AA6EE265ABDEEC56A16EE107A07
:106EB00016EE106A7745A8BF7646B942C8BF0E469F
:106EC00006EE106AB8EEC66A052A80ED046A3DF443
:106ED000C8AA94ED146A9DED115A25EE866AA5EEB6
:106EE000076AB0EE675AA6EE265ABDEEC56A16EEE0
:106EF000107A16EE106A7745A8BF7646B942C8BF29
:106F00000E4606EE106AB8EEC66A062A80ED056ADD
:106F10003DF4A7AA94ED186A9DED125A25EE866AF3
:106F2000A5EE076AB0EE675AA6EE265ABDEEC56A10
:106F300016EE107A16EE106A7745A8BF7646B9426B
:106F4000C8BF0E4606EE106AB8EEC66A072A80ED84
:106F5000066A3DF486AA94ED1C6A9DED135A65EE0F
:106F6000865AE5EE075AE6EEA57AFDEEE77A17EEC9
:106F7000902A9645A8BF96469142D8BF714607EE23
:106F8000901AF8EEE77AC0ED077AFDF76ABA822226
:106F9000FDF798BDDFED407AFDF760BDB9F9382007
:106FA000C9F8201007EE902A0121F8EEE77AC9F817
:106FB0006020C9F87C100022012DC9ED1C7AC9EDB2
:106FC0001B7AC9F8742001F0D080B5427EF446A83F
:106FD000B9F93A20C9F8642007EE902A002101226D
:106FE000F8EEE77AC9F82410C9F890200022012DA4
:106FF000C9ED217AC9ED207AC9F8882001F0B9805D
:10700000B5427EF45FA8B9F93C20C9F8682007EEC4
:10701000902A00210122F8EEE77AC9F82810C9F871
:10702000A4200022012DC9ED267AC9ED257AC9F8E0
:107030009C207EF47BA89FED198A032C1CD04FB1B5
:1070400007EE907AF8EEE77AF4EEC87AF1EE10FAED
:1070500001F143811249059BD9F868200968D8805D
:10706000002002EB560292FBF6F6C9F8286088620F
:107070000863C862FEF75CB8B0EE480A21F032F847
:1070800000B2DCE7F7EE006AFDF7D0BBF7EE006A6E
:10709000FDF745BCD840002000000243000000007E
:1070A000744400206E4D6F4E95ED004A95ED057AC3
:1070B000D5ED014A95ED066AD5ED046A95ED035AC2
:1070C000D5ED025A67EE897A06EB8402A4EE277AA0
:1070D00006EB8407A4EEA76A66EEC76AA5EE476AC8
:1070E000E5EEA76A20EE070A85ED056AC5ED066A9A
:1070F00029EE088A69EE288A82ED007A20F0F2FFF4
:10710000D5ED0E5AD5ED176A95ED091AD5ED121A7F
:1071100095ED0F5A95ED187A95ED0A2AD5ED132ABB
:1071200095ED0D6AD5ED167A95ED0C3AD5ED0B3A45
:1071300095ED154AD5ED144AE1EE085A002100B24A
:10714000E8EEA16ACAF80011CAF80411A2EE085AC2
:10715000CAF80811A8EEA27A26EE656A67EEE67A0A
:10716000A3EE655AA3EE886AA6EEC47AE8EEA47A86
:1071700085ED0E5AC7ED205A85ED0F6AC7ED406ABE
:1071800085ED177AC5ED187AFEF7D7BD76EEC65AAB
:10719000F0EE466AB9E4334A4FEA880502EBCE18AE
:1071A0009A0800EB050C554401F0398001324FEA92
:1071B000021E08EB0E0608F110020CF1100005F19A
:1071C000100112ED024A12ED035A12ED016A12ED9E
:1071D000047A50ED024A50ED035A50ED016A50ED29
:1071E000047A64EE244A65EE255A66EE266A67EE56
:1071F000277A1032964241ED024A41ED035A41EDA1
:10720000016A41ED047A00F1100001F11001D8D1BA
:10721000AEF1100290440CEB0200154413F0030E83
:107220003EF4E2AFB8EC017AF0EC017A67EE277A2F
:10723000BEF1010EE5EC017AF4D1FEF7D5BF0A4BA1
:107240001F68B7F93200FEF71EB9B6EE007AF4EE09
:10725000C75AF1EE10FA3FF728ADFCF7ACBF00BFFC
:107260000C400020A03D00209042002094ED006AD8
:107270009DED0C4AC84825EE866AFDEEE43AA4EE80
:10728000076AB0EE674AA6EE264A13EE901AB4EEED
:10729000C45AF1EE10FAB0EE446A88BFB0EE646AE8
:1072A000BDEEC66A16EE107A16EE106A7745A8BFD4
:1072B0007646B942C8BF0E4606EE106AB8EEC66AF8
:1072C000012A80ED006A3DF4C8A894ED046A9DEDA2
:1072D0000D4A25EE866AA4EE076AB0EE674AA6EE6E
:1072E000264AB4EEC45AF1EE10FAB0EE446A88BFF2
:1072F000B0EE646ABDEEC66A16EE107A16EE106A3B
:107300007745A8BF76468F42B8BF0E4606EE106A94
:10731000B8EEC66A022A80ED016A3DF49EA894ED9B
:10732000086A9DED0E4A25EE866AA4EE076AB0EE65
:10733000674AA6EE264AB4EEC45AF1EE10FAB0EE51
:10734000446A88BFB0EE646ABDEEC66A16EE107A73
:1073500016EE106A7745A8BF76468F42B8BF0E4634
:1073600006EE106AB8EEC66A032A80ED026A3DF4A2
:1073700074A894ED0C6A9DED0F4A25EE866AA4EE82
:10738000076AB0EE674AA6EE264AB4EEC45AF1EE9A
:1073900010FAB0EE446A88BFB0EE646ABDEEC66A09
:1073A00016EE107A16EE106A7745A8BF76468F4221
:1073B000B8BF0E4606EE106AB8EEC66A042A80ED23
:1073C000036A3DF44AA894ED106A9DED104A25EE3B
:1073D000866AA4EE076AB0EE674AA6EE264AB4EEC5
:1073E000C45AF1EE10FAB0EE446A88BFB0EE646A97
:1073F000BDEEC66A16EE107A16EE106A7745A8BF83
:1074000076468F42B8BF0E4606EE106AB8EEC66AE0
:10741000052A80ED046A3DF420A894ED146A9DEDE0
:10742000114A25EE866AA4EE076AB0EE674AA6EE18
:10743000264AB4EEC45AF1EE10FAB0EE446A88BFA0
:10744000B0EE646ABDEEC66A16EE107A16EE106AE9
:107450007745A8BF76468F42B8BF0E4606EE106A43
:10746000B8EEC66A062A80ED056A3CF4F6AF94EDE4
:10747000186A9DED124A25EE866AA4EE076AB0EE00
:10748000674AA6EE264AB4EEC45AF1EE10FAB0EE00
:10749000446A88BFB0EE646ABDEEC66A16EE107A22
:1074A00016EE106A7745A8BF76468F42B8BF0E46E3
:1074B00006EE106AB8EEC66A072A80ED066A3CF44A
:1074C000CCAF94ED1C6A9DED134A65EE865AE7EE4B
:1074D000045AE6EEA57AB4EEE75AF1EE10FAC8BF08
:1074E000F0EE647AFCF7A9BF2C4B9FED2D6AB3F93F
:1074F0000020B3F9023007EE902A06EE903AF8EE3B
:10750000E77AF8EEE66A27EEE87A60EE277AA0EEF0
:10751000267AE8EEA67A27EE067A67EE867AFFF7F5
:107520009CBB77EEC76AF0EE477AFFF7E0BBBB8EF5
:107530009FED1C7A07EE903AF8EEE77A1A4B67EE69
:10754000877AC3ED007AFCF7DEBFB7EE007A77EEFC
:10755000677AF4EEE75AF1EE10FA88BFF0EE675A58
:10756000FFF7B0BB07EE904ADFED106AF8EEE77A5E
:1075700066EEA65A9FED0E5A9FED0E6A9FED0E7AAB
:10758000A5EE856A26EEA55AA5EE867AE5EE076A8F
:1075900026EEA70AFFF720B9D84000208C5C002017
:1075A000CDCCCC3D6F12833A9800002084F9223F65
:1075B00092E741B99730083C15A82ABE94ED006ABD
:1075C0009DED0C4AD94825EE866AFDEEE43AA4EE1C
:1075D000076AB0EE674AA6EE264A13EE906AB4EE4A
:1075E000C45AF1EE10FAB0EE446A88BFB0EE646A95
:1075F000BDEEC66A16EE107A16EE101A7745A8BFD1
:107600007146BE42C8BF314606EE101AB8EEC66AD1
:10761000012A80ED006A3DF401AF94ED046A9DED0E
:107620000D4A25EE866AA4EE076AB0EE674AA6EE1A
:10763000264AB4EEC45AF1EE10FAB0EE446A88BF9E
:10764000B0EE646ABDEEC66A16EE107A16EE101A37
:107650007745A8BF7146B742B8BF314606EE101A4B
:10766000B8EEC66A022A80ED016A3DF4D7AE94ED09
:10767000086A9DED0E4A25EE866AA4EE076AB0EE12
:10768000674AA6EE264AB4EEC45AF1EE10FAB0EEFE
:10769000446A88BFB0EE646ABDEEC66A16EE107A20
:1076A00016EE101A7745A8BF7146B742B8BF3146EB
:1076B00006EE101AB8EEC66A032A80ED026A3DF49F
:1076C000ADAE94ED0C6A9DED0F4A25EE866AA4EEF0
:1076D000076AB0EE674AA6EE264AB4EEC45AF1EE47
:1076E00010FAB0EE446A88BFB0EE646ABDEEC66AB6
:1076F00016EE107A16EE101A7745A8BF7146B742FB
:10770000B8BF314606EE101AB8EEC66A042A80EDFC
:10771000036A3DF483AE94ED106A9DED104A25EEA8
:10772000866AA4EE076AB0EE674AA6EE264AB4EE71
:10773000C45AF1EE10FAB0EE446A88BFB0EE646A43
:10774000BDEEC66A16EE107A16EE101A7745A8BF7F
:107750007146B742B8BF314606EE101AB8EEC66A97
:10776000052A80ED046A3DF459AE94ED146A9DED4E
:10777000114A25EE866AA4EE076AB0EE674AA6EEC5
:10778000264AB4EEC45AF1EE10FAB0EE446A88BF4D
:10779000B0EE646ABDEEC66A16EE107A16EE101AE6
:1077A0007745A8BF7146B742B8BF314606EE101AFA
:1077B000B8EEC66A062A80ED056A3DF42FAE94ED58
:1077C000186A9DED124A25EE866AA4EE076AB0EEAD
:1077D000674AA6EE264AB4EEC45AF1EE10FAB0EEAD
